:020000040000FA
:040000006FD00400B9
:101000006F00907E00000000000000009020002093
:10101000AA220020A9BDF9F56C23002000000000E1
:10102000000000006C230020902000200000000041
:101030000000000090200020000000009020002010
:101040000000000090200020902000209020002030
:101050009020002090200020582F00209424002071
:101060000000000090200020902000201E2400207E
:1010700090200020D22300209020002090200020EB
:101080009020002090200020902000209020002020
:101090009020002001A04111B7170040985F3AC688
:1010A000945F3247E39CE6FE3245410182800111A4
:1010B00013078008F337078093F787083EC20100C3
:1010C0000100B7170040930570052380B70413068D
:1010D00080FA2380C7040100010083C6B70493F699
:1010E000F60DA385D704238007049246F3A6068055
:1010F0000100010093760502D5CEF336078093F602
:10110000860836C4010001002380B7042380C70489
:1011100001000100B70614007D89558D88C70100C4
:1011200001000100010023800704A246F3A6068007
:101130000100010073370780137787083AC6010062
:1011400001002380B7042380C704010001000100CF
:1011500001003727004093061005A303D7802380A2
:101160000704B247F3A70780010001009307800836
:10117000F3B7078093F787083ECE01000100B71749
:101180000040130770052380E704130780FA2380CB
:10119000E7040100010003C7B70413670708A3852C
:1011A000E70423800704F247F3A70780010001004A
:1011B0000561828093760504BDC6F336078093F6F9
:1011C000860836C8010001002380B7042380C704C5
:1011D00001000100B7061400938606047D89558D31
:1011E00088C7010001000100010023800704C246F6
:1011F000F3A6068001000100733707801377870884
:101200003ACA010001002380B7042380C70401000B
:1012100001003727004093062005A303D7802380D1
:101220000704D24781B773370780137787083ACC12
:10123000010001002380B7042380C70401000100DE
:1012400098471367070C98C723800704E24719BF24
:101250000111814601468145114506CE97000000E7
:10126000E780605893078008F3B7078093F78708F3
:101270003EC601000100B717004013077005238028
:10128000E704130780FA2380E7040100010003C785
:101290006704136717002383E70423800704B2471A
:1012A000F3A7078001000100F2400561828041112F
:1012B000814601468145114597000000E780A05214
:1012C00013078008F337078093F787083EC40100AF
:1012D0000100B7170040130670052380C70493066A
:1012E00080FA2380D70401000100FD552396B70240
:1012F00023800704A245F3A5058001000100733790
:101300000780137787083AC6010001002380C704CD
:101310002380D7040100010003C767041367170087
:101320002383E70423800704B247F3A70780010063
:10133000010001A0B1473305F50201007D1575FDDF
:101340008280411122C426C206C6AA8401446317C2
:101350009400B24022449244410182800504130566
:10136000803E420497000000E78000FD4180C5B741
:101370009305000273A04580824573901534924016
:101380002242B2424243D2436244F2440255925551
:101390002256B2564257D2576258F25806499649D9
:1013A000264AB64A464BD64B664CF64C065D965DD1
:1013B000265EB65E465FD65F09617300203041113C
:1013C000B7170040985F3AC6945F3247E39CE6FE49
:1013D000324541018280B71700401307000323887C
:1013E000E702854717170000232EF74673002030C9
:1013F000411122C42D6426C24AC006C637190040D6
:101400001304A4AAB704002023208900976000E0F9
:10141000E780203E9C408297976000E0E780603D37
:10142000E5B737370040834747009146BD8B639E41
:10143000D702B73600401306F00F973500009385AA
:10144000E51F9737000083D7672F03C7A6001377E0
:10145000F70F1DE3B7E70400BC4F09468945171590
:1014600000000345A5F7829731A099466394D70001
:10147000834757007300203003C786001377F70FA8
:10148000E365F6FC13851700AE97173800002317A5
:10149000A82A2380E70075B7B787004003C7670015
:1014A000098B6309071003C77700930600031377BE
:1014B0000703630DD708173800000348F87717367D
:1014C0000000130666740547B30606012380E60094
:1014D00083C577001737000013070775429793F508
:1014E000F50F2300B70003C58700973500009385EB
:1014F000A572C2951375F50F2380A5000347070059
:1015000089451377F703630CB70C63E7E50A6306B5
:10151000071A8545630CB7129737000083C7D77148
:101520003307F600034707001377F70F19CB85073A
:1015300093F7F70F3D476363F71A17370000A30DC2
:10154000F76EB787004009472383E700B78700405D
:1015500083C77700E207E18763DE0704973700005F
:1015600083C7976D173700001307076A3E978546B4
:101570002300D700173700001307076B3E97930629
:1015800000032300D700173700001307E7683E97D2
:10159000A14685072300D70093F7F70F3D47636403
:1015A000F71417370000A309F768B7870040094709
:1015B0002383E70073002030930610026300D70EE8
:1015C000930620026305D70693060002E316D7F4BC
:1015D00003C727021377C70F13672700D5A803C7D0
:1015E00067001377070465CB03C7A702173800000D
:1015F00013080843173500001305453A1347070839
:101600002385E70203C7A7021377370F1367870005
:101610002385E702814713070004B305F5008C41D9
:10162000B306F80091078CC2E399E7FEF5B503C74E
:10163000A702134707042385E70203C7A70213770E
:10164000C70F136727002385E702F9B503C76700B3
:101650001377070449C303C767021738000013084C
:10166000E82F1735000013052527134707082383A4
:10167000E70203C767021377370F136787002383D7
:10168000E702814713070004B305F5008C41B30658
:10169000F80091078CC2E399E7FEBDBD03C767025E
:1016A000134707042383E70203C767021377C70FB3
:1016B000136727002383E70285B503C76700137705
:1016C000070411CB03C727021377370F136787006F
:1016D0002381E70291B5238006003DBD97370000C6
:1016E000A38C0754B9BD97370000A387075475BD75
:1016F0002303048015472303E48001002302A48010
:10170000828083076480E3CE07FE23030480828007
:1017100083076480E3CE07FE03454480828083070D
:101720006480E3CE07FE2302A4808280411126C498
:101730004AC24EC006C61377F50BAD47AA892E895B
:101740009544630CF700194597000000E78080FA84
:1017500097000000E78020FB8D444E859700000035
:10176000E78040F9FD59FD1463983401B240A2446A
:101770001249824941018280135509011375F50F01
:1017800097000000E780E0F92209F1BF011126CCA3
:1017900006CEB704080097000000E780C0F61545A4
:1017A00097000000E78000F597000000E78080F6D2
:1017B00097000000E78000F62AC697000000E78047
:1017C00080F432459377150089EB13651500137586
:1017D000F50FF240E24405618280FD14E9F0014515
:1017E000CDBF397126DC4ADA4ED852D656D45AD2F9
:1017F0005ED006DE62CE66CCB7E700E07D5783AAF6
:10180000070022C603AA470023A0E71823A2E7186F
:10181000B7170040130770052380E704130780FA09
:101820002380E70483C74704930B75FFB684E20760
:1018300093FBFB0F8546AA892E8B32893724004003
:10184000E187015763FA76016308D50089461307DB
:1018500000026313D5000157D98F93F7F70FB71C18
:1018600000402382FC0411472303E4801305F00F9A
:1018700097000000E78000E8094C97000000E7802F
:1018800080E863657C15B7050700DA9537870700A0
:10189000795563FEE504B3879500636AF704370B57
:1018A0000800A94733EB65016395F90881E8814495
:1018B00097000000E78020E5268515A8DA85094510
:1018C00097000000E780C0E605090345F9FFFD1415
:1018D000050B97000000E780C0E481C49377FB0FFD
:1018E000E5F797000000E780A0EA69F17D55B7179A
:1018F0000040130770052380E704130780FA238054
:10190000E70403C74704418B2382E704F250B7E79B
:1019100000E023A0571123A24711E2543244525948
:10192000C259325AA25A125B825B724CE24C21615C
:101930008280A547639BF90685691309F00FB306FA
:101940009900B3742B01B6941349F9FFB37499004D
:10195000856B33796901416B9387F9FFB3F72701F1
:1019600099E363FC340193D94900C147E3E637FFAB
:101970003DBF0569C1697D19D9B71305800D63881D
:101980006901130500026384790113051008CA85F3
:1019900097000000E780C0D997000000E78040DF93
:1019A00031D54E99B38434416DBFDA852D4597000A
:1019B0000000E780E0D7CA94E30B99EE0509970091
:1019C0000000E78020D5A30FA9FEFDB79387F9FF9C
:1019D00093F7F70F636DFC0C83C71C0413073008E3
:1019E0006315F706370708006361EB06B3079B0032
:1019F000B706100063FBD704334BEB0089476399AC
:101A0000F9068980D549E38404EADA850945970017
:101A10000000E780E0D111090327C9FF9147232087
:101A2000E48003076480E34E07FE23033481FD173F
:101A3000EDFBFD14110B81C49377FB0FE9FF9700B9
:101A40000000E780E0D461F155B5B717004003C747
:101A50005704B70708001377070219E3B787070091
:101A60007955E376FBE833079B00E3F9E7F841B5E6
:101A70008547E380F9F0DA852D4597000000E7807F
:101A800020CB9389F4FFE38404E297000000E78011
:101A900060C893F7390091EB83260480032709007F
:101AA00093074900E396E6E03E89CE84D9BFB54767
:101AB0006399F9001305900B97000000E78080C33D
:101AC000FDB3B1471305B00AE388F9FE9947639760
:101AD000F904B7050800B365BB002D459700000069
:101AE000E78000C581448D4BA14997000000E78045
:101AF00060C263967401832704802320F900850463
:101B0000E39534FF8327048013172B0163550700E7
:101B10002312F90069BB2322F90051BB9D47639F43
:101B2000F90281451305B00497000000E78040C02A
:101B3000BD442320090023220900FD59970000001D
:101B4000E78040BD93F77400CA9703C70700FD14F0
:101B5000398D2380A700E39334FF91BBA14763979E
:101B6000F90697000000E780A0C28144630D0B00D6
:101B70008D479304C0036308FB00930400056304CE
:101B80008B01930440041375C507E30295D21945F0
:101B900097000000E78000B697000000E780A0B63D
:101BA000054597000000E780E0B426859700000017
:101BB000E78020B7094597000000E78080B69700CE
:101BC0000000E780E0BCE31405CE0DB39147639FAE
:101BD000F9001305600697000000E780A0B19700A8
:101BE0000000E78040B213059009F9B5E38109CC04
:101BF000F1547DB9BD660147173600001306462132
:101C0000938606A685458347060093F7F70F91C391
:101C100082800507E3F9E6FE97370000238AB71EA6
:101C2000DDB77D166206618693178601E18763D46E
:101C3000070001458280931726003307F500AE9711
:101C400018439C4363E7E7007D16E37FF7FC7D556F
:101C5000828005458280FD15E205E18513978501A7
:101C6000618793F7F50F63480700FD15139725006B
:101C70002A97584365D713851700620561858280CE
:101C80003308B5021C4283A80600B335B502C297DB
:101C900033B50701AE98469585486367B5006394F0
:101CA000A50063E3070181480C43C6950CC388C2B5
:101CB0001CC2828081471397870161876343B70005
:101CC0008280139727002A97232007008507E5B70E
:101CD0008147014793968701E18663C5B6001335B6
:101CE0001700828093962700AA9694428507558F05
:101CF000D5B793D755408A07AA979C430545331516
:101D0000B5007D8D828017F3FFDFE702833D2A84D3
:101D100097000000E78060F405C5931725003E9406
:101D20000327C4FF814711EB7D1516053E9542053B
:101D3000418517F3FFDF6700033D05838507E5B79E
:101D40000145C5BF81471397870161876343C7007A
:101D5000828013972700B386E50094422A9785076F
:101D600014C3D5B77D1662066186014793178601B5
:101D7000E18763D50700133517008280931726008B
:101D8000B306F500AE9794429C437D16B58F5D8FE8
:101D9000F1BF8A05AA9501476363B500828083A6D7
:101DA000C5FFF11593D71600D98F9CC11397F60183
:101DB000E5B72A830148014701456343D700828084
:101DC000B387050183A80700B30706019C43C697A4
:101DD000AA976384F80033B517010507B308030118
:101DE000620723A0F80061871108C1BF2A83014759
:101DF0008147014563C3D70082803388E50083288B
:101E00000800330EE600032E0E003388A840330886
:101E1000C8416384080133B508018507B308E300AE
:101E2000E20723A00801E1871107E9B717F3FFDFF5
:101E3000E702232B0111B286B2842E86AA850A8579
:101E400097000000E780C0FA2A84A6850A859700DB
:101E50000000E78020E833348000060413351500C5
:101E6000018D056117F3FFDF6700E32917F3FFDF3B
:101E7000E702A3244111AA89AE8A328BB68402C23A
:101E800002C402C60144131C8401135C8C416349E3
:101E90009C02939B1400FD1B0549138CF4FFF15C1D
:101EA00033048901620461846340740792478E049D
:101EB000CE9423AEF4FE410117F3FFDF67006323E6
:101EC00013192400B30B2B01014A93172A00D6974C
:101ED00083A50B0088437800340050009700000071
:101EE000E78040DA050A93178A01E187F11BE35E78
:101EF000FCFC92474E9905042320F900A2473EC2FC
:101F0000B24702C63EC441B7131A8901135A8A4127
:101F1000131D240093178A01E18763CF970092472E
:101F20000A044E941CC0A24705091379F90F3EC25A
:101F3000B24702C63EC4ADB7B3079A0313152A00D1
:101F400056950841780034005000050AEA97DA9760
:101F50008C4397000000E780E0D26DBF197106C284
:101F600012C416C61AC81ECA22CC26CE2AD02ED219
:101F700032D436D63AD83EDA42DC46DECAC0CEC2C9
:101F8000D2C4D6C6DAC8DECAE2CCE6CEEAD0EED2F9
:101F9000F2D4F6D6FAD8FEDA971500009385058CB0
:101FA0008841E700050092402242B2424243D243B8
:101FB0006244F244025592552256B2564257D257C5
:101FC0006258F25806499649264AB64A464BD64BBD
:101FD000664CF64C065D965D265EB65E465FD65F45
:101FE0000961730020300000972100209381810156
:101FF000175100201301018117F5FFFF1305C500DC
:102000009705002093850500171600201306C6FDCE
:1020100063FAC5008322050023A055001105910530
:10202000E3EAC5FE170502001305C5F89715002061
:102030009385C5FB171600201306C66563FAC50015
:102040008322050023A0550011059105E3EAC5FE92
:102050001715002013050564974500209385052773
:102060006377B500232005001105E36DB5FEFD4241
:10207000739002BC8D4273904280B722000093821D
:10208000828873900230970200209382A2F793E235
:1020900032007390523097520000938202957390F1
:1020A00012346FB0F47573002030397101436EC67D
:1020B00019A0397141536AC866CA62CC5ECE19A0B4
:1020C000397101535AD056D252D44ED64AD826DA54
:1020D00022DC06DE33016140828241114AC026C201
:1020E00022C406C68282B24D4101024D924C224C5E
:1020F000B24B4101024B924A224AB2494101024984
:1021000092442244B240410182803D432A87637356
:10211000C3029377F700BDEFADE5937606FF3D8AE6
:10212000BA960CC34CC30CC74CC74107E36BD7FE30
:1021300011E28280B306C3408A0697020000969699
:102140006780A6002307B700A306B7002306B700E1
:10215000A305B7002305B700A304B7002304B70005
:10216000A303B7002303B700A302B7002302B700FD
:10217000A301B7002301B700A300B7002300B700F5
:10218000828093F5F50F93968500D58D9396050182
:10219000D58D61B7939627009702000096968682A8
:1021A000E78086FA9680C1171D8F3E96E374C3F8C8
:1021B000A5B73367B500FD530D8B79E7B7877F7FF0
:1021C0009387F7F710419441B372F6003363F6003A
:1021D000BE92B3E262006397720C6318D606504158
:1021E000D441B372F6003363F600BE92B3E26200EC
:1021F0006398720A631BD60410459445B372F600C7
:102200003363F600BE92B3E262006391720A631E0A
:10221000D6025045D445B372F6003363F600BE9241
:10222000B3E26200639A72086311D60210499449BE
:10223000B372F6003363F600BE92B3E262006393BA
:1022400072085105D105E30FD6F6131706019397CF
:102250000601631CF7001357060193D706013305E7
:10226000F7409375F50F91E982804183C18333056F
:10227000F7409375F50F91E182801377F70F93F78D
:10228000F70F3305F74082800346050083C605003B
:10229000050585056313D60065FA3305D6408280AF
:1022A00011059105E312D6FE014582802105A105A5
:1022B000E31CD6FC014582803105B105E316D6FC4E
:1022C000014582804105C105E310D6FC01458280AD
:1022D000B717004003C777051377E70FA38BE70411
:1022E000130700F8A38DE7043D47238CE704130789
:1022F0005003A38CE70403C7A7051377D70F238DDB
:10230000E7048280B717004003C7E7020D89411137
:102310001377C70F498F93068008F3B6068093F6AC
:10232000860836C601000100930670052380D70495
:10233000930680FA2380D704010001002387E70277
:1023400023800704B247F3A7078001000100410181
:10235000828041112A83014E930E407E130F001993
:10236000930F400663E56E129308001913034006AD
:10237000B3781503854E0D4FA14F337365020D8958
:102380001335150063EFBE121308F6FF79467298F5
:102390004208135808013307C70213D61700BE07B7
:1023A00032976146B3F6C60213068070B386C60242
:1023B0003697A166F58F42075D8FB716004083C739
:1023C000F60293F70708A303F1000346710083C7E1
:1023D000F60293F70708E394C7FE83477100B71628
:1023E000004093F7F70F6388071293078008F3B74D
:1023F000078093F787083EC401000100B71700402B
:10240000930670052380D704930680FA2380D704AF
:102410000100010023AA070383C6170393E60608F9
:10242000A388D70223800704A247F3A707800100EF
:1024300001001166B71700407D16D45BC85F938515
:102440004703A98EF18EF5FA93068008F3B606804D
:1024500093F6860836C601000100930670052380B6
:10246000D704930680FA2380D7040100010098C1A5
:1024700003C7170313670704A388E7022380070431
:10248000B247F3A7078001000100410182807D135C
:102490003368E3039308E016630E08003368F30320
:1024A0009308D016630808009378330093B8180097
:1024B0009388D81633081E01131E0801135E0E01FF
:1024C00055B56393E5030548638608000148630337
:1024D00003002A8871087298FD15131E0801C205B1
:1024E000135E0E01C18179BD13F8150063F4BF00BE
:1024F0007908D5B713381800E5BF83C7F60293F7FC
:102500000708A303F1000346710083C7F60293F79F
:102510000708E394C7FE8347710093F7F70FF1DFD5
:10252000E9B531714AD966CB06DF22DD26DB4ED70D
:1025300052D556D35AD15ECF62CD6AC96EC7AA8C26
:1025400002D897100000E78020B12A8993078008FD
:10255000F3B7078093F787083EDA01000100B71749
:102560000040130770052380E704130780FA2380D7
:10257000E7040100010003C7F7021377770FA38771
:10258000E70203C7F70213678700A387E7022380E8
:102590000704D257F3A70780010001000545970003
:1025A0000000E78060D6130780C13347E902116A53
:1025B00093070AE893065002BD69930BA004814A71
:1025C000014B13048008930470057D1AB347F90288
:1025D0003307D7023EC0FD873ECC938709A69309F7
:1025E000803E3347F7023AC27D873AC43347390306
:1025F0008549B399990193D93940B306D702B30BF2
:102600007703B3C6F602B3CBFB0236C6FD8636C8E7
:1026100093D6FB4136CEB7460F0093860624334946
:10262000D9028566938606FAB3969601B389E902C4
:10263000130760553309D90293060010B389E902E4
:102640003349D902B3C9F9029316390036CA37198A
:102650000040FD8636D0930D090493D7F9413ED250
:10266000F336048093F6860836DC010001009307F8
:1026700070052380FD00930680FA2380DD000100B1
:1026800001008346390593F6860FA309D9048346D2
:10269000390593E61600A309D90423800D00E256FC
:1026A000F3A6068001000100130C80FA116DF336C9
:1026B000048093F6860836DE01000100930770055A
:1026C0002380FD0023808D01010001008346390530
:1026D000216693E60602A309D90483560905B3E6E9
:1026E000A6012318D90483560905D18E2318D904CD
:1026F00023800D00F256F3A60680010001008346F8
:10270000390593F606026381061A03463905218AC4
:102710006DDE081897100000E7800098733604807B
:1027200013768608B2C20100010023809D00238039
:102730008D0101000100B717004003C6370513766D
:10274000F60DA389C70403C6370513660602A389DD
:10275000C704835609052166B3E6A6012318D904E8
:1027600083560905D18E2318D90423800D0096467F
:10277000F3A60680010001008346390593F60602A0
:10278000638B061483463905A18AEDFE970000206D
:10279000E7806090AA8636D497000020E780A08F5B
:1027A000A256E30AD5FE835609054255B3E6A601B3
:1027B0002318D90497100000E780C08F834639059D
:1027C000A18AEDDE03560905834629058247337643
:1027D000CA00B306DA0293D5F641B296B388F64042
:1027E000E24733B8C6002E983308F840A247B3B684
:1027F00016013308D84063C70701631DF8009247EC
:1028000063FA1701C247634FF80E63950701B24799
:1028100063EAF80E894663E9660FF24693151800DD
:1028200013D3F8015E8613951800B365B30042D642
:1028300046D497C00100E780C0DC3258050B137BFB
:10284000FB0F63470001631A0838A25863870838F2
:1028500013081500B336A800B69513D6F5013298C3
:10286000B336C800AE9613581800FE06B3E606014C
:102870007336048013768608B2C6010001002380F7
:102880009D0023808D01010001000356C902B2960C
:10289000C206C1822316D90223800D00B646F3A6D4
:1028A00006800100010021B5F336048093F6860806
:1028B000B6C00100010023809D0023808D0101002E
:1028C00001008346390593E60602A309D904238053
:1028D0000D0086460DB5F336048093F68608B6C41F
:1028E0000100010023809D0023808D010100010073
:1028F0008346390593E60602A309D90423800D0017
:10290000A646BDB5E30B0BF0F336048093F68608BC
:10291000B6C801000100930680FA23809D00238041
:10292000DD00010001008346390593F5FC0F93F6A5
:10293000860FA309D90483463905CD8EA309D9048E
:1029400023800D00C646F3A6068001000100130592
:1029500080FA03463905930639051D8A631C9629BA
:102960007336048013768608B2CC0100010013068A
:1029700080FA23809D002380CD000100010003C662
:1029800006001376F60D2380C60003C60600136604
:1029900006022380C600835609051166D18E2318CE
:1029A000D904835609052166D18E2318D9042380C2
:1029B0000D00E646F3A6068001000100130680FA2A
:1029C0008346390593F60602638006268346390559
:1029D000130C3905A18AFDDA081897000000E7807A
:1029E000A06BF336048093F68608B6D00100010090
:1029F000930680FA23809D002380DD000100010002
:102A000083460C00116693F6F60D2300DC00834626
:102A10000C0093E606022300DC0083560905D18EE4
:102A20002318D904835609052166D18E2318D904A9
:102A300023800D008656F3A60680010001001306D0
:102A400080FA8346390593F60602638A0620834698
:102A50003905A18AEDFE97F0FF1FE780C0632A8C3D
:102A600097F0FF1FE7802063E30C85FF835609057D
:102A700011664255D18E2318D90497000000E780D3
:102A800060638346390513063905A18AFDDAF336FA
:102A9000048093F68608B6D401000100930680FAFC
:102AA00023809D002380DD00010001008346060095
:102AB00093F6F60D2300D60023800D00A656F3A64C
:102AC0000680010001008356090503462905D24707
:102AD000B376DA003306CA021305800C9355F6412B
:102AE0003696330DF6408257333CD6002E9C333653
:102AF000A601330CFC40330CCC40330885039256BE
:102B00004E86B335A5033305A503C29597C00100D2
:102B1000E78020AF63468001631E0C16630C0D1620
:102B2000130615003335A6002E959356F5013696FB
:102B3000B335D600AA959396F50105828585D18E89
:102B40006346B000639D051A638B061A0356C902DB
:102B500015823305D6003336C500B2956348B00000
:102B6000639105241306F00F637DA622894663F363
:102B7000561593078008F3B7078093F78708BED6EA
:102B80000100010037170040930770052300F70488
:102B9000930780FA2300F704010001008356C7025F
:102BA00089678117D58FC207C1832316F7022300D7
:102BB0000704B657F3A7078001000100FA506A54D2
:102BC000DA544A59BA592A5A9A5A0A5BFA4B6A4C49
:102BD000DA4C4A4DBA4D296182801308F5FF33352E
:102BE000A800FD152E951356F5013298B336C8008E
:102BF000AA9695B9F336048093F68608B6CA010002
:102C0000010023809D002380AD0001000100834668
:102C10003905CD8EA309D90423800D00D646F3A62D
:102C200006800100010035B3F336048093F6860870
:102C3000B6CE0100010023809D002380CD0001005D
:102C400001008346390593E60602A309D9042380CF
:102C50000D00F646F3A606800100010095B3F33699
:102C6000048093F68608B6D20100010023809D00FF
:102C70002380CD00010001008346390593E606025A
:102C8000A309D90423800D009656F3A606800100FF
:102C9000010045BB9306F5FF33B5A600FD152E9543
:102CA0009355F501AE96B3B5B600AA951396F50106
:102CB000858269B5F336048093F68608B6D801009C
:102CC0000100930680FA23809D002380DD0001002F
:102CD00001008356C9020566011693F6F60FD18EE0
:102CE000C206C1822316D90223800D00C656F3A660
:102CF000068001000100850A93FAFA0F95B233E6C7
:102D0000B60045C20356C9023305D0403338A0008F
:102D1000B305B040B385054115826345B000D1E1EC
:102D20006371A608894663F0560593078008F3B7D8
:102D3000078093F78708BEDA01000100B71700404B
:102D4000130770052380E704130780FA2380E70444
:102D50000100010003D7C7027D8B2396E702238081
:102D60000704D65781BDF336048093F68608B6DC97
:102D700001000100930680FA23809D002380DD007E
:102D8000010001008356C9020566011693F6F60F8D
:102D9000D18EC206C1822316D90223800D00E656C9
:102DA000B9B793078008F3B7078093F78708BEDEAB
:102DB0000100010037170040930770052300F70456
:102DC000930780FA2300F704010001000356C702AD
:102DD00093975600B297C207C1832316F7022300C8
:102DE0000704F657C1BB914763EEB70217D701003E
:102DF0001307871E8A05BA959C41BA978287B71731
:102E0000004003A7470B1345F5FF698F23AAE70A84
:102E100003A7070B698F23A8E70A03A7070A798D81
:102E200023A0A70A8280B717004083A6470B134749
:102E3000F5FFF98E23AAD70A83A6070B558D23A881
:102E4000A70A83A6070A758F23A0E70A8280B7170F
:102E5000004003A7470B498F23AAE70A03A7070BE4
:102E60001345F5FF45BFB717004083A6470B13472F
:102E7000F5FF758F23AAE70A03A7070A598D4DB7F7
:102E8000B717004003A7470B498FEDB7914763EE93
:102E9000B70217D70100130767158A05BA959C4139
:102EA000BA978287B717004003A7470D1345F5FF70
:102EB000698F23AAE70C03A7070D698F23A8E70CE6
:102EC00003A7070C798D23A0A70C8280B7170040B9
:102ED00083A6470D1347F5FFF98E23AAD70C83A6C7
:102EE000070D558D23A8A70C83A6070C758F23A06B
:102EF000E70C8280B717004003A7470D498F23AA2C
:102F0000E70C03A7070D1345F5FF45BFB7170040B2
:102F100083A6470D1347F5FF758F23AAE70C03A778
:102F2000070C598D4DB7B717004003A7470D498FC0
:102F3000EDB7797122D43714004026D24AD0035914
:102F400024028354040206D64209C2044ECE52CC57
:102F500056CA13590901C1802DE11379F9F793F489
:102F6000F49F4209C20413590901C18093078008E4
:102F7000F3B7078093F787083EC401000100930769
:102F800070052300F404930780FA2300F404010081
:102F90000100231124032310940223000404A247F8
:102FA000F3A7078001000100B25022549254025945
:102FB000F249624AD24A45618280B7F507008146EC
:102FC0003000B105194597000020E7808081A247B5
:102FD00013972701E34A07FC1369090893E40440A7
:102FE00093098008F3B7098093F787083EC0010072
:102FF0000100930A700523005405130A80FA230088
:10300000440501000100231124032310940223002E
:1030100004048247F3A7078001000100294597F0C7
:10302000FF1FE7802031F3B9098093F989084EC268
:1030300001000100230054052300440501000100A4
:103040008357040293E707202310F40223000404AB
:103050009247B9B7B7170040884742054181937737
:10306000050491EB9377F5013755E80113050580C9
:103070003345F50282809377050C130700046397AC
:10308000E7009377F50137459C1CCDB72165130503
:1030900005D0828037E700E01C435443A183E20659
:1030A000D58F1CC1FD572320F7182322F7188280E3
:1030B00013178500B7E700E023A0E710618123A282
:1030C000A7108280B7F700E08847CC47828081470D
:1030D00037370040A14663C4C7003285828003456C
:1030E000B740E38EA6FE3385F5000345050085074E
:1030F0002304A740CDB797070020938727EF9C4371
:10310000173700201307871C3E95636EE5001737BD
:1031100000201307274F6368A70017070020232705
:10312000A7EC3E858280FD57EDBF8280411122C40D
:1031300006C62A8497000000E78000F22947B307FB
:10314000E502B2408D83B3D7870222449507B3D7F7
:10315000E70237370040C207C1832316F700410159
:103160008280411137150E0006C697000000E780E7
:1031700020FCB7370040130770F82381E7000D47A4
:10318000A381E70013070004A380E7000547238716
:10319000E700B24041018280373700408347270073
:1031A0001A0593F7F703C98F93F7F70F2301F70079
:1031B0008280B737004003C7170019C9D98DA38093
:1031C000B70003C70700136787002380E7008280EA
:1031D00093C5F5FFF98DA380B7008280AE872A875B
:1031E000B736004021463738004089E71703000012
:1031F0006700E3F383C8B600E30916FF05078348B9
:10320000F7FFFD17C20723041801C183F9BF41115D
:1032100022C406C62A8497000000E780E0E329471D
:10322000B307E502B2408D83B3D7870222449507E6
:10323000B3D7E70237370040C207C1832316F740F0
:1032400041018280716541111305052006C6970072
:103250000000E78000FCB7370040130770F82381B7
:10326000E7400D47A381E74013070004A380E74030
:1032700005472387E740B24041018280CC4141119C
:1032800006C6328503C6150083C5050022064D8E8D
:1032900042068D654186138875A2630C0611634B47
:1032A000C804138845A26300060D634AC8009385CD
:1032B00035A26301B6082390060029464DA0138865
:1032C00055A26305060D938565A2E316B6FE8D45EE
:1032D0001D4663E6E5081146198E63F3C7003E8676
:1032E000B7E704002390C600FC4797D501009385FB
:1032F00025D29DA0138895A263030611634E060D87
:103300001388A5A263000613938505A5E315B6FAF5
:1033100099451D4663E5E504198E63F3C7003E86B3
:10332000B7E704002390C600FC479705002093856B
:1033300025D61DA09D451D4663E3E5022146198E55
:1033400063F3C7003E86B7E70400FC472390C6003E
:103350009705002093858534BA9582970146B2403F
:10336000328541018280AD451D46E3EAE5FE3146E6
:10337000198E63F3C7003E86B7E704002390C600AA
:10338000FC4797D50100938525CBF9B7B1451D467C
:10339000E3E7E5FC3546198E63F3C7003E86B7E7E1
:1033A00004002390C600FC4797D501009385C5C94A
:1033B00065B78D451D46E3E4E5FA1146198E63F3C2
:1033C000C7003E86B7E704002390C600FC4797D5A8
:1033D00001009385A5C449B78D451D46E3E1E5F895
:1033E0001146198E63F3C7003E86B7E704002390A9
:1033F000C600FC4797D501009385C5C6B1BFA5455A
:103400001D46E3EEE5F42946198E63F3C7003E86B8
:10341000B7E704002390C600FC4797D501009385C9
:10342000A5C01DBFB5451D46E3EBE5F23946198E33
:1034300063F3C7003E86B7E704002390C600FC474D
:1034400097D501009385C5BB01BFB7E7040003A36F
:103450000713970600209386A6C24146A545170587
:1034600000201305E5B80283797126D252CCAE84D0
:103470002A8A97D501009385E5C017D50100130569
:10348000E5C206D63AC622D44AD0368432894ECE18
:1034900056CA97B00100E7800062A28517D50100E7
:1034A0001305C5C197B00100E780E060294597B0DA
:1034B0000100E780206583C7840093F70702F9EFD6
:1034C00083C904008947054532476391F90AD4400E
:1034D00083C7160083C60600A207D58FC166138670
:1034E00016FE638DC7028D16638BD7088D66938693
:1034F00026902945639CD706B7E70400A28622548C
:1035000003A34714B250F249D24A4A86A68502590B
:1035100092545285624A8547456102832D4539E7B9
:10352000130A0002354563638A04B7EA040083A7DF
:10353000CA04C8442286CA8582978149630A440125
:10354000C84483A78A0433068A408145229582971E
:10355000970700209387872F9C43014581CB9C438D
:1035600091C74E852286CA8582970145B250225462
:1035700092540259F249624AD24A456182802D45ED
:1035800075F79307700F3545E3E287FEB7E7040050
:10359000FC47C8442286CA8582975DBF2145F9B79A
:1035A0002D455DE703C505000947631FE50803A82E
:1035B0004500411106C6034718003285034608003E
:1035C00022074168518F930828FE6307170563E9B6
:1035D000E80005186303070323900600294591A816
:1035E000130648FE630AC7041518E31707FF1546BC
:1035F0003E87637BF600154701A8130600023E874D
:103600006374F60013070002B7E704002390E60096
:10361000FC471316070111A83E8691C30546B7E77C
:103620000400FC472390C6004206CC4541828297A5
:103630000145B24041018280130600083E87E375D0
:10364000F6FC13070008C9B72390060005458280E1
:103650008280416779176304E504411122C406C6DC
:1036600085472A84639FF500B7E70400228522443A
:10367000B24003A38713970500209385651C410181
:10368000028389476399F500B7E7040083A7070B16
:103690008545829771D9B24022444101828082805F
:1036A000411122C437E404008327841326C2AA846C
:1036B000416506C697050020938585187D1582977C
:1036C0008327C40A170500001305E5F8858882974B
:1036D00095C0032304132244B2409244970600206D
:1036E000938686AC4146C545170500201305C59A4B
:1036F00041010283B240224492440145410182804B
:1037000019C59707002023A3A714014582804545CA
:103710008280011122CC06CE26CA4AC84EC69147E5
:10372000094463ECA70417D70100130767940A053F
:103730003A951C41AE84B285BA9782879387F4FF8D
:10374000C207C1837D4761446369F702B7E904009A
:1037500083A7C904170900201309C9F426864A85DE
:1037600082971306000201446389C40083A7890479
:10377000058E81453305990082972285F240624487
:10378000D2444249B2490561828085476144E3964B
:10379000F4FEB7E70400FC470546170500201305B3
:1037A00065F282970144D1BF9307700F6144E3969D
:1037B000F4FCB7E70400FC471306700F1705002060
:1037C000130585F0F9BF930700086144E397F4FA05
:1037D000B7E70400FC47130600081705002013058F
:1037E00025FEC1B795476144E399F4F8B7E70400B3
:1037F000FC471546170500201305C5045DB74111A8
:1038000026C2B7E4040083A7C41322C44AC006C674
:103810002E84970500209385A5022A898297058921
:1038200005C5970700209387278783D7A70BA28515
:1038300003A3440D2310F4002244B24092444A856D
:103840000249014641010283B240224492440249A6
:1038500049454101828097070020238B07FE970787
:10386000002023A907FEB717004003A7070CB706DF
:10387000C0FFFD16758F23A0E70C03A7070DB70641
:103880004000558F23A8E70C03A7070C3D9B23A0FE
:10389000E70C03A7070D1367070123A8E70C828035
:1038A000B717004003A5470C83A7470C5981134560
:1038B0001500C18B058999E3136525009707002042
:1038C00083C707F96380A702970700202382A7F820
:1038D00011C9970700209387E7F703A30700630345
:1038E000030002838280114517F3FFFF6700A3C323
:1038F000011122CC06CE3714004026CA4AC84EC653
:1039000052C483447405034AB405834984050349BA
:10391000940597F0FFFFE780E09B8347A40593F4AD
:10392000F40F137AFA0F93E71700230DF40493F9B9
:10393000F90F1379F90FB717004003C7A705058BD7
:103940006DFF03D5C705A38D4705238C3705A38CD1
:103950002705A38B9704F2406244D2444249B249FE
:10396000224A0561828041119397050122C406C64F
:1039700026C2C1872E8463DC0700B7E40400FC5430
:10398000829719C1BC5482972165218D15A893F7A0
:10399000150013C515008DE793F725009DC7970007
:1039A0000000E78020F0B7E70400BC4F1306000AD0
:1039B000894517050020034565EA829713452400D1
:1039C000B24022449244410182809397250163D8FA
:1039D0000702B7E4040083A7C41E82979700000083
:1039E000E780A0F0BC4C3756070013060630896507
:1039F00017050020034585E68297096579B79397F7
:103A000015010145E3DE07FA17C50100130505732B
:103A100097B00100E7800022B7E70400BC4F13060F
:103A20000064916517050020034545E38297116501
:103A3000A9BF1D71A2CC37E404005C5C485886CE57
:103A4000494697C501009385E56A829711E917C534
:103A500001001305656B97B00100E780A01D01A070
:103A6000B7F600E0795798CAFD57DCCA0567B7E793
:103A700000E023A0E7101306F00290C223A0E7188D
:103A80000100010037070020184713060004814594
:103A90009706002023A2E6DC4157A38AE7403C4476
:103AA00008088297970700209387C7783EC88567E4
:103AB00013870740938757D1231AE1002312F1029D
:103AC0001307B00F97F7FFFF938707602310E102FA
:103AD0003ED81547970700009387C7E1B7F5070061
:103AE000A30FE1003EDC0547970700009387E7DF5F
:103AF00081463000E10519452301E1023EDE97F0E1
:103B0000FF1FE78000CE18088147994630003E9697
:103B10000346060085070507A30BC700E398D7FEF9
:103B2000C24791C70357410185676373F70001A03E
:103B3000B7E7040083A7470A08088297AA8511C936
:103B400017C501001305855D97B00100E780A0F659
:103B500001A0F640664425618280411126C2B7E487
:103B6000040083A7040806C622C417050000130535
:103B7000C5DF829717040020130444CE2300A4005D
:103B800097000000E780800297000000E780E0CC0B
:103B900003450400224403A38405B2409244130663
:103BA0000032896541010283797106D622D4130758
:103BB0008008F337078093F787083EC201000100B1
:103BC000B7170040930570052380B704130680FAE9
:103BD0002380C7040100010083C6F70293F6A60FF5
:103BE000A387D702238007049246F3A6068001002C
:103BF000010073370780137787083AC4010001007A
:103C00002380B7042380C7040100010003C7F70223
:103C100013672700A387E70223800704A247F3A7BF
:103C2000078001000100054597E0FFFFE780C06DB8
:103C300097000000E78060CB014781468147054639
:103C400085451305407E97E0FFFFE780C07037E4AD
:103C500004003C446800514681458297B707C0A8DC
:103C60003EC8B787E803938707D03ECA97E7FF1F90
:103C70009387E7743EC67C5868008297B2502254FE
:103C800045618280411197D50100938565AD17C5C7
:103C900001001305A54106C697B00100E780A0E129
:103CA00017D50100130585C497B00100E780A0E097
:103CB000B2402945410117B301006700A3E4411157
:103CC00097D50100938505AB17C501001305053E87
:103CD00006C697B00100E78000DE17D50100130586
:103CE000A5BF97B00100E78000DDB2402945410142
:103CF00017B30100670003E1411122C406C68347E0
:103D000005002A849DC797D50100938565AC17C52A
:103D100001001305A53997B00100E780C0D94C40D8
:103D200017D501001305C5CE97B00100E780A0D8D4
:103D30003DA058410DEF97D50100938565A917C5A2
:103D400001001305A53697B00100E780C0D617D54E
:103D50000100130565CD97B00100E780C0D522446E
:103D6000B2402945410117B301006700A3D9A167FB
:103D70009386D7036313D70297D50100938545A592
:103D800017C501001305853297B00100E780A0D266
:103D900017D50100130545CA7DBFED0797D5010072
:103DA000938505A317C5010013054530631BF70074
:103DB00097B00100E78020D017D50100130505C991
:103DC00059BF97B00100E78000CF4C4017D50100E4
:103DD0001305C5C991BF411197D501009385C59AB7
:103DE00017C501001305852C06C697B00100E780B2
:103DF00080CCB2402945410117B30100670083D050
:103E0000797122D426D24AD02E842A898145B2845F
:103E10004800714606D697E0FFFFE780402F97F7EE
:103E2000FF1F93876759DC4783D7070023142101BD
:103E30002313F10097500000E78060E98547A30550
:103E4000F1009307401F3EC6FD572305A100230A3A
:103E5000F10097500000E780C0FB2686A28548004D
:103E600097500000E78080E9B250225492540259E2
:103E700045618280972700202391078C97170020A7
:103E8000238A077AB7E70400BC47411106C64146BA
:103E90008145170500201305252882971707002064
:103EA000034787299307F00A6315F7029307F0F891
:103EB0008945170500201305252817070020230D25
:103EC000F72697070020A389072697600000E78060
:103ED000A09B97600000E78020C78145370504005C
:103EE0009707002023A80722970700202391072285
:103EF00097070020238E072097070020239C071890
:103F000097070020239A071697070020239F071E74
:103F100097070020239A072097300000E780602E43
:103F2000014597600000E780209F97D501009385A9
:103F3000258817C501001305651797B00100E780B4
:103F400080B717D501001305A5B897B00100E78029
:103F500080B6B2402945410117B30100670083BA1A
:103F60004111814617F6FF1F130646428545170586
:103F700000200355251006C697C00000E780602585
:103F800015C997D501009385658317C501001305F1
:103F9000E51197B00100E78000B217D501001305C5
:103FA00025A397B00100E78000B1294597B0010033
:103FB000E78040B597D501009385458017C501007E
:103FC0001305C50E97B00100E780E0AE17D50100DC
:103FD000130545A197B00100E780E0AD294597B0F2
:103FE0000100E78020B217F5FF1F1305E53C5C4593
:103FF00005472390E70097400100E780E0D597C58B
:1040000001009385A57B17C501001305250A97B00C
:104010000100E78040AA17D501001305E59D97B080
:104020000100E78040A9B2402945410117B30100D2
:10403000670043AD011122CC06CE26CA4AC84EC63F
:1040400093F715002E84C1C7854497000000E780D0
:1040500060F197170020238F975C930710F81707DC
:104060000020230BF70C9707002083D76700170762
:104070000020A303F70C9145A18317050020130529
:10408000A50B17070020230AF70A97070020A3862D
:10409000070A97500000E780207F970700202387BA
:1040A0009706B7E70400BC4F0D661306062093057C
:1040B000001017F5FF1F0345E57A8297134514009A
:1040C000F2406244D2444249B2490561828093F78A
:1040D0000510B9CF054597600000E780E08317150C
:1040E00000200355856597500000E780204F970713
:1040F000002083C7A70195C7170500201305C50138
:104100009707002023840700034715008347050015
:10411000D98F0347F500D98F89C797200000E78022
:10412000A03997200000E78060271345041049BF9D
:1041300093F72500E9CF17070020035747FD69C70C
:10414000AD64B71900409384A4AA23A099009706F0
:104150000020938626FC944297D7010093874799C5
:10416000170600200346C6FA8145170500201305EF
:10417000A5FA97700000E780802123A0990097F7A7
:10418000FF1F239FA7122A8941C197C5010093856C
:10419000A56917C50100130565F197B00100E78017
:1041A0008091CA8517C501001305050897B0010065
:1041B000E7806090294597B00100E780A0949707B9
:1041C0000020239607F4930710F817070020230513
:1041D000F7F69707002083D7A7E917070020A30D5C
:1041E000F7F4A183170700202309F7F491458D47C1
:1041F00017050020130545F417070020A30FF7F259
:1042000097500000E78040681345240055BD93F7A0
:104210004500D1C397C501009385056117C501000D
:104220001305C5E897B00100E780E08817C50100D5
:104230001305450197B00100E780E087294597B055
:104240000100E780208C930720F817070020230542
:10425000F7EE9707002083D7E7E317070020A30DA9
:10426000F7ECA183170700202309F7EC8547170710
:104270000020A304F7EC97500000E78080B91705F1
:104280000020130565EB914597500000E780C05F63
:104290001345440035B593F78500A9C797C50100BC
:1042A0009385855817C50100130545E097B00100B7
:1042B000E780608017C50100130505FA97A001008B
:1042C000E780607F294597B00100E780A0839707CA
:1042D0000020239E07E297700000E780201B134513
:1042E0008400F9BB93F70501D1C38545170500206C
:1042F000035545DA97600100E780E0D097C50100DB
:104300009385855217C50100130545DA97A0010072
:10431000E780607A17C50100130545F597A00100F5
:10432000E7806079294597A00100E780A07D930789
:1043300030F8170700202301F7E09707002083D704
:1043400067D517070020A309F7DE1705002013051E
:10435000A5DEA1838D45170700202300F7DE9750C7
:104360000000E78060521345040199BB93F70502F2
:10437000D1C797C501009385254B17C501001305CB
:10438000E5D297A00100E780007317C5010013056F
:1043900025F097A00100E7800072294597A0010051
:1043A000E7804076930740F8170700202306F7D8E8
:1043B0009707002083D747CC17070020A30EF7D616
:1043C000A18317070020230AF7D685471707002087
:1043D000A305F7D697070020239007CA975000003F
:1043E000E78020A317050020130505D591459750B8
:1043F0000000E780604913450402D9B193F7050432
:10440000FDC397C501009385254217C5010013051B
:10441000E5C997A00100E780006A17C501001305F0
:10442000A5E897A00100E7800069294597A0010051
:10443000E780406D9707002083C707D01307700AF5
:104440006386E7061307800A638CE7081307600A90
:104450006393E704930760F817070020230EF7CC57
:104460009707002083D767CA17070020A306F7CC59
:10447000A183170700202302F7CC854717070020E8
:10448000A301F7CCB145170500201305E5CA9750E5
:104490000000E780603F97500000E7808097134559
:1044A000040497070020239207C619B9930770F8F0
:1044B000170700202302F7C89707002083D7E7C417
:1044C00017070020A30AF7C6A183170700202306B9
:1044D000F7C6854717070020A302F7C6994565B7B9
:1044E000930780F8F1B793F705080145E38A07BC05
:1044F00097C501009385453317C50100130505BB1A
:1045000097A00100E780205B17C50100130545DB7C
:1045100097A00100E780205A294597A00100E78075
:10452000605E9307A0F8170700202307F7C09707DE
:10453000002083D767BF17070020A30FF7BEA18312
:1045400017070020230BF7BE854717070020A30697
:10455000F7BE97070020239907BC97500000E7801B
:10456000408B17050020130525BD9145975000008D
:10457000E780803113450408A1B6411122C497C5D4
:104580000100938525262A8417C50100130505B26D
:1045900006C697A00100E78000524C4017C50100F5
:1045A0001305854097A00100E780E050294597A0BA
:1045B0000100E7802055034704009307F00F631FB5
:1045C000F70297C501009385E52117C50100130582
:1045D000E5AD97A00100E780004E4C4017C50100F3
:1045E0001305853D97A00100E780E04C2244B240CE
:1045F0002945410117A301006700C350B24022447E
:1046000041018280411122C426C22E84AA8497C50A
:1046100001009385E51817C50100130525A906C6F5
:1046200097A00100E780204917C501001305C54880
:1046300097A00100E7802048294597A00100E78066
:10464000604C97070020239797A29707002023919B
:1046500087A2854797C501009385851417C501007A
:104660001305C5A4170700202315F7A097170020EE
:104670002395870C97A00100E780E0439715002061
:1046800083D5A50B17C501001305854397A001002D
:10469000E7806042294597A00100E780A04697F790
:1046A000FF1F938767D1DC4703D70700C167FD175A
:1046B0006312F7022244B7E70400B240924403A316
:1046C000870517F5FF1F0345E5191306000A854501
:1046D00041010283B2402244924441018280B1C12F
:1046E000411122C417C501001305459C2E8497C5AE
:1046F00001009385250A06C697A00100E780A03B2C
:10470000A28517C501001305653A97A00100E7804F
:10471000803A2244B2402945410117A301006700B5
:10472000633E8280011122CC37E404005C5C06CE3B
:10473000354697C501009385A51C17D501001305C3
:1047400025ED829711E917C501001305E59B97A098
:104750000100E780204E01A097F7FF1F93874711C4
:104760003EC4B7F50700856793870780814617F633
:10477000FF1F1306660FE10519453EC697E0FF1FB0
:10478000E78020067C44194697F5FF1F9385C50DE9
:1047900017050020130545908297340017F6FF1F78
:1047A0001306860C97C501009385056917C501009E
:1047B0001305056A97700000E78060922A841DCD7A
:1047C00097C501009385450517C501001305058EA2
:1047D00097A00100E780202EA28517C501001305D0
:1047E000251397A00100E780002D294597A001001F
:1047F000E7804031F24062440561828097E000002A
:10480000E78060F817C50100130585079760000071
:10481000E780A08697A00000E780A04C9760010089
:10482000E78020B117F5FF1F130585B597600100DC
:10483000E780C09917C50100130585059760010041
:10484000E780A0B12A8497600000E780E0EC971031
:104850000100E780008997800100E780202297709F
:104860000000E780C04897600000E780E062973072
:104870000100E780604A97C501009385E5F917C5F7
:1048800001001305A58219C897A00100E780A022A6
:10489000A28517C501001305E509A1B797A001007E
:1048A000E780602117C501001305050B97A00100E3
:1048B000E7806020294597A00100E780A024973079
:1048C0000100E780402697F00000E78000457DC5A5
:1048D00085453705040097300000E780809297C532
:1048E0000100938565F317B501001305257C97A09A
:1048F0000100E780401C17C501001305650797A05C
:104900000100E780401B294597A00100E780801F38
:1049100097F7FF1F9387C79983D7070017170020C2
:10492000231DF7E08547171700202305F7D097F7D9
:10493000FF1F938767A8DC4703D70700C167FD17F0
:104940006316F70097F0FFFFE780C06197700000E3
:10495000E78000C41305C50597700000E78000C418
:1049600097200000E78040B997200000E78000A36F
:10497000054597500000E78020FAB7E70400BC4FD8
:10498000130600649305001017F5FF1F034585ED1E
:10499000829797C50100938525E817B50100130597
:1049A000E57097A00100E780001117C5010013050D
:1049B00065FE97A00100E780001005BD97C50100C6
:1049C000938585E517B501001305456E97A0010095
:1049D000E780600E17C501001305850F97A0010041
:1049E000E780600D294597A00100E780A0110145EF
:1049F00097500000E78040F269BF411122C437E4BC
:104A000004008327041A06C6829797500000E780A7
:104A1000C0C08327040817F5FFFF1305E5618297DF
:104A200097F7FF1F2380A7E417F5FF1F1305C5980D
:104A300097400000E78080702244B2404101170394
:104A40000000670063CEB7E70400FC471171A2DDE8
:104A5000CAD986DFA6DBCED72E8432892E86AA85D8
:104A600017F5FF1F1305456D829717F7FF1F1307F3
:104A7000A76C83470700930680029387E70793F7A5
:104A8000F70FE3ECF610BA898A0717B7010013078E
:104A9000276BBA979C43BA9782878D4797C50100C9
:104AA0009385C5D917B5010013054560630FF40060
:104AB00097A00100E780200017C501001305C596E7
:104AC00097A00100E78020FFBDA497A00100E78028
:104AD00080FE17C501001305A59697A00100E78089
:104AE00080FD294597A00100E780C001930720F8C9
:104AF000114697F5FF1F938525644A8517F7FF1F19
:104B0000230CF76297F7FF1FA389076297F0FFFF57
:104B1000E780402F2A841DC997C50100938505D2DF
:104B200017B501001305855897A00100E780A0F88C
:104B3000A28517C501001305659497A00100E780C1
:104B400080F7294597A00100E780C0FB97C50100C9
:104B50009385C5CE17B501001305455597A00100F3
:104B6000E78060F517C501001305859297A0010045
:104B7000E78060F4294597A00100E780A0F841652F
:104B8000930730FA054697F5FF1F9385E55A7D1583
:104B900017F7FF1F2302F75A97F0FFFFE7808026E1
:104BA0002A841DC997C50100938545C917B5010021
:104BB0001305C54F97A00100E780E0EFA28517C558
:104BC00001001305A58B97A00100E780C0EE2945E1
:104BD00097A00100E78000F3B7E70400BC4F05662B
:104BE000130606C8A14517F5FF1F0345A5C7829701
:104BF000FE506E54DE544E59BE5911618280914769
:104C00006303F40297C50100938545C317B50100FE
:104C10001305C54997A00100E780E0E917C5010029
:104C20001305458A71BDB7E70400FC4F914517F5A0
:104C3000FF1F034525C3829797C50100938505C0D3
:104C400017B501001305854697A00100E780A0E68F
:104C500017C501001305C58897A00100E780A0E5EE
:104C6000294597A00100E780E0E997400000E78030
:104C7000401A914535A485476303F40297C50100A6
:104C80009385C5BB17B501001305454297A00100E8
:104C9000E78060E217C501001305058615B597F793
:104CA000FF1F2399273FB7E704000566BC4F130693
:104CB00006C8C1450DBF8D476303F40297C50100C7
:104CC0009385C5B717B501001305453E97A00100B0
:104CD000E78060DE17C501001305C583D5B39307D0
:104CE00040F8114697F5FF1F938505454A8517F74C
:104CF000FF1F2303F74497F7FF1FA380074497F094
:104D0000FFFFE78020102A84E30405EE97C5010029
:104D10009385C5B217B501001305453997A0010069
:104D2000E78060D9A28517B501001305257597A006
:104D30000100E78040D8294597A00100E78080DC8A
:104D400045BD9147E31CF4F6B7E70400FC4F93051B
:104D5000000217F5FF1F0345E5B0829797C50100D4
:104D60009385C5AD17B501001305453497A0010023
:104D7000E78060D417B501001305457BF1BD894775
:104D800063E3870297C50100938545AB17B5010022
:104D90001305C53197A00100E780E0D117B50100E8
:104DA0001305057A31BB97F4FF1F83C4043997F7C5
:104DB000FF1F83C7773897C50100938525A8A204F4
:104DC00017B501001305852EDD8C97A00100E78043
:104DD00080CEA28517B501001305C57797A0010005
:104DE000E78060CDC204294597A00100E78080D10B
:104DF000C1849305D4FF93960401C1824A8693F53A
:104E0000F50F17F5FF1F1305553397200000E780B6
:104E10000043E35F90DC930750F817F7FF1F230D63
:104E2000F73083C73900228697F5FF1F9385C53079
:104E300085074A8517F7FF1FA301F73097F0FFFF9B
:104E4000E78040FC2A84E30505DA97C501009385D5
:104E5000E59E17B501001305652597A00100E780C1
:104E600080C5A28517C50100130545C3C9B589478B
:104E700063E3870297C501009385459C17B5010040
:104E80001305C52297A00100E780E0C217B5010015
:104E90001305056E35B197400000E78080F7A285C5
:104EA00017F5FF1F1305452997500000E780C09DA7
:104EB00081B38D476303F40297C50100938505987C
:104EC00017B501001305851E97A00100E780A0BE5D
:104ED00017B501001305856BE5B6B76602000146FC
:104EE000B7750200054597E0FF1FE780808F9307A5
:104EF00060F817F7FF1F2301F72497F7FF1FA38E12
:104F000007229307000617F7FF1F2309F722894797
:104F100017F7FF1FA304F72297F7FF1F238107222C
:104F200097F7FF1FA38D0720C14717F7FF1F23091E
:104F3000F720930720F917F7FF1FA303F720314647
:104F400097F7FF1FA38FA71E97F5FF1F9385C51E19
:104F50004A8597F7FF1F2386071E97F0FFFFE7801C
:104F600060EA2A84E30605C897C501009385058D8C
:104F700017B501001305851397A00100E780A0B3C2
:104F8000A28517B501001305E56155B3B147630369
:104F9000F40297C501009385658A17B501001305D2
:104FA000E51097A00100E78000B117B501001305D7
:104FB000256139B6B7E70400FC4F9305000417F5E7
:104FC000FF1F0345258A829797400000E78060E431
:104FD000B145F9B5914763E3870297C50100938511
:104FE000E58517B501001305650C97A00100E78062
:104FF00080AC17B501001305655ED9B497F4FF1FA7
:1050000083C4C41397F7FF1F83C73713A204DD8C33
:105010008E04B77702006D14BE942286A68517B55C
:1050200001001305E55C97A00100E780C0A8B7E781
:105030000400FC47228697F5FF1F93853510280052
:10504000829793160401C1823000A685094597D046
:10505000FF1FE78000792A8409C917B501001305ED
:10506000E55A97A00100E780E0BC930770F8194665
:1050700097F5FF1F9385450C4A8517F7FF1F230DF2
:10508000F70A97F7FF1FA38B870A97F0FFFFE780C8
:1050900060D72A84E30E05B497B501009385057A9D
:1050A00017B501001305850097A00100E780A0A0B7
:1050B000A28517B501001305655695B99947630B8D
:1050C000F41297B501009385657717B501001305B4
:1050D000E5FD97A00100E780009E17B501001305CC
:1050E0006555F9BA914763E3870297B50100938547
:1050F000E57417B50100130565FB97A00100E78073
:10510000809B17B50100130565545DBA97F4FF1F26
:1051100083C4C40297F7FF1F83C73702A204DD8C44
:105120008E04B77702006D14BE942286A68517B54B
:1051300001001305E55297A00100E780C097B7E78B
:105140000400FC47228697F5FF1F938535FF280052
:10515000829793160401C1823000A6850D4597D031
:10516000FF1FE78000682A8409C917B501001305ED
:10517000E55097A00100E780E0AB930780F819465F
:1051800097F5FF1F938545FB4A8517F7FF1F2305FA
:10519000F7FA97F7FF1FA38387FA97F0FFFFE780DF
:1051A00060C62A84E30605A497B5010093850569C6
:1051B00017B50100130585EF97A00100E780A08FC8
:1051C000A28517B501001305A54C95B69947630351
:1051D000F40297B501009385656617B501001305C4
:1051E000E5EC97A00100E780008D17B501001305DD
:1051F000A54BF9B0B7E70400FC4F9305000417E591
:10520000FF1F03452566829797400000E78060C036
:10521000994579B18D476303F40297B501009385F1
:10522000E56117B50100130565E897A00100E78067
:10523000808817B501001305A54859B017B50100BE
:105240001305054997A00100E780C09E1305C01211
:1052500097D0FF1FE780E00E014597E0FFFFE78052
:10526000A0E30D4597100000E780A0A0294597D046
:10527000FF1FE780000D97D0FF1FE78060FD8DBA0C
:1052800099476303F40297B501009385255B17B531
:1052900001001305A5E197A00100E780C08117B5C3
:1052A00001001305A54329B817F7FF1F034717E9A6
:1052B00097F7FF1F83C787E822075D8F9166BA962D
:1052C000C2061166C1821306F6EF8D476365D602EA
:1052D00097E7FF1F9387470E9C4B17F6FF1F034668
:1052E000D6E59386C7002DC203D6070069CA890791
:1052F000E39CD7FE89471307A0F8114697F5FF1FD7
:10530000938585E34A8597F6FF1F2387E6E217F723
:10531000FF1FA304F7E297F0FFFFE780A0AE2A8407
:10532000E308058C97B501009385455117B5010039
:105330001305C5D797900100E780E077A28517B5E0
:1053400001001305E53AE5B203D60700630EE60A4D
:105350008907E39BF6FE8D4779BF91476304F4020A
:1053600097B501009385854D17B50100130505D448
:1053700097900100E780207417B501001305C53828
:105380006FF00FF4B7E70400FC4F9305000817E532
:10539000FF1F0345254D8297C9B897B50100938536
:1053A000E54917B50100130565D097900100E78026
:1053B000807017B501001305A5366FF06FF02390CC
:1053C000E70017E5FF1F130525FF97300100E78071
:1053D000009B97B501009385654617B5010013053D
:1053E000E5CC97900100E780006D17B5010013052B
:1053F000253497900100E780006C294597900100C3
:10540000E78040708147C5BD2390070017E5FF1F67
:10541000130585FA97300100E780609697B5010083
:105420009385C54117B50100130545C89790010044
:10543000E780606817B50100130505315DBF4111B4
:1054400022C406C6834705002A849DC797B501007C
:105450009385853A17B50100130545C5979001005E
:10546000E78060654C4017B50100130565699790AA
:105470000100E7804064E1A05841B707CF0093875F
:10548000777D631DF70697B501009385E53617B55F
:1054900001001305A5C197900100E780C0611C447D
:1054A0008356E4008355C40003C6070017B5010006
:1054B0001305856697900100E780E05F2945979086
:1054C0000100E78020640357E4009707002083D79A
:1054D000C7266309F7008355C400084497E0FFFF1F
:1054E000E78000D00356E4008355C40008442244FA
:1054F000B240410117F3FFFF67002355B707CC0007
:105500009387777D6315F70497B501009385C52EC2
:1055100017B50100130585B997900100E780A059E0
:105520001C448356E4008355C40003C6070017B526
:1055300001001305655E97900100E780C057224483
:10554000B24029454101179301006700A35BB707EB
:10555000CE009387777D6304F70297B501009385AA
:10556000A52917B50100130565B497900100E780E0
:1055700080544C4017B501001305454FCDBDB240D6
:10558000224441018280411122C44AC006C626C27B
:105590009307D00D2A892E841306D00D63E3B7003C
:1055A0002E86B7E70400FC4742064182CA8517F5FC
:1055B000FF1F130565B8829797B501009385C5292C
:1055C00017B50100130585AE97900100E780A04E46
:1055D00097F5FF1F83C545B617B501001305C5CF65
:1055E00097900100E780204D294597900100E780C2
:1055F000605197F4FF1F938424B483C7040041478C
:105600009387070693F7F70F636CF75A17B70100F4
:10561000130747BD8A07BA979C43BA978287994771
:1056200063E7870297B501009385052317B501004D
:105630001305C5A797900100E780E04717B5010063
:10564000130505CA97900100E780E0468DA497F7FF
:10565000FF1F83C777AEDDCB17F7FF1F0347F7ADFB
:1056600097F7FF1F83C767AD22075D8F97F7FF1F6F
:1056700083C7C7ACC2075D8F97F7FF1F83C717ACFF
:10568000E207D98F17F7FF1F2326F7A883C7640007
:1056900097B501009385451C17B50100130505A1B9
:1056A00017F7FF1F2306F7A697900100E780A04099
:1056B00097F7FF1F938707A68C4317F6FF1F034634
:1056C00026A517B50100130565C397900100E78073
:1056D000803E294597900100E780C04297F7FF1F61
:1056E000A38C07A42244B24092440249930700F8D5
:1056F00017F7FF1F2302F7A49D4517F5FF1F13059A
:10570000A5A341011743000067000318976000003C
:10571000E78040E797F7FF1F2381A7A293578500F3
:1057200017F7FF1FA30BF7A0935705012A8417F75C
:10573000FF1F2305F7A093578501014517F7FF1FAA
:10574000A30EF79E97600000E78020E897F7FF1F01
:105750002387A79E97B501009385051017B5010013
:105760001305C59497900100E780E03417F6FF1FFA
:105770000346E69CA28517B501001305A5B9B1B78C
:10578000C94763E3870297B501009385E50C17B518
:1057900001001305A59197900100E780C03117B56E
:1057A00001001305A5B879BD37E404007C444146E7
:1057B00097F5FF1F9385559817F5FF1F1305C5959E
:1057C000829797F7FF1F83C7479817F7FF1F034775
:1057D000B797A20703238405D98F17F7FF1F231854
:1057E000F7921306000A89452244B24092440249C6
:1057F00017E5FF1F0345050741010283894763E35E
:10580000870297B501009385250517B5010013059B
:10581000E58997900100E780002A17B5010013057C
:10582000A5C00DB517F4FF1F0344249197F7FF1F80
:1058300083C7979097B5010093850502220417B599
:1058400001001305A5865D8C97900100E780A026D6
:10585000A28517B501001305E5AE97900100E7801A
:105860008025294597900100E780C0290D4697F5CE
:10587000FF1F9385658C228597E0FFFFE7808058A6
:10588000AA8421C197B50100938505FD17B50100D4
:105890001305C58197900100E780E021A68517B523
:1058A0000100130565AB97900100E780C0202244FA
:1058B000B240924402492945410117930100670013
:1058C000632497E7FF1F2397877CB7E704001166DF
:1058D00003A38705130606E8914539B7894763E3B3
:1058E000870297B50100938525F717A501001305D9
:1058F000E57B97900100E780001C17B501001305B8
:1059000065C189B317F4FF1F0344248397F7FF1F72
:1059100083C7978297B50100938505F4220417A5E4
:1059200001001305A5785D8C97900100E780A01811
:10593000A28517B50100130565A397900100E780C4
:105940008017294597900100E780C01B0D4697E519
:10595000FF1F9385657E228597E0FFFFE780804AE1
:10596000AA841DC197B50100938505EF17A5010015
:105970001305C57397900100E780E013A68517B55E
:1059800001001305E59F05B797E7FF1F2396876E74
:10599000B7E70400116603A38705130606E893051D
:1059A000000299B5894763E3870297B501009385A3
:1059B000A5EA17A501001305656F97900100E78020
:1059C000800F17B501001305A5B7ADB997E4FF1F08
:1059D00083C4A47697E7FF1F83C7177697B50100A6
:1059E000938585E7A20417A501001305256CDD8CBE
:1059F00097900100E780200CA68517B501001305DC
:105A0000A59997900100E780000B29459790010028
:105A1000E780400F228697E5FF1F9385E571268575
:105A200097E0FFFFE780003E2A84630C051A97B5D4
:105A30000100938565E217A501001305256797907E
:105A40000100E7804007A28517B501001305059600
:105A500099BD854763F78718834519002244B240F2
:105A600092440249B335B00097E7FF1F238EB76217
:105A700017B501001305C594410117930100670094
:105A80008303A2852244B24092444A8502494101DF
:105A90001703000067002324954763E3870297B547
:105AA0000100938565DB17A501001305256097901C
:105AB0000100E780400017B50100130525C259B663
:105AC00017E4FF1F0344646797E7FF1F83C7D76688
:105AD00097B50100938545D8220417A50100130549
:105AE000E55C5D8C97900100E780E0FCA28517B52E
:105AF00001001305658E97900100E780C0FB2945E2
:105B000097900100E7800000194697E5FF1F9385F5
:105B1000A562228597E0FFFFE780C02EAA841DC101
:105B200097B50100938545D317A5010013050558C6
:105B300097900100E78020F8A68517B501001305AE
:105B4000A58A95B397E7FF1F2390875EB7E7040008
:105B5000116603A38705130606E89305000869B1DB
:105B600097B50100938545CF17A50100130505548E
:105B700011E897900100E78000F417B501001305C4
:105B8000E587C9B497900100E780E0F217B50100FE
:105B90001305458897900100E780E0F1294597902B
:105BA0000100E78020F62244B2409244024997E780
:105BB000FF1F239E07544101176300006700038DF8
:105BC00097B50100938545C917A501001305054E3A
:105BD00097900100E78020EE17B50100130545B44A
:105BE00095B4B2402244924402494101828041115D
:105BF00006C622C497E0FFFFE780C02021CD97E7CB
:105C0000FF1F83D7874A85072A8417E7FF1F231EB4
:105C1000F74897B501009385A5C597E7FF1F239720
:105C2000A74817A501001305654897900100E78074
:105C300080E8A28517B50100130545E6979001009D
:105C4000E78060E72244B2402945410117930100F3
:105C5000670043EB97E7FF1F83D76745B2402244B5
:105C6000850717E7FF1F2314F74441018280411184
:105C700022C491462A8417E6FF1F1306265A9D6503
:105C80002D4506C697D0FF1FE780A0B5B7F70700E0
:105C900003C70701A5476313F70001A0930600108F
:105CA00001469D65254597D0FF1FE78080B397E7A4
:105CB000FF1F238587562244B240914617E6FF1FF7
:105CC0001306C6559D652945410117D3FF1F67007F
:105CD00043B11171CED7B7E9040083A7C904CAD96B
:105CE00017E9FF1F13094945A2DD2E8686DFA6DBD3
:105CF0002E84AA854A85829797E7FF1F83C7C743EB
:105D00001307700A6385E710636DF7001307600AD5
:105D10006385E704FE506E54DE544E59BE5911613E
:105D200082801307800A6385E7161307900AE393BE
:105D3000E7FE8D476306F41C97B50100938545E99E
:105D400017A501001305853697900100E780A0D6BE
:105D500017B50100130505E525A08D47630CF40276
:105D600097B501009385C5E617A501001305053415
:105D700097900100E78020D417B501001305C5DB1B
:105D800097900100E78020D3294597900100E78094
:105D900060D749B7854717B501001305A5DB17E79D
:105DA000FF1F2303F73097900100E780A0E8B77545
:105DB0000200B76602000146054597D0FF1FE78045
:105DC00040A2930760F817E7FF1F2307F73697E70E
:105DD000FF1FA38407369307002617E7FF1F232F13
:105DE000F734E5779387072117E7FF1F231AF73466
:105DF000B14597E7FF1F2386073497E7FF1FA3826C
:105E0000A7344A8597000000E780E01621B7914744
:105E100063E3870297B50100938585DB17A5010031
:105E20001305C52897900100E780E0C817B5010069
:105E3000130545D4B1B797E4FF1F83C4243097E717
:105E4000FF1F83C7972FA204DD8C83A7C9046D149D
:105E5000228697E5FF1F9385752E280082978E0472
:105E600093160401B7750200C1823000A69509455A
:105E700097D0FF1FE780E096930770F817E7FF1FA2
:105E8000230CF72A994597E7FF1FA389A72A95BFF7
:105E9000914763E3870297B50100938565D317A502
:105EA00001001305A52097900100E780C0C017B539
:105EB00001001305A5CDE9B597E4FF1F83C40428AD
:105EC00097E7FF1F83C77727A204DD8C83A7C90448
:105ED0006D14228697E5FF1F93855526280082972B
:105EE0008E0493160401B7750200C1823000A69596
:105EF0000D4597D0FF1FE780C08E930780F8BDBF88
:105F000017B50100130545CB97900100E78080D2BB
:105F1000930790F82304F100834719008D4528006A
:105F2000A304F100834729002305F1009700000036
:105F3000E78060041305C01297C0FF1FE780604030
:105F4000014597D0FFFFE78020150D459700000021
:105F5000E78020D2294597C0FF1FE780803E97C089
:105F6000FF1FE780E02E7DB397E7FF1F23A0A72C3C
:105F7000828097E7FF1F9387672B03A307006303C4
:105F800003000283174300006700039041114AC0D9
:105F900097F6FF1F83D6667A328917D6FF1F0356FE
:105FA000C64322C426C206C62A84AE8497000000D7
:105FB000E780C05F35C12DC0994763FF97048347D1
:105FC000140003470400A207D98F13978700A18309
:105FD000D98FC2073167C1831307C755639EE70294
:105FE00097D7FF1F83D7673FA301F400A183230244
:105FF000F40097F7FF1F83D7477491C7A302F400FB
:10600000A1832303F400A68517B50100130545C03D
:1060100097900100E78020AA97F7FF1F83C7876149
:10602000A5C797D5FF1F83D5453B17B501001305BD
:10603000E5BF97900100E78000A82686A28517D5C6
:10604000FF1F0355853997000000E78080BA63067B
:10605000090497F7FF1F83C7E75DA1E397E7FF1FD9
:1060600083C7071D9DCB95C897E7FF1F83C7C7034D
:106070008DE722852244B2400249A685924441011F
:10608000174300006700438017B50100130505BBE7
:1060900097900100E78000BA5DBFB240224492446D
:1060A000024941018280834755008345450017B569
:1060B00001001305A5B4A207DD8D17930100670049
:1060C000839F17B50100130565B2179301006700A0
:1060D00063B68D4763FBB70A011126CA06CE22CCF0
:1060E0000344350097E4FF1F83C4941497B501005F
:1060F000938585B5B337800017E7FF1FA30AF71212
:1061000009C497B501009385E5B417B501001305DF
:10611000E5B497900100E780009A97E7FF1F83C7D7
:1061200037116386970097000000E780E02C97E71F
:10613000FF1F83C7F70F8DC785472306F100B7E719
:10614000040083A7471770008545130550308297D8
:1061500017B50100130585B197900100E78080AD68
:106160009967938757EE2316F1006800854791459C
:10617000A30781002307F10097000000E780A0DF5C
:10618000F2406244D244056182808280894763F78D
:10619000B708011122CC06CE26CA834425008547C4
:1061A0002A84639DF404914763F5B70403454500D1
:1061B0008347340022055D8D97D7FF1F239FA720BB
:1061C00097000000E78060479967938767EE231484
:1061D000F1008347340023059100A305F1008347B4
:1061E0004400954528002306F10097000000E78051
:1061F00080D8F2406244D24405618280FDF89967FC
:10620000938767EE2314F10097D7FF1F83D7E71C0E
:10621000A305F10023050100A183E1B782800111EC
:10622000996722CCD51717F4FF1F1304A440231439
:10623000F1008347040026CA97F4FF1F9384E44FBC
:106240002305F10083D7040028009545A305F1003C
:10625000A18306CE2306F10097000000E780A0D1BD
:1062600003D604008345040017B50100130585A17A
:1062700097900100E7802084F2406244D244056197
:1062800082809D677971D9172316F10097F7FF1F58
:1062900083C7473A06D62307F100A9C3B7E704002E
:1062A000FC47414697E5FF1F938505E71305F1007D
:1062B00082976800CD4597000000E780C0CB97F536
:1062C000FF1F83C5253717B501001305A59E9780CD
:1062D0000100E780407EB25045618280B7E704004C
:1062E000BC47414681451305F1008297D9B745C5A2
:1062F000411106C622C4930750FA2300F500930704
:10630000A005A300F50089472301F5009147A301EB
:10631000F5009307F003A302F50097F7FF1F93879B
:10632000673183C70700230205002A842303F50091
:1063300097E7FF1F9387D7EF83C70700414697E58D
:10634000FF1F938565DDA303F50097F7FF1F83D734
:10635000C73E2304F500A183A304F50097D7FF1FD0
:1063600083D7A7072305F500A183A305F500B7E7A9
:106370000400FC47310582972285F1459700000013
:10638000E780C01E230EA4002181A30EA400B2400A
:10639000224441018280828079710A8506D6970065
:1063A0000000E78000F50A86F945014597D0FFFF18
:1063B000E7806036B25045618280411122C426C216
:1063C0004AC02A84AE843289AA858566014625455D
:1063D00006C697C0FF1FE780C040A2852244B24096
:1063E000CA862686024992442945410117C3FF1FE8
:1063F0006700233F0111B7C7A55A22CC9387C73343
:1064000017E4FF1F1304D4E23EC4834704002C00AA
:106410002146196506CE3EC697000000E78020FAA7
:106420008345040017B501001305C5979780010047
:10643000E7806068F2406244056182800111A146F4
:10644000300099652D4522CC06CE97C0FF1FE7800E
:106450004039A24737C4A55A1304C4336395870251
:10646000B24517B5010013052587B335B00097E78E
:10647000FF1FA38FB7DA97800100E780C063F24067
:106480006244056182809165A1463000938505F0E4
:106490002D4597C0FF1FE780C034A247E38287FCE9
:1064A00097E7FF1FA38607D8814517B5010013059D
:1064B000E584D1B7B7C7A55A79719387F7353EC63A
:1064C000B7E70400FC4706D6AA854146080882972C
:1064D0006C005146116597000000E78040EE17B54B
:1064E00001001305E58F97800100E780A074B2508A
:1064F000456182807971D146700091652D4522D425
:1065000006D697C0FF1FE780C02DB24737C4A55AF3
:106510001304F43563988702B7E70400FC4717E5D6
:10652000FF1F130565BF41460C08829717B5010090
:106530001305C58297800100E780C06FB2502254D6
:10654000456182809165D1467000938505E82D45AF
:1065500097C0FF1FE780E028B247E38F87FA17B59F
:1065600001001305A581F9B7C16769768146FD175A
:1065700005061397060141836364B7003E85828058
:106580003307D50003470700B98F214713F81700D9
:10659000858363050800B18FC207C1837D17137718
:1065A000F70F6DF78506F1B741C5A547054763F2BB
:1065B000B70883471500034705003168A207D98F44
:1065C00013978700A183D98FC207C1831308C855C9
:1065D000054763900707411106C622C426C203443B
:1065E0002500914763F087049307540063ECF5029C
:1065F000A301C50021822302C5009304340091C683
:10660000A302D500A1822303D5002A84A685970082
:106610000000E780A0F526942300A4002181A300B8
:10662000A4000147B240224492443A85410182804D
:1066300005473A8582800111B7C7A55A22CC9387B6
:10664000E7342A842AC621462C00156506CE3EC4AE
:1066500097000000E780A0D6A28517A501001305CA
:10666000657697800100E780004597000000E7808D
:10667000E0D2F2406244056182800111A1463000FF
:1066800095652D4522CC06CE97C0FF1FE78060158B
:10669000A24737C4A55A1304E43463958702B24570
:1066A00017A501001305856797D7FF1F2397B7D25A
:1066B000C205C18197800100E780E03FF24062445B
:1066C000056182809165A1463000938505EE2D45D8
:1066D00097C0FF1FE780E010A247E38287FCD14705
:1066E00017D7FF1F231BF7CED14517A501001305B0
:1066F000E564C9B721C1411126C206C622C4AE84D1
:106700008DC52A8497000000E780E06097E7FF1FAF
:1067100083C707B299CB22852244B240A685924412
:1067200041011733000067002316B240224492440F
:1067300041018280828001114AC806CE22CC26CA3D
:106740004EC693F715002E899DCBAD6737170040D5
:106750009387A7AA1CC3B7E70400BC4F1306001910
:10676000854517D5FF1F034525C782971345190097
:10677000F2406244D2444249B2490561828093F7B3
:106780002500638A071C17F7FF1F0357E7FA954791
:1067900063F9E70C014417F6FF1F1306E6E99306B9
:1067A000300513055004130810049308B0041303B4
:1067B0009005930764006374F7043A84FD5997F4D5
:1067C000FF1F83C464E797F7FF1F83C7F7E6A204A0
:1067D000DD8CAD679387B755638BF41463E3970A39
:1067E000A9679387A755638EF414A28517F5FF1F39
:1067F000130585E497000000E78000F031A2B3079D
:10680000860083C50700639AD50483C51700639685
:10681000A50483C527006392050583C53700639EE1
:10682000D50283C54700639A150383C75700639653
:106830006702A2890DE897F5FF1F83D5E5EFB385C1
:106840003541C20517F5FF1F130505DFC1814E95C0
:1068500097000000E78040EAE1A00504420441807F
:1068600089BF3A84FD598547E3EB87F45DC48545CC
:1068700017F5FF1F130545DC97000000E780C0E710
:1068800069A8B1679387C7556380F404B567938798
:10689000D755E39CF4F4A28517F5FF1F1305C5D95E
:1068A00097300000E78040FE8947630FF4049305AA
:1068B000E4FFC205C18117F5FF1F130505D8970036
:1068C0000000E780404589A097200000E78020F283
:1068D00097000000E780804311C9A28517F5FF1FCC
:1068E000130585D597000000E780E0420546A285A4
:1068F00017F5FF1F130545D497F0FFFFE7804069A8
:1069000097200000E780A0EEA68517A501001305DB
:10691000254F97800100E780001AFD57E39DF9F0AD
:1069200097F7FF1F239A07E01345290091B5A28529
:1069300017F5FF1F130545D097F0FFFFE780E076BE
:10694000E1B7A28517F5FF1F130505CF97F0FFFFED
:10695000E780607755BF93F745000145E38A07E07C
:1069600017A501001305054B97800100E780802CD7
:1069700097300000E780001F13454900D5BB411147
:1069800022C437E404005C5C06C6354697A50100C6
:10699000938505F717B50100130585C7829711E99F
:1069A00017A501001305C54797800100E7808028DF
:1069B00001A08327041C82972A84054597C0000004
:1069C000E780C0DB97600100E780E060976001002E
:1069D000E780E03597B00000E78040ED2285B240C7
:1069E0002244410182804111054506C622C426C2C7
:1069F00097C0FFFFE78020541305A00497B0FF1F46
:106A0000E780E06A757585457D1597C0FFFFE780D3
:106A1000C03D7D7585451305F53697C0FFFFE780BE
:106A20002047371400408327840A8D451305002032
:106A300093E707202324F40A97C0FFFFE780E03A9A
:106A4000B7E4040097D0FFFFE7800080C858978024
:106A50000100E780201E17B50100130565BB978074
:106A60000100E780201D8327840C8545414593E77D
:106A700007082324F40C97C0FFFFE78060418D4591
:106A80001305000897C0FFFFE780804097C0FFFF15
:106A9000E780606D37A507001305051297C0FFFF5B
:106AA000E7800069014597C0FFFFE780206F9545AB
:106AB0000545894717F7FF1F2302F7C897C0FFFF57
:106AC000E780606FB7E700E013070006238DE7401B
:106AD0003707000423A0E71097D0FFFFE780A0F559
:106AE00097D0FFFFE780A00797000000E78060E9EC
:106AF00097000000E780C09497000000E78020B86E
:106B000097E0FFFFE780A0EF97000000E780E0211B
:106B100097000000E780E00A83A70408170500003B
:106B20001305A5C1829797D7FF1F2387A78ABC4C5F
:106B3000130600648545829797C0FF1FE780408B4E
:106B400001458280B7F7070003C70701A547AE8656
:106B50006316F7009397450191C301A0AA850146EA
:106B6000254517C3FF1F6700C3C74111B2862E8694
:106B7000AA852D4506C697C0FF1FE78080C6B24094
:106B80000145410182809307000463E8C7021D713B
:106B9000A2CC2A84080886CE32C697800100E780FE
:106BA00020E6B2461008A285294597C0FF1FE7805E
:106BB00040C3F64066442561828039558280411188
:106BC0000D658D4506C697C0FFFFE7800022B71709
:106BD00000408D6623A6D70A17F5FF1F130545B69B
:106BE0001387C70A9387870A1CC15CC585668967B6
:106BF0005CC958C114C518C9B7E70400B24003A363
:106C0000871E410102838145B307B50083870700D2
:106C100089E717230000670023C48505C205C181E9
:106C2000E5B797A701009387A7391357C5003E978B
:106C300003470700011106CE2304E1001357850026
:106C40003D8B3E970347070023060100A304E100A4
:106C5000135745003D8B3D893E97AA970347070090
:106C600083C7070028002305E100A305F100970072
:106C70000000E78080F9F24005618280411126C260
:106C8000E97797F4FF1F938424BC22C49387A75508
:106C90002E842381B4002E86AA8517F5FF1F1305C5
:106CA000E5BA06C62390F400A38104009780010092
:106CB000E78000D593052400C205C18117F5FF1FA9
:106CC0001305A5B897000000E780408AB3878400C9
:106CD0002382A7002181A382A70093056400224498
:106CE000B24026859244C205C181410117230000AC
:106CF000670083B609C99307800263E6B7001703EC
:106D000000006700E3F7828017F5FF1F0345C5A465
:106D1000828097F7FF1F83C7E7B289E71723000038
:106D2000670083B3828097F7FF1F83C7C7B499EFCB
:106D3000411106C697200000E780E0A9B2408547D0
:106D400017F7FF1F2309F7B2410182808280630792
:106D5000054A6385054A5D71CAC04EDE86C6A2C477
:106D6000A6C252DC56DA5AD85ED662D466D26AD04F
:106D7000B9472A89AE8963F9B706394697A5010054
:106D80009385C51197800100E78020C531ED8347C9
:106D9000E900130710036394E702854717F7FF1F05
:106DA0002302F7AA17A501001305451097F7FF1F47
:106DB000239907A897000000E78020E571A013073A
:106DC000000317A5010013056511E395E7FE97F78A
:106DD000FF1F238907A697F7FF1F239407A617A570
:106DE00001001305250EF9B797F7FF1F83C787A585
:106DF00063870722BD6AB96B938CFA55014A17FB6A
:106E0000FF1F130BAB95138CEB65938AFA6605A8ED
:106E1000B307490183C6070097F7FF1F83D767A20F
:106E2000B1E39307A005639BF600854717F7FF1FA3
:106E30002319F7A097F7FF1F2382D792050A93170C
:106E40000A01C183E3E637FDB6402644964406496D
:106E5000F259625AD25A425BB25B225C925C025D8A
:106E600061618280054D639BA7039307500A639E6F
:106E7000F600894717F7FF1F2315F79C930750FA71
:106E800017F7FF1FA30CF78C55BF9307A005E387E7
:106E9000F6FA97F7FF1F2396079A4DB71387170047
:106EA0004207DA9741832380D70017F6FF1F231A82
:106EB000E6988D47E3F4E7F817F4FF1F0344348A9C
:106EC00097F7FF1F83C7A78922045D8C9307F4FF00
:106ED000C207C1839306F00DE3EDF6FA9307640051
:106EE000C207C183E31CF7F493052400C205C181E6
:106EF00017F5FF1F1305A58697F0FFFFE7800067D2
:106F000033078B008347570003474700A207D98FF9
:106F100017F7FF1F231707926318F50E8144630CC0
:106F2000A40197F4FF1F83C4A483A20497F7FF1F53
:106F300083C71783DD8C170500001305E5DB97F089
:106F4000FFFFE780A00263878407636D9C0293873D
:106F5000EB556382F40497F7FF1F83C767800547EB
:106F60006389E70681CB1387A7051377F70F8D4653
:106F700063F2E6081307F0072300E100A300F10025
:106F800089459DA063829405E39754FD97F0FFFF28
:106F9000E780602F11A8A28517E5FF1F1305457C28
:106FA00097F0FFFFE7802013014597F0FFFFE78090
:106FB000E0FB69B5A28517E5FF1F1305657A97F019
:106FC000FFFFE780E01CCDB797F0FFFFE78060256B
:106FD000E1BF930710F8130511002300F10097F0AB
:106FE000FFFFE7800031FD450A8597000000E7803C
:106FF00020C95DBFA28517E5FF1F1305657697F0D1
:10700000FFFFE78040CD4DB79307F00789450A851C
:107010002310F10097000000E78080C605B5BD474A
:1070200063F83717414697A50100938565ED4A85BA
:1070300097800100E780609A631C051417A5010082
:10704000130545ED97000000E78020BC17E5FF1F02
:107050000355A56E97000000E780E0BC97E7FF1F8F
:1070600083C7475D17A50100130545E289E717A50A
:107070000100130525E297000000E78000B917A57D
:1070800001001305A5EA97000000E78000B817C5C6
:10709000FF1F0355253297000000E780C0B817A5F1
:1070A00001001305E5E897000000E78000B617C56A
:1070B000FF1F0355853297000000E780C0B617A573
:1070C0000100130565E797000000E78000B417D5BD
:1070D000FF1F0355C5FD97000000E780C0B417A54A
:1070E00001001305E5E597000000E78000B217D521
:1070F000FF1F035585FB97000000E780C0B217A56E
:107100000100130565E497000000E78000B017D583
:10711000FF1F0355A5F997000000E780C0B017A531
:1071200001001305A5E297000000E78000AE17C537
:10713000FF1F0355E51897000000E780C0AE17A5B4
:107140000100130525E197000000E78000AC97D708
:10715000FF1F83C767FCA20717D5FF1F0345D5FB99
:107160005D8D97000000E78000AC97D7FF1F83C7B5
:10717000C7FAA20717D5FF1F034535FA5D8D9700A3
:107180000000E78040AA179501001305E54E1DB1E8
:10719000C14763FE3705414697A501009385C5DBCE
:1071A0004A8597800100E780408331E183470901E8
:1071B00013071003639CE700854717E7FF1F230DA4
:1071C000F75817A50100130565DAEDB6130700039C
:1071D00017A50100130585DCE39EE7BC97E7FF1FB9
:1071E000238C075617A501001305C5D9E1B6CE8536
:1071F0004A8597C0FFFFE780A0FEB9B182804111A8
:1072000026C2AE848D4522C406C62A8497C0FFFFDD
:10721000E78000C8B717004099C803A5C70C418D87
:1072200023A6A70CB240224492444101828003A5C8
:10723000870C418D23A4A70CF5B7834705000347AE
:107240001500A207D98FC2076177C18713072720CE
:10725000639AE70083452500370504001703000003
:10726000670023FA828017E6FF1F13062661814715
:10727000B2861303F00FA9483308F600034808004C
:1072800013F7F70F6307A80C630668008507E395FB
:1072900017FF2947B387E6002380A70097E7FF1F62
:1072A0009387875E5DA8411113D7650013471700C8
:1072B00006C693F63500058B954791CA0546994752
:1072C0006387C60009469D476383C600A14713F63E
:1072D00045003336C00093F68503050685C2A145F7
:1072E000638BB604E145638AB60493058002638824
:1072F000B604930580036393B600914697E5FF1F9C
:107300002389F57E97E5FF1F2384C57E97E5FF1F40
:10731000A380D57EBE8517A50100130565CE9770A5
:107320000100E7804079B240854717E7FF1FA302BD
:10733000F77C410182808546D1B78946C1B78D4629
:1073400075BF17A50100130525CE1773010067004F
:10735000837617E7FF1F13072753BA972380B700D9
:10736000E147E302F5F493077002E30CF5FC828039
:107370002A8723800500814717E5FF1F1305055065
:107380001308F00F2946B306F50083C6060063967E
:10739000E60297E6FF1F9386264FB69783C707003E
:1073A00005452380F5009947636EF7029D4763FD0D
:1073B000E700E147630DF7008280638506018507DA
:1073C000E393C7FC0145C5B7238005008280B7372A
:1073D000004003C7370083C7050093F70704D98F20
:1073E0002380F50082805D7152DC56DA5ED6716AC8
:1073F00097FBFF1F938B0B818D6AA6C24EDE62D472
:1074000086C6A2C4CAC05AD866D26AD06ECEC14956
:107410005E8C97E4FF1F9384E447130A0A20938A43
:107420007ADC17F9FF1F0349E980B3872B0183C773
:10743000070093F7F70FC9EFB787004003C767004E
:10744000058BE310077C03C76700118BE30D077EF4
:1074500083C75700918B99E36F10200317E7FF1F35
:107460000347677D85476304F7006F10400197E786
:10747000FF1FA380E76897E7FF1F238D074C97E75F
:10748000FF1F238B075897E7FF1F2389076497E7A0
:10749000FF1F2386076497E7FF1FA38D074A97E71F
:1074A000FF1FA38B075697E7FF1FA389076297E784
:1074B000FF1FA386076297E7FF1FA38D076297E769
:1074C000FF1FA38A0776B787004011476F007077C8
:1074D0009307190093F7F70F3D476364F70617E723
:1074E000FF1F2309F77497E7FF1F9387A773CA97B6
:1074F00083C707001307100293F7F703638EE71E95
:107500006366F70405446385871CE38C07620947BB
:10751000638EE71013070002E384E74EB7E700E04D
:107520003707400023A0E7180100010062992300FB
:107530000900FD1923A0E71093F9F90FE39309EE71
:10754000E5BD97E7FF1F2387076E71BF1307300262
:107550006388E70C63E8E71613074002638CE70AC9
:1075600013070003E39CE7FA97E7FF1F9387876AF7
:10757000CA9703C70700A1471377F70FE31BF71458
:1075800083C7640097E6FF1F238CF65497E7FF1F1D
:1075900083C7B73091C7FD5797E6FF1F2382F65484
:1075A00097E5FF1F83C5152F97E7FF1FA38AB752E3
:1075B00097E7FF1F83C7072E13FB070893060004F6
:1075C00093F70706639FD74C9307A009638DF516C1
:1075D00063EAB7129307F0056386F54A93075009EB
:1075E0006384F52A014497E7FF1F83C7774F154748
:1075F000E392E736B7E700E03707400023A0E7183B
:1076000001000100B786004023808602130680FC3B
:107610006F00500EFD5717E7FF1F2302F74CFDBD0B
:10762000FD5717E7FF1F230BF74ACDBD17A5010034
:10763000130505B197700100E780C05F97E7FF1F52
:107640009387475DCA9703C40700014B97ECFF1F60
:10765000938CCC3C1374F40F17AD0100130DCDAE19
:1076600063478B04294597700100E780A04985474F
:1076700017E7FF1FA302F73A17E7FF1F230F87380B
:1076800017E7FF1F2308F74637E700E0B70640007B
:107690002320D71801000100378600408347A60247
:1076A00093F7370F2305F6022320D71085BDB38744
:1076B0006C0183C507006A85050B97700100E780A0
:1076C000803F79BF854717E7FF1F2307F734B9B518
:1076D00017E7FF1F130707544A970347070097E66A
:1076E000FF1FA389F62697E6FF1F2386E62617E7E6
:1076F000FF1F2301F7401DB5854717E7FF1F230B29
:10770000F72429BD9307400A6389F5349307200BBA
:107710006384F5369307100AE396F5EC838724001B
:107720000144E3D207EC97E7FF1F83C7D71693F610
:107730003700638A061A0546638AC622094663959E
:10774000C61A1D4755A217E5FF1F0345C514C947B3
:1077500097ECFF1F83CC3C1497E5FF1F83C5C5132F
:1077600017E4FF1F034454136315F510CD476392CC
:10777000FC1093077008639CF5021307300FB717CE
:107780000E006308E4001307900DB7B704006314FC
:10779000E40817E7FF1F232BF734BE8517A5010068
:1077A0001305059B97700100E780E03025BD930726
:1077B0008008639DF500B307804013F4F70FB77797
:1077C0004600938787CDB3D78702E1B79307900828
:1077D000639AF500B307804013F4F70F916793871E
:1077E000C766D5B79307A008639BF500B307804031
:1077F00013F4F70FB7173D0093870790E9B7930786
:10780000B008639AF500B307804013F4F70F91674F
:10781000938797D04DBF93F5F5078D47639BF50090
:10782000B307804013F4F70FB7975B00938707D82F
:1078300059BF8947639BF500B307804013F4F70FE6
:10784000B7770B009387071BBDBF8547639AF50089
:10785000B307804013F4F70FDD67938767E3A5B79D
:10786000D28785F9B307804093F7F70FB3D7FA02B1
:107870000DB797000000E780409FA28566859700BE
:107880000000E780809EB9BB9305610017E5FF1FEC
:107890000345650017E4FF1F0344F4FF9700000051
:1078A000E78040AD93057100228597000000E780D6
:1078B00060AC3C0017E7FF1F2324F73483476100C7
:1078C0002304F10083477100A304F100894717E7FF
:1078D000FF1F2307F7208357810017E7FF1F231B94
:1078E000F7FA094409B3154793F64700B336D000B9
:1078F00093F78703850685C32146638BC7066146D8
:10790000638AC706130680026388C70613068003CE
:107910006393C700914717E6FF1F230BD61C97E61A
:10792000FF1FA387F61C97E7FF1F2384E71C17E7B9
:10793000FF1F034767F69376070497E7FF1F83C788
:10794000B7F58DEE1377770C93067008630CD702AA
:107950001377F7078D466312D70CB307F040B7953E
:107960005B0093F7F70F938505D849A81947ADBF7A
:10797000854755B7894745B78D4771BF930670084E
:107980006311D7021307300FB7150E006389E702A2
:107990001307900DB7B504006383E702130770085F
:1079A00045BF9306800C6311D702B307F040B7754B
:1079B000460013F7F70F938785CDB3D5E70297E716
:1079C000FF1F23A5B712D9BB9306900C631CD700E9
:1079D000B307F04093F5F70F91679387C766B3D568
:1079E000B702F1BF9306A00C631DD700B307F040A8
:1079F000B7153D0093F7F70F93850590B3D5F502C2
:107A00007DBF9306B00CE315D7F4B307F04093F5B0
:107A1000F70F9167938797D0D9B78946631BD70033
:107A2000B307F040B7750B0093F7F70F9385051B6D
:107A3000F1B78546631AD700B307F040DD6593F7C9
:107A4000F70F938565E35DBFD28535FBB305F04045
:107A500093F5F50FB3D5BA029DB783C72400C18B48
:107A600099C7854717E7FF1F230FF706A5BE97E7BE
:107A7000FF1F238A0706BDB6854717E7FF1FA30A26
:107A8000F7068DB63C0017E7FF1F232BF7160947B3
:107A9000930700032314F10097E6FF1F2382E604F7
:107AA0002DBD63940756A94763E5B74217970100B8
:107AB000130747528A05BA959C41BA97828717E403
:107AC000FF1F034454DD894C6306940D63E68C0666
:107AD00085476303F4089307F00F17E7FF1F034779
:107AE000270063F6E70017E7FF1F230BF7FE97EC6D
:107AF000FF1F83CCECFE9307000413F4FC0F63F428
:107B000097011304000497E7FF1F9387670F03ADE6
:107B1000070022862685EA85B38C8C40229D9770CB
:107B20000100E780E0ED97E7FF1F238B97FB97E7C6
:107B3000FF1F23A7A70D45BC8D47630CF40A994787
:107B4000E31BF4F8979701009387474F17E7FF1F50
:107B50002328F70AA94751B717E7FF1F0347A70DC7
:107B600097E7FF1F9387C7F94946979501009385CB
:107B7000E5556306870097950100938525513E855D
:107B800097700100E780C0E717E7FF1F232AA706C9
:107B9000C947A1B797E6FF1F83C6E609054797E7E0
:107BA000FF1F9387E7F56394E6023E851306700294
:107BB000979501009385054F97700100E78040E499
:107BC00017E7FF1F232EA7029307700239B73E85E0
:107BD00013063004979501009385054797700100BF
:107BE000E78000E217E7FF1F232CA700930730046C
:107BF000EDB597E5FF1F83C505CA1795010013056D
:107C0000655697700100E78000EB054D97EDFF1F6B
:107C100083CD6D0297E5FF1F83C5E5C7179501006A
:107C2000130545546398AD0B97700100E780A0E8F9
:107C300097E7FF1F83C727C6B5CBE36EF4E8179419
:107C400001001304E44C638CB70117940100130482
:107C5000A44C63869701179401001304644D228598
:107C600097700100E78040FE1375F50F930715002C
:107C7000860717E7FF1F2305F7E88D4717E7FF1F64
:107C8000A300F7E897E7FF1F938787E70147BE86C2
:107C90001376F70F89076365A60297E7FF1F23A1F5
:107CA000D7F697E7FF1F83C7A7E505BD97970100A4
:107CB0009387073F17E7FF1F2324F7F4914731BD50
:107CC0003306E40003460600A3800700050723806F
:107CD000C7007DBF97700100E780E0DD97E7FF1FD9
:107CE00083C767BBE1D7E368F4DE17940100130490
:107CF000243F638CA701179401001304E43E6386BC
:107D00009701179401001304A43F22859770010086
:107D1000E78080F31375F50F93071500860717E7C3
:107D2000FF1F230FF7DC8D4717E7FF1FA30AF7DCC0
:107D300097E7FF1F9387C7DC0147BE861376F70FCF
:107D40008907E37CA6F43306E40003460600A3801B
:107D5000070005072380C700D5B797E5FF1F83C538
:107D600085B3179501001305A54097700100E780C2
:107D700080D497E7FF1F83C777D893E7470017E7BB
:107D8000FF1FA30DF7D683C7240017E7FF1FA30526
:107D9000F7D689B8179501001305C53E9770010005
:107DA000E78040E997E7FF1F938707D583C7070060
:107DB00017E7FF1F2300F7AE17E4FF1F034444D269
:107DC000333480000DB0179501001305E53C977022
:107DD0000100E78020E697E7FF1F83C737D293E7CC
:107DE000070117E7FF1FA30BF7D083C7240017E78E
:107DF000FF1F2303F7D06FF0EFFE17950100130567
:107E0000E53A97700100E780E0E203C704007D8B4C
:107E100051EFB787004003C767021377C70B13679B
:107E200027002383E70203C7A7021377C70B136753
:107E300027002385E70203C7E7021377C70B136701
:107E400027002387E70203C727031377C70B1367AE
:107E500027002389E702854717E7FF1F230CF7AEAA
:107E600017E7FF1F230AF7BA17E7FF1F2308F7C614
:107E700017E7FF1F2305F7C697E7FF1FA38C07AC83
:107E800097E7FF1FA38A07B897E7FF1FA38807C4D8
:107E900097E7FF1FA38507C497E7FF1FA38C07C4BD
:107EA00097E7FF1FA38907D86FF0CFF389476312C5
:107EB000F70297E7FF1F83C7279E9146638CD70879
:107EC00063E0F604638EE70C6369F70A0547638095
:107ED000E70EFD5717E7FF1FA304F7C03707400061
:107EE000B7E700E023A0E71801000100B7860040D3
:107EF0001306F0FC2381C60223A0E7106FF00FE207
:107F0000130720086382E7086362F702130710086B
:107F1000E391E7FC378700408347670293F7C70B7D
:107F200093E727002303F7026FF0CFEB1307300826
:107F30006389E70213074008E39DE7F837870040AD
:107F40008347270393F7C70B93E727002309F7021B
:107F50006FF04FE9378700408347270393F73707D0
:107F6000F5B7378700408347E70293F7C70B93E7DE
:107F700027002307F7026FF0EFE6378700408347BB
:107F8000E70293F73707F5B7378700408347A70223
:107F900093F7C70B93E727002305F7026FF08FE4F1
:107FA000378700408347A70293F73707F5B737872E
:107FB00000408347670293F73707ADB71795010075
:107FC0001305C51F97700100E780C0C697E7FF1F24
:107FD0002382078CD5B3179501001305251F9770D1
:107FE0000100E78020C597E7FF1F2395078A97E7E1
:107FF000FF1F9387E7AE03C40700894763F3870039
:1080000009441374F40F6FF00FDE13070002E392BC
:10801000E7EC631B0B0A638FF50093072002638371
:10802000F508179501001305E51D97700100E7801D
:1080300080A845B5179501001305051A9770010032
:10804000E78040BF0144179D0100130D2D1AA14C7C
:10805000B387840083C507006A8505049770010013
:10806000E78060A5E31694FF178501001305C56638
:1080700097700100E78000BC17E4FF1F0344C48130
:1080800001E897D7FF1F2389077E014B6FF0AFD51B
:108090008947E310F4E4854717D7FF1F230EF77CC9
:1080A0006FF04FD417D6FF1F0346F67E97D5FF1FFC
:1080B00083C5657E179501001305C51397700100F0
:1080C000E780609F6FF00FD26380F5069307100280
:1080D000E399F5F497D5FF1F83C5057C179501003B
:1080E0001305451397700100E780E09C97E7FF1F99
:1080F00023A897B097E7FF1F9387479F944383D7A1
:10810000470017E7FF1F0347C79E17D6FF1F23230C
:10811000D6781D4497D6FF1F2390F67897D7FF1F78
:10812000238DE7766FF02FCC97D5FF1F83C5C576DB
:10813000179501001305850F97700100E780A09740
:1081400097D7FF1F238A077297D7FF1F23940774BF
:108150006FF02FF92547638FE7C8994637870040AE
:108160006394D70223008702B7E700E0B706400018
:1081700023A0D71801000100130600FC2301C70249
:1081800023A0D7106FF08FB99306100A639FD70012
:1081900023008702B7E700E0B706400023A0D71806
:1081A00001000100130680FCD1BF9306A009E38102
:1081B000D7FE9306400AE38DD7FC93062002639D09
:1081C000D700B7E700E0B706400023A0D7180100AA
:1081D000010023008702F9B78546E384D7FE9307A1
:1081E0000008E300FBFEB7E700E0B706400023A06D
:1081F000D71801000100130620FC23008702BDBF31
:1082000017E7FF1F0347D78D6302F71E63E7E702F7
:1082100095476300F7109947630AF704B786004053
:1082200023800602B7E700E03707400023A0E718E5
:10823000010001001306A0FC75B99307F005630A5D
:10824000F700930750096306F70093071002E3173E
:10825000F7FCB7E700E03707400023A0E71801006C
:108260000100B7860040130620FC69B117EBFF1F21
:10827000034B0B87930700045A8D63F46701130DBA
:10828000000497E7FF1F9387A79783AC0700137439
:10829000FD0F2286E685268597600100E7804076FF
:1082A000B3078B40669417E7FF1F230BF78297E70E
:1082B000FF1F23A78794B7870040630C0B0223801E
:1082C000A703B7E600E03706400023A0C618010068
:1082D000010003C72702134707042381E70203C7EE
:1082E00027021377C70F2381E70223A0C6106FF080
:1082F000EFA22380070237E700E0B7064000232003
:10830000D71801000100130620FC2381C7026FF07B
:10831000AFB9378700408347370097D6FF1F83C622
:10832000B67D93F70708D58FA301F700B706400085
:10833000B7E700E023A0D718010001001306A0FC56
:1083400035BD97E7FF1F9387E78CCA9783C7070060
:1083500093F7F70FC1CF97E7FF1F83C7C78DD9E703
:1083600017D7FF1F0347D777930700026310F7085B
:1083700083AD040017DDFF1F034D0D5297DCFF1F77
:1083800083CC9C5117DBFF1F034B2B51E6876A8779
:10839000DA866E8697D5FF1F83C5054E17950100B7
:1083A000130545EA97600100E780E07097D7FF1F4B
:1083B00023AEB77397D7FF1F238CA77397D7FF1FE1
:1083C000A388977397D7FF1F2385677397D7FF1FDE
:1083D000A383874AB7E700E03707400023A0E718E8
:1083E00001000100B78600406FF04FA2B7E700E040
:1083F0003707400023A0E71801000100B7860040BE
:1084000015BD97E6FF1F83C606830547639CE604F8
:1084100029472381E70209472383E7022385E702EF
:1084200097D7FF1FA388076C97E7FF1FA3850780D7
:10843000B7870040A381070017D7FF1FA30E076A65
:1084400005472383E700B640264496440649F2597F
:10845000625AD25A425BB25B225C925C025DF24D80
:108460006161828029472381E70209472383E7026C
:108470002385E7022387E7022389E70255B717D749
:10848000FF1FA30AF73E6FE01FFF854717D7FF1FA7
:108490002302F74C17D7FF1F2300F75817D7FF1FEA
:1084A000230EF76217D7FF1F230BF7626FE0BFFEA3
:1084B000854717D7FF1F230FF74817D7FF1F230D37
:1084C000F75417D7FF1F230BF76017D7FF1F230899
:1084D000F76017D7FF1FA30F074617D7FF1FA30D7E
:1084E000075217D7FF1FA30B075E97D7FF1FA3885D
:1084F000075E8280411106C697000000E78080FB7E
:10850000B787004023800700130740FC2386E7005D
:108510001307C004A386E70017D7FF1F1307873789
:108520002398E70017D7FF1F1307C73A239AE700DE
:1085300017D7FF1F13074746239CE70017D7FF1FD6
:108540001307C751239EE70029472381E702094704
:108550002383E7022385E7022387E7022389E702D3
:10856000A3810700930600F8A380D700930690022A
:108570002380D700FD562383D7002381E70093068D
:10858000000537E700E0230BD740B7064000232063
:10859000D71003C7170013671700A380E700B24086
:1085A00097D7FF1F239A075441018280411106C6C5
:1085B00097000000E78000F0B787004023800700A5
:1085C000130700FC2386E7003147A386E70017D78F
:1085D000FF1F1307272C2398E70017D7FF1F130748
:1085E000672F239AE70017D7FF1F1307E73A239C4B
:1085F000E70029472381E70209472383E702238510
:10860000E702A3810700930600F8A380D700930632
:1086100090022380D700FD562383D7002381E700F3
:108620009306000537E700E0230BD740B70640006C
:108630002320D71003C7170013671700A380E70094
:10864000B24097D7FF1F2399074A41018280F16703
:108650009387072017D7FF1F232AF748854717D787
:10866000FF1F2317F748A14717D7FF1F2303F7481A
:1086700097D7FF1FA38F074697D7FF1F238C074667
:1086800097D7FF1F238A071E97D7FF1FA385071EB3
:10869000814717D5FF1F1305651EFD5517D6FF1F10
:1086A0001306861E2947B306F5002380B600B306DD
:1086B000F600238006008507E397E7FE97D7FF1FA4
:1086C000A381074297D7FF1FA38F074097D7FF1FAC
:1086D000238A074097D7FF1F2385074097D7FF1F9F
:1086E0002384074097D7FF1FA38E073E97D7FF1F0E
:1086F000238B073E814717D6FF1F1306A65041471D
:10870000B306F600238006008507E39BE7FE828020
:1087100017D7FF1F0347275285476316F700170334
:1087200000006700E3E8170300006700E3DC411185
:1087300022C406C617D7FF1F0347E74F85472E867B
:1087400013F4F50FAA856317F70417D5FF1F130558
:10875000A52897600100E780A02A97D7FF1F238DE7
:10876000072AB787004023848702B7E600E0370670
:10877000400023A0C6180100010003C7A702137719
:10878000C70F2385E702B240224423A0C61001454B
:108790004101828017D5FF1F1305C517976001009F
:1087A000E780002697D7FF1F2386071AB787004068
:1087B00023828702B7E600E03706400023A0C618F0
:1087C0000100010003C767021377C70F2383E70285
:1087D0005DBF411106C697000000E78080E7B24008
:1087E0004101170300006700E3F2411106C697F04C
:1087F000FFFFE78080BF97D7FF1F83C7B715A1CBC7
:1088000097D5FF1F83C5251589C917D5FF1F1305E8
:10881000A51497E0FFFFE780C05397D7FF1FA38BF6
:10882000071297D7FF1F2387072C37E700E0B7060B
:1088300040002320D71801000100378600408347FD
:10884000660293F7370F2303F6022320D710B240B6
:108850004101828041C9D9C597D7FF1F83C7C72966
:10886000D1C3011122CC4AC84EC656C25AC006CE48
:1088700026CA52C42E89AA890144930A0004371BD0
:10888000030063772403B3078940C207C183BE8412
:1088900063F4FA0093040004C204C180130A1BD4D9
:1088A00097D7FF1F83C7070B9DE37D1A631C0A0040
:1088B000F2406244D2444249B249224A924A024BAF
:1088C0000561828097F0FFFFE78020B2D1BF33853A
:1088D00089002694A685420497000000E78060E5A1
:1088E000418045B7828097D7FF1F9387673818422A
:1088F0009C4383D645000345070083C5C700035644
:1089000046006396A50083D5E700638DD50201116B
:1089100006CE2386A7002397D700B705CF00DC4BF0
:108920009385757D05077D162EC2230001003AC48C
:108930002316C1002317D10099C30A858297F240FC
:10894000056182808280DC4DDC4B81CFB7E704007B
:10895000904503A38705914517D5FF1F0345853132
:10896000028382806D713C083EC6B707E500232272
:1089700091103EC8AA843C083285232611103ECAB5
:1089800023248110232021112E8997300000E780B5
:10899000E05C2A84979501009385458E1775010048
:1089A0001305C57097600100E780E010A285179558
:1089B00001001305259D97600100E780C00F294540
:1089C00097600100E7800014B705CB009385757DA3
:1089D000680097100000E7806062A2856800973009
:1089E0000000E780004A014781467000CA8526855D
:1089F00097200000E780E08505CD2A849795010047
:108A00009385C587177501001305456A97600100B6
:108A1000E780600AA28517950100130565979760A6
:108A20000100E7804009294597600100E780800D3B
:108A30008320C110032481108324411003290110D5
:108A40005161828097D7FF1F9387872218429C43EA
:108A5000797122D406D60348070083C807012A8407
:108A600083D64500035546006396080183D8270145
:108A7000638DD8022388070105072399D70037089B
:108A8000CC00DC4B1308787D3ACC1307F5FF42CAC3
:108A900023080100231EE100231FD10099C7080805
:108AA00032C62EC482973246A24522859700000026
:108AB000E78080EBB2502254456182806D713C08A2
:108AC0003EC0B707E5003EC23C083EC42326111055
:108AD0002324811023229110231701002318010061
:108AE00023190100231A0100231B010097B7FF1F60
:108AF00083D7079199E3C167FD172316F10097B754
:108B0000FF1F83D7079091EB97D7FF1F93874716D7
:108B10009C439C43DC4783D7070017B4FF1F130413
:108B2000248E584C2317F10083574400484B2318D8
:108B3000F10031E1978501009385457B17750100B0
:108B40001305C55697600100E780E0F61785010020
:108B50001305057B97600100E780E0F529459760E4
:108B60000100E78020FA8320C110032481108324B0
:108B700041105161828097B7FF1F83C7D78889EB67
:108B8000B7E70400BC5782975C4C23AA0700E1BFFB
:108B9000FD1797B6FF1FA388F68603560701834784
:108BA00004014C470A85230BF10097300000E78051
:108BB000602A97D7FF1F9387A70B9C4301478146E5
:108BC00088430A866C0097100000E7808068AA84BA
:108BD00029C19785010093856571177501001305FB
:108BE000E54C97600100E78000EDA6851785010040
:108BF0001305C57197600100E780E0EB2945976098
:108C00000100E78020F0584CB7E70400BC57484B00
:108C10009DBF97A7FF1F83C7177FF5D7B7E704004E
:108C2000BC4F1044854517D5FF1F0345A504829707
:108C30001DBF5C4EDC4BB9CFB1CD411122C41775BD
:108C400001001305A5462E8497850100938545688C
:108C500006C697600100E78000E6A285178501003F
:108C60001305856D97600100E780E0E42945976072
:108C70000100E78020E9B7E704002244B24003A3E3
:108C8000870517D5FF1F0345E5FE130640069145EE
:108C9000410102838280411122C417A4FF1F1304E3
:108CA000E4731C4C06C689C7DC4399C34C488297C1
:108CB000584CB7E70400BC57484B82975C4CB24015
:108CC000224423AA07004101828017A7FF1F130730
:108CD000E772834707009306F00B850793F7F70FBA
:108CE00063E9F60097A6FF1F238AF6700345070085
:108CF0008280930700F8FDB783574500638607100D
:108D000001114AC817A9FF1F1309896F52C4032A0A
:108D1000C90106CE22CC03274A0126CA4EC656C236
:108D2000F15735E31307D00DFD57636EC704B7E95C
:108D3000040083A709072A841305860042054181A0
:108D4000B284AE8A8297232AAA000325C9015C490E
:108D5000A9E7978501009385A555177501001305AF
:108D6000E53497600100E78000D517850100130501
:108D7000E56497600100E78000D429459760010011
:108D8000E78040D8DD57F2406244D2444249B249BC
:108D9000224A924A3E850561828093874400B70546
:108DA000CF002319F5009385757D310597100000DC
:108DB000E780C0240325C90183456400310597304D
:108DC0000000E780000C0325C9012686D685310501
:108DD00097300000E78000087146A2854A859760B9
:108DE0000100E780E0C1504419CA83A78905854581
:108DF00017D5FF1F034505E88297814769B797009C
:108E00000000E780E0CBD5BFFD573E858280411151
:108E100026C297A4FF1F9384A45ED84C22C437E4D3
:108E200004003C54484B06C68297DC4C0323C4051F
:108E30002244B240924423AA070017D5FF1F0345DE
:108E400065E3854541010283411126C297D4FF1F86
:108E5000938404E29C4006C622C44AC0D5C3DC43C6
:108E6000C5C35CC12300B5002A84978501009385A2
:108E7000653F177501001305652397600100E780C2
:108E800080C3294597600100E780C0C79C4023A4A8
:108E9000070023A2070097A7FF1F93872754DC4FE3
:108EA000DC4B91C7295597000000E78000DF97A7AA
:108EB000FF1F9387E754DC4FDC4B89C79700000006
:108EC000E78020F537E904008327C905894517D5D0
:108ED000FF1F034525DA82978327C905914517D5DA
:108EE000FF1F034525D982979C4003A347016309CF
:108EF000030022852244B240924402494101028388
:108F0000B2402244924402494101828001113285DB
:108F100006CE22CC26CA2E8497300000E7800004BB
:108F2000AA849785010093852537177501001305DD
:108F3000E51797600100E78000B803078400035637
:108F4000640083554400A686178501001305C540BB
:108F500097600100E78020B6294597600100E7800F
:108F600060BA97A7FF1F83C7C747639D9700014556
:108F700097000000E78060D281450A8597000000D5
:108F8000E780C0ECF2406244D244056182806D719A
:108F900023248110232611102322911093F74500DA
:108FA0002E84638707143C083EC0B707E5003EC225
:108FB0003C083EC4231701002318010023190100B7
:108FC000231A0100231B010097A7FF1F83D7074126
:108FD00099E3C167FD172316F10097A7FF1F83D7F9
:108FE000074091EB97D7FF1F938787C89C439C430B
:108FF000DC4783D7070017A7FF1F1307273E231758
:10900000F100544F835747002318F100DC4AA1E7D1
:10901000978501009385852C1775010013050509B7
:1090200097600100E78020A9178501001305452DF1
:1090300097600100E78020A8294597600100E7803C
:1090400060AC134544008320C110032481108324A5
:1090500041105161828097A7FF1F83C7973825551C
:10906000D9C3FD1717A6FF1FA30DF63603D60601B9
:1090700083470701CC460A85230BF1009730000097
:10908000E78040DD97D7FF1F938787BE9C4317A7D4
:10909000FF1F1307A734978601009386662988432C
:1090A0000A866C0097100000E780A01AAA8451D9A4
:1090B000978501009385852217750100130505FF2B
:1090C00097600100E780209FA685178501001305A2
:1090D000E52397600100E780009E29459760010025
:1090E000E78040A2268597000000E78000BB91BF83
:1090F00093F725009DC7B7E70400BC47414681456B
:1091000028088297255597000000E78000B92808B5
:109110009305F00F97000000E78040D3134524002B
:109120001DB793F71500014599DF97000000E78010
:1091300020991345140001BF5C4D411106C688C338
:1091400017D7FF1F2326F7B2B7E7040083A7070846
:10915000170500001305E5E38297B24097D7FF1F7C
:10916000238AA7B001454101828001113335A00057
:10917000A307A100B7E7040083A7471706CE13068D
:10918000F1008545130550308297F24005618280D9
:109190008280411122C406C697D7FF1F83C707AF3D
:1091A000014489EF97B7FF1F83C79708054499E7E4
:1091B00017B4FF1F0344C40713441400228597000B
:1091C0000000E780C0FA178501001305252A09E48D
:1091D000178501001305852A2244B2404101176317
:1091E00001006700438D41119397050122C406C613
:1091F00026C2C1872E8463D40702B7E40400FC545E
:1092000017A5FF1F0345C522829719C1BC54829739
:109210002165218DB240224492444101828093F71E
:1092200015008DC7B7E7040083A7471A17A6FF1FCD
:109230001306061F97D5FF1F938585A417A5FF1F4B
:109240000345051F829713451400E9B793F72500DE
:1092500099CFB7E70400BC4F13060064894517A5F2
:10926000FF1F0345E51C82971345240065B793F75C
:10927000850085CF97D7FF1F83C707A285E7B7E78C
:10928000040003A8871A1307401F97A7FF1F83C76F
:10929000271A814613064006994517D5FF1F035527
:1092A000259F029813458400B5B793F74500014503
:1092B000B5D3B7E4040083A7041817D5FF1F0355DF
:1092C000259D8297BC4C13060064914517A5FF1F8E
:1092D000034505168297134544002DBF97D7FF1FFE
:1092E00083D7079B6398A70217D7FF1F2313B79A4B
:1092F00017D7FF1F2310C79A17D7FF1F231DD79813
:109300002E86178501001305E51DBE851753010044
:109310006700637A178501001305451E1763010076
:10932000670043910357450097D7FF1F83D74796A0
:10933000631EF704C1674111F91722C417D7FF1F35
:109340002328F79437E4040097D7FF1F23A407943A
:1093500097D7FF1FA38C079297D7FF1F238E0792E3
:109360007C4C06C6894517A5FF1F0345650C8297EF
:109370007C4C914517A5FF1F0345850B829722441E
:10938000B2404101170300006700E3E017850100C8
:109390001305C516176301006700C3897D1595473E
:1093A00063E2A71C178701001307C70A0A053A954D
:1093B0001C41011122CC06CEBA972E8482871785D4
:1093C00001001305251497600100E780A086A1A283
:1093D00003C7250099476311F7022E859700000007
:1093E000E78080F48345640017850100130585122A
:1093F00097500100E780206C97B7FF1F238A07E290
:10940000178501001305C5127DBF03C725009547C9
:109410006319F702C16717D7FF1F03576787F9174B
:1094200003D5A5006309F702B7E7040083A7C717B0
:109430008297178501001305A51097500100E7805A
:10944000607F854717B7FF1F2304F7DE17850100EC
:10945000130585118DBF97D7FF1F239BA78283D745
:10946000E50097D6FF1F2396F68283D7050197D68E
:10947000FF1F2391F68283D7250197D6FF1F239CD8
:10948000F68097D7FF1FA3830780631BE502B7E72A
:109490000400BC4F096613060690A14517A5FF1FDF
:1094A000034505F982970356E4008355A400178508
:1094B00001001305250A97500100E780C05F51B7EE
:1094C0009307700F2316F100B7E7040083A7870DF9
:1094D00017A6FF1F0346C6F56C0082974DF9854716
:1094E00017C7FF1FA304F77A5DB71785010013059F
:1094F0006508D1BD83C5250091476392F5021785A4
:1095000001001305A50897500100E780A07297009D
:109510000000E78040C8F2406244056182809947BC
:109520006392F502228597000000E780E0DF834523
:109530006400178501001305E5FD97500100E780E1
:109540008057D1BF9547639AF50083471400E1F334
:10955000178501001305C505BDB517850100130565
:10956000A505E1BF82803757315F97A7FF1F93871B
:1095700067ED130777D598C39356C5001787010089
:10958000130707F3BA9683C5060093568500BD8A74
:10959000BA9603C6060093564500BD8A3D89BA9621
:1095A0002A9783C606000347070023840700238306
:1095B000D700A383E7002382B700A382C70097A741
:1095C000FF1F938727E92383B700A383C700238462
:1095D000D700A384E7008280411106C622C4970009
:1095E0000000E78080F837E404008327841417A67E
:1095F000FF1F130626E5D54501458297032344172F
:109600002244B24017A6FF1F1306C6E4CD4513053A
:1096100070304101028361712324811A37E4040010
:10962000832704082326111A2322911A2320211BA1
:10963000232E311917050000130525BB829717A9A2
:10964000FF1F1309E9DE994785442300A900231C65
:10965000F100978501009385A5E4930740061775EF
:1096600001001305A5A4231CF1082308910097C944
:10967000FF1F9389890C97500100E780C04383D571
:109680000900178501001305A5E097500100E78048
:109690008042294597500100E780C04603D5090064
:1096A000896997000000E78040EC83274417100881
:1096B00085451305503082978327441717A6FF1F4F
:1096C000130646D9CD45130570308297832744177A
:1096D00017A6FF1F130606D6B545130560308297FF
:1096E0008327441730088945130510318297832753
:1096F0004417300989451305203182978327441583
:10970000938509900D458297832744159385099089
:1097100011458297A30591002306910002CD2308ED
:109720000100230C0100832784163009914513059D
:1097300070408297832784161306B1008545130570
:1097400000408297832784167000854513051040DA
:109750008297832784163008854513052040829719
:109760008327841610088545130550408297832768
:1097700004157D558297832744137D5582977D5527
:1097800097A0FFFFE78000F28327440C829797A001
:10979000FFFFE780C0CB8327841417A6FF1F1306A3
:1097A00066CAD5450145829789471306700F8145E2
:1097B00028092306F1009790FFFFE78040958D4729
:1097C0001306000881452808230CF1089790FFFF35
:1097D000E780E0939147230CF1009767010093879E
:1097E000677E984383C747003AC8230AF10097D0A1
:1097F000FFFFE780A0BA70008545054597A0FFFFF1
:10980000E78060F130099305700F094597A0FFFFCD
:10981000E78060F03008930500080D4597A0FFFF32
:10982000E78060EF10089545114597A0FFFFE7809E
:1098300080EEC16717C7FF1F13078745F9171CC3C1
:109840002322070017A5FF1F130545BE97A0FFFFA2
:10985000E78040EB8327C41D17C5FF1F1305C541D3
:1098600082973C4803450900854582978320C11AA9
:109870000324811A8324411A0329011A8329C11957
:109880005D618280C16717C8FF1F03586840F917E0
:109890006301F8083DCDB5CD011126CAB7E4040037
:1098A00083A7841222CC2E862315B10006CE2A84EB
:1098B00001478146ED45428582972AC611ED1785FD
:1098C0000100130525C097500100E780A036F24043
:1098D0006244D24405618280FC440356A100A28503
:1098E00082972C0017C5FF1F0355853A97A0FFFFED
:1098F000E78020F169DD178501001305E5BD97506C
:109900000100E780203383A7C412ED452800829729
:109910007DBF828015C5854717A7FF1FA301F7B23A
:1099200097A7FF1F238E07B0B7E7040003A34717CD
:1099300017A6FF1F130606B0B54513056030028356
:1099400097A7FF1FA38D07AEE1BF97C7FF1F83C770
:10995000A734A9EFC16717C7FF1F03576733F9176C
:109960006306F7044111854722C417C7FF1F23056B
:10997000F73237E404007C4C06C6A14517A5FF1F4B
:10998000034505AB82970323841A2244B24097A76C
:10999000FF1F83C7E7A917C5FF1F0355652F1307CF
:1099A000401F8146314699454101028382806D7195
:1099B000232481102326111023229110328401CDFB
:1099C0008947630AF5028320C11003248110832490
:1099D000411051618280178501001305A5BEAE8438
:1099E00097500100E7800025A285268597C0FFFFDC
:1099F000E780A0B9C9BFB7E70400FC4728008297F9
:109A0000178501001305C5BC97500100E78080222F
:109A10008347810039C41307000B6380E702138773
:109A2000A7051377F70F8D4663EDE602A2852800A0
:109A300097C0FFFFE780202A79B78547E3F587F8CD
:109A4000834591001775010013058597B335B00064
:109A500097A7FF1F238AB76497500100E780A005EE
:109A60009DB703479100A207D98F35671307D755D4
:109A70006385E7086368F7022D671307B7556387A7
:109A8000E70631671307C755638AE7042967130799
:109A9000A7556394E702A285280097C0FFFFE780DF
:109AA000806215B739679306E7656381D70863E974
:109AB000F6001307E7556384E706A28528003DB743
:109AC0003D679306F755638AD7061307F766E39653
:109AD000E7FE97C0FFFFE780007BF5B50146A28552
:109AE000280097C0FFFFE780A04AF1BDA2852800AB
:109AF00097C0FFFFE780605BF9B58947E3F587EC26
:109B000097000000E780A0E49305E4FFC205C1814F
:109B10001305A1009790FFFFE780806C6DB5A285CB
:109B2000280097C0FFFFE780005B71BDA285280079
:109B300097C0FFFFE780C06579B597C0FFFFE7805A
:109B4000406E51B5C16717C5FF1F03556514F9175E
:109B50006307F500B7E7040003A3C71702838280F9
:109B6000854717C7FF1F2303F712014517F3FFFFB0
:109B70006700E35F1783FFFFE702C3542A840845A9
:109B80002E89B28919C900C1971500009385A58651
:109B9000610597300100E780200581447D5A9710C8
:109BA0000000E780E03963C7A404814497100000F7
:109BB000E780003A63C8A40497C7FF1F9387070E86
:109BC0009C43DC47B307F94091872302F400638389
:109BD00009048327C900B307F4409587A302F40062
:109BE0001C4C89C79C4799C3228582971783FFFF26
:109BF000670083505C44139714008504BA97239040
:109C0000470171BF1C48139714008504BA9723902D
:109C1000070069BF832789000547B307F44095878C
:109C2000A302F40083570400638EE7028DC3094743
:109C30006384E7040D47E395E7FA9787010093876C
:109C4000E7EB1CCC97870100938747EC11A8978717
:109C50000100938727B21CCC97870100938787B2B6
:109C60005CC8BDBF978701009387C79D1CCC9787B1
:109C700001009387279EEDB7978701009387C7EC74
:109C80001CCC97870100938727EDD9BF95E51783F3
:109C9000FFFFE702C34400461844834794007583DE
:109CA0009D8B6317F70097100000E78060B448C4ED
:109CB0001783FFFF6700E34482801783FFFFE702FB
:109CC000634013893500C16442094111AA890144E6
:109CD000F11413590901054A2EC697100000E780B8
:109CE0002026B2456348A400014541011783FFFFC8
:109CF0006700834083A7090013171400BA9783D71E
:109D000007006388B7006394970063742A01050411
:109D1000E1B70545D9BF1783FFFFE702C339AA8919
:109D20002E89328BB6843A8ABE8A97A00000E780DB
:109D3000C0FE71C9268597200000E780C00C8D47C2
:109D400063E7A7007D551783FFFF6700433A83DB76
:109D5000440097100000E780A0242A849710000098
:109D6000E78040259307740031443305850263CDB5
:109D7000A70297100000E780A02297100000E7805C
:109D800020222A8497100000E780C02293077400E5
:109D900031443305850263C3A70497100000E780B0
:109DA00020209307450029A897100000E780802015
:109DB000330585021307F0179307C017E35FA7FA6F
:109DC0002D55E3C277F963040B02D6865286A68529
:109DD0004A8597200100E780C0BDB5B79710000005
:109DE000E780401D330585029307C5FFD1BF832758
:109DF00049001385C90083D5270097000000E7803C
:109E000000EC61F581B769553DBF97C7FF1F2399E6
:109E1000A7E897C7FF1F938767E8904381470C46E1
:109E20003307F500420741836393B70082805446AD
:109E3000139847008507C2962390E600D5B797C7C9
:109E4000FF1F9387A7E59C4303C58700828017C542
:109E5000FF1F0355E5E482801783FFFFE7022328F5
:109E6000C1671387D7FF630BE502636AA700F11789
:109E70006300F50201451783FFFF670083281387FE
:109E8000E7FF6302E502FD171D8D13351500E5B7E9
:109E900097500000E780602A7D15C5BF97500000ED
:109EA000E780E0FED5BF97500000E78000FDEDB7EA
:109EB0001783FFFFE702A3224111AA8401442EC6A3
:109EC00097100000E780C008B2456348A400014530
:109ED00041011783FFFF6700C3229C48131514003C
:109EE0003E9583570500E385B7FE0504C9BF0348C7
:109EF0005500814693F7F60F63E5070181473E85DC
:109F00008280584593975600BA9703D72700631667
:109F1000B70003D70700E304C7FE8506E1BF834609
:109F2000450001479377F70F63E4D700814711A8F5
:109F30001C45131657000507B29703D60700E31315
:109F4000B6FE3E8582801783FFFFE702A3179317B3
:109F50000501C18797CAFF1F938A4AD4635BF00843
:109F600083A70A00C0479C4703570400198D420588
:109F700041816368F500014422851783FFFF670074
:109F8000A31712052A94CDBFDC4713944900014A58
:109F90003E94834744006341FA02014A83475400D8
:109FA0006349FA028509C20993D9090183A70A0006
:109FB0009847E3EBE9FCC1B71C4413195A00A68586
:109FC0003E994A8597000000E780C0EE05E1050A4A
:109FD000C9B75C4413195A00A6853E994A85970073
:109FE0000000E78020ED19E1050A4DBFE30C09FAF6
:109FF00061B7AA8481495DBF1783FFFFE702230E83
:10A000001C452A8481E79307C5001CC51C44231204
:10A0100004001CC09307F00F63EDB70093F5F50F34
:10A02000228597200000E780C0E51783FFFF6700C7
:10A03000430D93940501C167C18063F9F500A685BE
:10A04000228597200000E780E0E8C5B7C18193F53D
:10A05000F50F228597200000E780A0E2A6852285E3
:10A0600097200000E780E0E3C9B797C7FF1F9387F9
:10A07000E7C2884382801C4599C797C7FF1F23AF5B
:10A08000A7C0014582807D55828097C7FF1F9387B7
:10A09000E7C0984383474500484792073E95828032
:10A0A0001783FFFFE702A303617100451C183EC63A
:10A0B000B70780013EC81C183ECA8357440002CE31
:10A0C00002D002CC231EF100834784002A8902D2E9
:10A0D0002301F1023C083ED402D697000000E7803D
:10A0E00000FB835705002316F10297500000E7801C
:10A0F00000C82307A1025C4003556400F18313F7F5
:10A1000017008347F10252055181F99BD98FA307AC
:10A11000F10297100100E780207939CDAA84035518
:10A12000050097A00000E78020C083D704002AD252
:10A130006800231CF10083D72400231DF1001C4874
:10A1400003D647008C4397200000E780A0D08347C8
:10A15000B400CA8617760100130646488117A30586
:10A16000F4006C00481097200100E78080845D6156
:10A170001783FFFF6700E3F82155D5BF1C45B1CF1A
:10A1800003C5A700894613576500630BD7028D46A8
:10A19000630ED70285466300D702130740063305D6
:10A1A000E50203C7B700418B15CB83C7B700BD8B52
:10A1B0003355F54082801375F5031307803EC5B70C
:10A1C00009671375F50313070771D1BF3727090016
:10A1D0001375F5031307077CD9B7014582801783F0
:10A1E000FFFFE702C3EF03A98500630C090483475F
:10A1F000B900AE8493F7070E85C303459900930514
:10A2000020030D810505B305B5028844610597302B
:10A210000100E78080AD35A02E8597000000E78023
:10A2200020F62A8419CD97000000E780605C832522
:10A23000C900B307B54063FA87002E94B305A44064
:10A24000E9F51783FFFF6700C3EB85457DBF1783E3
:10A25000FFFFE702C3E82A8403D50500011132C6D7
:10A2600036C43AC22EC002CA02CC02CE97A0000069
:10A27000E78080AB82452ACA22852ECC9700000059
:10A28000E780E0E003570500231EE100975000003F
:10A29000E780E0ADA24632469247230FA100368701
:10A2A0004C08B2862285014697000000E780E0A6B0
:10A2B00005611783FFFF6700C3E41783FFFFE70211
:10A2C00003E261711C183EC6B70780013EC81C1826
:10A2D0003ECA3C0800453ED4AA8402CC02CE02D03D
:10A2E00002D202D697000000E78060DA83570500AB
:10A2F00035592316F10297500000E78040A7230745
:10A30000A10209C48357440081EB21594A855D614C
:10A310001783FFFF6700E3DE035564005205518198
:10A3200097100100E78040582A8965D18347B4001F
:10A3300093F7070E99C71305840197300100E78052
:10A34000009D83574400231EF100834784002301AE
:10A35000F1025C4003550900D98313F707088347CE
:10A360001102231CA10093F7F707D98FA300F10274
:10A3700083572900231DF1005C40F18313F7170078
:10A380008347F102F99BD98FA307F10297A0000040
:10A39000E78080992AD235D98347940068001397C3
:10A3A00057008347B400FD8BD98FA305F4001C48E8
:10A3B00003D647008C4397200000E780A0A9A6871A
:10A3C0001777010013078721740005464C10268576
:10A3D00097000000E78060942A890DD98347B40074
:10A3E000A685FD8BA305F40097000000E78060DFE1
:10A3F00031BF1783FFFFE70283CE832485FE2A84C3
:10A400004111268597000000E78080D7834734FFFD
:10A4100093F7070E8DCB2AC6268597000000E780AC
:10A4200060C809CD834734FFB245FD8BA309F4FE14
:10A4300091C5228597300100E780208B4101178369
:10A44000FFFF670003CC7DD98327C4FF2685829751
:10A4500075F5834734FF93F7070E91C72285973030
:10A460000100E780C08A032584FE97000000E78092
:10A4700000E5E9B71783FFFFE70263C39C41411181
:10A480002A8903C7070089472E8493566700638093
:10A49000F6040D466388C6049307F0076304F702C9
:10A4A0002E8597200000E78060ABAA848149C16BAC
:10A4B000130C490097B7FF1F9387477E9C4398472B
:10A4C00063E4E90441011783FFFF670003C203D778
:10A4D00045008547E3F8E7FE2E8597200000E780DA
:10A4E00040ADE1B703D74500E3FEE7FC2E8597209A
:10A4F0000000E780A0A6AA84228597200000E780BC
:10A5000000A8C204C98C5DB7DC470355A900139AA3
:10A5100049003E9A93170501C187635DF000835798
:10A520000A006397A70263E774038327CA00034DF9
:10A530005A002DA0A1672167A98F1307F7EFE374D5
:10A54000F7FE6397090097000000E780209161FD06
:10A5500085098DB783278A00034D4A00835DA900D2
:10A5600003576900216A138BC7003AC6814A33CA70
:10A570004D01631E5D0197B7FF1F9387A7729C4330
:10A58000E1DBA2866286814526858297D1B7A167E5
:10A590009387F7EF930C4BFF63F24703B2455A855D
:10A5A00097F0FFFFE780A0710DC103278B001047D4
:10A5B00009CE10436382C4023107D5BFEE8566859C
:10A5C00097000000E780008F71F993861A0093FAD4
:10A5D000F60F130B0B0271BF835644005C43E3E993
:10A5E000F6F622853AC697200000E7802081A16711
:10A5F0009387D7042A8A035D4400324763E89700B3
:10A600008347D90093E707F8A306F9001C4766853E
:10A610002286E2858297C1670844FD17337AFA00E3
:10A62000529508C02312A40125B797B7FF1F93873F
:10A63000E7669843814715C31447814763FFD500F8
:10A64000939745004C47BE9519C903C755008147EC
:10A650006375E600DC451606B2973E85828003C727
:10A6600045008147E37BE6FE16069C45F5B7178358
:10A67000FFFFE70223A5AA892E8A814497BAFF1F0C
:10A68000938ACA6183A70A00984763E6E4001783A8
:10A69000FFFF670063A6DC471394440001493E9422
:10A6A00013BB140083474400634BF900014913BBFB
:10A6B000140083475400634FF9008504E1B7084450
:10A6C000931759005287DA860146A2853E958299F2
:10A6D0000509C9BF4844931759005287DA860546D1
:10A6E000A2853E9582990509E9B71783FFFFE70226
:10A6F000039F814517F5FFFF1305054897B7FF1F17
:10A700002390075A97000000E780A0F61783FFFF09
:10A710006700239F97B7FF1F938747589C4395C3B4
:10A720001783FFFFE702A39B814517F5FFFF130582
:10A73000A54497000000E780C0F31783FFFF670080
:10A74000439C82801783FFFFE702C39737E404002E
:10A750008327841241112315E100AE893289368A9C
:10A760003A8681460147ED45AA8482972AC621C9C7
:10A770000356A100D28597400100E7806028832717
:10A78000C413CE8526858297058905C98327440D84
:10A790002314210101462C00268582972A8401C9B1
:10A7A000B7E7040083A7C712ED45280082972285EA
:10A7B00041011783FFFF670023944944D5B76554CF
:10A7C000FDB75C41FD175CC182801783FFFFE70284
:10A7D0000391B7E70400FC5F829795473305F502C4
:10A7E00081450D811783FFFF6700A3911783FFFF4A
:10A7F000E702E38EB7E70400FC5F829795473305D5
:10A80000F5020D811783FFFF6700A38F1783FFFFFA
:10A81000E702E38CB7E7040083A7870B0355050025
:10A8200082971783FFFF6700C38D1783FFFFE7023F
:10A83000038B035505003287AE861796FF1F03561C
:10A8400086C797B5FF1F9385254697000000E780D0
:10A85000A0EF1783FFFF6700C38A1783FFFFE7029C
:10A860000388B7E7040083A7C71782971783FFFF02
:10A87000670023891783FFFFE7026386B7E70400B9
:10A8800083A7871397B5FF1F9385054282970145DC
:10A890001783FFFF6700E3861783FFFFE702238428
:10A8A000B7E7040083A7C71F81451795FF1F03550E
:10A8B00085BC82971783FFFF6700A3841783FFFF80
:10A8C000E702E381B7E7040083A7871397B5FF1F6B
:10A8D0009385853E829701451783FFFF670063825A
:10A8E0001773FFFFE702A37FB7E7040083A7C71F23
:10A8F00081451795FF1F035505BE82971783FFFFFC
:10A90000670023801773FFFFE702637D2E85978022
:10A910000000E78080B397800000E78080F0177325
:10A92000FFFF6700037E1773FFFFE702437B9780FB
:10A930000000E78080FA1773FFFF6700837C5C49A3
:10A94000E1175CC95CC583572501A1072319F500F0
:10A9500083570501A1072318F5008280F1473305CD
:10A96000F50297B7FF1F938727379C433E95828058
:10A970008D476315F60803D74600854763F0E7085F
:10A980001773FFFFE702A375368536842E8997106B
:10A990000000E780A05C29C9835744009314050197
:10A9A000C18063E39704228597100000E780005B75
:10A9B000FD14231294009307A0026300F50293078D
:10A9C000B0026307F50293079002631FF50022852A
:10A9D00097000100E780608901A80146CA852285A9
:10A9E00097A00000E78000B41773FFFF6700637152
:10A9F000228597100000E7806007FDB7828097B638
:10AA0000FF1F9386A62D9C42014599CF9843D442BF
:10AA100017B6FF1F2324E62C6396D70097B6FF1FB7
:10AA200023A0E62C1385C7FE82801773FFFFE70281
:10AA3000036B97000000E780A04B7144330585024B
:10AA4000914597900000E780C0EC11E565551773BC
:10AA5000FFFF6700036B97B7FF1F23ADA726970083
:10AA60000000E780E048330585029145979000009B
:10AA7000E78020EA61DD97B7FF1F23AFA724970087
:10AA80000000E780E04697B7FF1F239FA7229700AB
:10AA90000000E780E04597B7FF1F2398A72297772C
:10AAA00001009387E7B817B7FF1F2323F722970703
:10AAB0000000938707E917B7FF1F2329F7200145F7
:10AAC00079B71773FFFFE7028361AA8517B5FF1FE8
:10AAD0001305851F97100000E780605F1773FFFF65
:10AAE000670023621773FFFFE702635F97000000B0
:10AAF000E78060FD97100000E780E05E97B7FF1FDA
:10AB00009387C71D9C4391CF1387C7FE19CB83D56D
:10AB1000C7FF17B5FF1F1305E51C97200100E7804D
:10AB2000C01C1773FFFF6700C35D1773FFFFE702C9
:10AB3000035B97000000E780C0EC09CD83478500E8
:10AB40002A8493F7070499EB0355E500970000006A
:10AB5000E78080F91773FFFF6700A35A8347C5009A
:10AB60009304450117B9FF1F1309491785E383278C
:10AB700009005CC997B7FF1F23A2971683274900D6
:10AB8000F1FB97B7FF1F23AD9714E9B7FD17230615
:10AB9000F500610597800000E78060DA8307840094
:10ABA00063CB07048347840093E707F82304F4008A
:10ABB000B7E704009C5F82974205A947418133753E
:10ABC000F5028347840093F707FCC98F2304F40040
:10ABD0008347D4003E951C402318A40089CF984396
:10ABE00019CB8347C4005040814585073305F502E2
:10ABF000420541810297832709005CC897B7FF1F70
:10AC000023AE970C8327490089E797B7FF1F23A935
:10AC1000970C8347C4009DDF8355040117B5FF1FC0
:10AC20001305450C97200100E780200C25B717730A
:10AC3000FFFFE702C34A97B7FF1F9387E72F9C47A1
:10AC400001448583858B85E3AE84B2853A8697106F
:10AC50000000E780204F2A8419C597100000E78084
:10AC60006045829408CC22851773FFFF6700634913
:10AC70001773FFFFE702034541112E8932C6AA89E7
:10AC800097000000E780C031324713060502CA86EC
:10AC9000970500009385C5CC17B5FF1F1305C502A6
:10ACA00097000000E780E0F82A8425C99304C500D6
:10ACB00097000000E780E0411946AA852685971095
:10ACC0000000E78020198545268597100000E78061
:10ACD000001517750100130565934E958345050012
:10ACE000268597100000E780C0195C4831468145F1
:10ACF000A1075CC85CC483572401E1172319F40041
:10AD000083570401E1172318F4001C4C3E8597700B
:10AD1000FFFFE780C03FA30425012285410117738F
:10AD2000FFFF6700633D1773FFFFE702433B4111DD
:10AD3000AA842EC632C497100000E780003A004D66
:10AD4000B2452246834784000CC050C093F7F703F6
:10AD500093E707042304F4002318040026859710C2
:10AD60000000E780203583479400A9462317A400FC
:10AD700013D7370005073307D7029D8B85072306B6
:10AD8000F400A306E40083C70401D8488507230F15
:10AD9000F7FE17B7FF1F130767F45843232A040071
:10ADA0009307440129E317B7FF1F232BF7F217B7C7
:10ADB000FF1F2325F7F217B4FF1F1304A4F2228507
:10ADC00097200100E780A0E41C44858B5D8D19E588
:10ADD0008145228597200100E78020F1410117730A
:10ADE000FFFF670003321CC317B7FF1F232AF7EECC
:10ADF000D9B71773FFFFE702832E970500009385ED
:10AE000065B7014597000000E78000B00145177362
:10AE1000FFFF6700032F1773FFFFE702432C970024
:10AE20000000E78080B01773FFFF6700832D834722
:10AE3000C500A5E31773FFFFE702632A2A840355C1
:10AE4000E50097000000E78000C821C18347840027
:10AE500093F7F7FB2304F4001C4091C7DC4381C740
:10AE60004C400145829797000000E78080B917B5F4
:10AE7000FF1F130525E797200100E78040E90355F0
:10AE8000E40097000000E78020C61773FFFF67000B
:10AE9000432782801773FFFFE702632497B7FF1FE2
:10AEA0009387C7E397050000938565C817B5FF1F13
:10AEB000130545E323A0070023A207009720010004
:10AEC000E78080D21773FFFF6700A3231C4D91CF4B
:10AED000DC4381CF1773FFFFE70263208345070040
:10AEE00082971773FFFF6700C321828097B7FF1F08
:10AEF000938787E19C4303C50700828097B7FF1FB4
:10AF0000938787E09C4303C51700828097B7FF1F94
:10AF1000938787DF9C4303C52700828097B7FF1F75
:10AF2000938787DE9C4303C54700828097B7FF1F46
:10AF3000938787DD9C4303C53700828097B7FF1F47
:10AF4000938787DC9C4303C55700828097B7FF1F18
:10AF5000938787DB9C4303C56700828097B7FF1FF9
:10AF6000938787DA9C4303C57700828097B7FF1FDA
:10AF7000938787D99C4303C58700828097B7FF1FBB
:10AF8000938787D89C4303C59700828097B7FF1F9C
:10AF9000938787D79C4303C5A700828097B7FF1F7D
:10AFA000938787D69C4303C5B70011E11D45828076
:10AFB00097B7FF1F938747D59C4303C5C70082807F
:10AFC00097B7FF1F938747D49C4303C5D700828060
:10AFD00097B7FF1F938747D39C4303C5E700828041
:10AFE00097B7FF1F938747D29C4303D50701828001
:10AFF00097B7FF1F938747D19C4303C527018280E2
:10B0000097B7FF1F938747D09C4303D547018280A2
:10B0100097B7FF1F938747CF9C4303D56701828073
:10B0200097B7FF1F938747CE9C4303D58701828044
:10B0300097B7FF1F938747CD9C4303C5A701828025
:10B0400097B7FF1F938747CC9C4303C5B701828006
:10B0500097B7FF1F938747CB9C4303C5C7018280E7
:10B0600097B7FF1F938747CA9C4303C5D7018280C8
:10B0700097B7FF1F938747C99C438857828097B72C
:10B08000FF1F938767C89C4303D5C702828097B789
:10B09000FF1F938767C79C4303D5E70219E1130598
:10B0A000800C828097B7FF1F938707C69C4303C518
:10B0B0000703828097B7FF1F938707C59C43C85B30
:10B0C000828097B7FF1F9387A7C38843828097B773
:10B0D000FF1F938727C38843828019E17D558280B3
:10B0E000F5DE984265DFFDD917B7FF1F1307C7E4E8
:10B0F0001847AA877155058B631D072403C50700F0
:10B100001547E37DA7FC03C737001305F0057D173E
:10B110001377F70FE364E5FC03C35700E30003FC78
:10B1200083C86700E38C08FA03C77700494579179D
:10B130001377F70FE364E5FA03C7A7001148130577
:10B14000F7FF1375F50FE36BA8F803CE97000D48D2
:10B150001305FEFF1375F50FE362A8F803C8B700E7
:10B160006309080065181378F80F1305600DE3678D
:10B1700005F703C5C700794879151375F50FE36F17
:10B18000A8F403C8D7000D457D181378F80FE367BE
:10B1900005F503D80701930E4017511842081358BC
:10B1A0000801E3ED0EF303C8E7007D181378F80FEC
:10B1B000E36605F303C827017D181378F80FE36FE2
:10B1C00005F103C88700C54E75181378F80FE3E73B
:10B1D0000EF103D86701856E938EBEE06D184208AC
:10B1E00013580801E3EC0EEF03D847016D1842082D
:10B1F00013580801E3E40EEF03D8870179184208D9
:10B2000013580801E36C05ED03C8A7017D181378F6
:10B21000F80FE36505ED03C5B7011D487D151375EE
:10B22000F50FE36DA8EA03C5D701714879151375C9
:10B23000F50FE365A8EA03D5E7011308E00F7D15D4
:10B2400042054181E36CA8E803C507024948791526
:10B250001375F50FE364A8E8C85301C937C8340073
:10B260005915130858BFE36BA8E603A8870237C532
:10B270003400130555BF5918E36205E717B5FF1FE2
:10B280002322C5A803C6050117B5FF1F232EF5A667
:10B290000545E375C5E403D82501D0493376060397
:10B2A000E31E06E203C61501E30A06E217B6FF1F16
:10B2B0002328B6A483C5270001466387A50003C6DB
:10B2C0001700F1453306B60283C707039305C00292
:10B2D00072971A071307C70516031A979608469719
:10B2E000B387B70241553E97329742074183636265
:10B2F000E8061773FFFFE70283DE368597800000BC
:10B30000E780406C97000100E780C04B2A8497A03B
:10B310000000E780205E2A9497F00000E780002A72
:10B320002A9497900000E78040852A9497F0FFFFC9
:10B33000E780E06F2A9497400000E78000972A9406
:10B3400097700000E78040A022951773FFFF670009
:10B3500043DB82801773FFFFE70263D84111A30725
:10B36000A10097A00000E78040C99305F1001705F0
:10B3700000001305E5B597F0FFFFE780802F01453A
:10B3800041011773FFFF6700C3D71773FFFFE70281
:10B3900083D217B4FF1F130424BA032884007959F9
:10B3A0009368180097B4FF1F23AC14B913781800E2
:10B3B00063100802BA84BE89368B328A2E89AA8A23
:10B3C00097F0FFFFE780E0A77D15269519E5315935
:10B3D0004A851773FFFF670083D197F0FFFFE7806F
:10B3E00040A67D152695A167E353F5FE97B7FF1F8D
:10B3F000938747EB98433E8C814B01CB014597F0F7
:10B400000000E780C047933B15004A85DA865686E0
:10B41000D28597900000E78060512A8911CD1C44A5
:10B42000F99B17B7FF1F232DF7B083270C00CDD34F
:10B43000E3800BFA829769BF268597B7FF1F23AF7A
:10B4400007AE97F0FFFFE780809C4146CE8517B599
:10B45000FF1F1305E5B797300100E780605A97D0CA
:10B460000000E780E09C0325040B97D00000E780F4
:10B47000A0A0054597D00000E780A0A7054597004C
:10B480000000E78060EDA9B797B7FF1F9387C7AAB1
:10B490009C47858BEDC71773FFFFE70243C417B5C1
:10B4A000FF1F130525B197B7FF1F23A707A897B75D
:10B4B000FF1F23A507A897B7FF1F23A307A897205F
:10B4C0000100E780C08497500000E78080F9971062
:10B4D0000100E780405097100100E780405697B781
:10B4E000FF1F9387E7A39C4391C705459780000002
:10B4F000E780E02397B7FF1F9387478C9C4399C74A
:10B5000041657D1597700000E780E0A597F0000089
:10B51000E780804197D00000E780209397B7FF1F16
:10B52000938747B69C43139717016356070097F01C
:10B530000000E780A0B097B7FF1F23AB07A897B71D
:10B54000FF1F23A907A897B7FF1F23A707A897B72F
:10B55000FF1F23A507A897000000E780008C970035
:10B560000000E780A07597F0FFFFE780401897F094
:10B570000000E780E0D91773FFFF670083B882807F
:10B5800097B7FF1F9387479B8843828097B7FF1F1A
:10B590009387879AC8438280B7E7B00093870750A4
:10B5A00063E1A70297B7FF1F93870799D843FD5719
:10B5B0006367E50097B7FF1F23A2A79881473E85E1
:10B5C0008280B957EDBF1773FFFFE70243B1978041
:10B5D0000000E780607597800000E780C0771773F0
:10B5E000FFFF670003B21773FFFFE702A3AD2A84D2
:10B5F0009304140201112E85B289A685214636C610
:10B600003A8997300100E780403D0DE9B24638089D
:10B610002686CE851305940497500000E78060418C
:10B6200021462C084A8597300100E780003B1335FE
:10B63000150005611773FFFF670003AC0145D5BF17
:10B640001773FFFFE702A3A99305450617A5FF1F80
:10B650001305C56B97100100E78020691773FFFF82
:10B66000670023AA1773FFFFE70263A741112EC6E5
:10B6700097F0FFFFE780C017B24588C141011773FB
:10B68000FFFF670003A81773FFFFE702A3A3AA84C5
:10B690002E8497800000E780006CAA89854522856A
:10B6A00097000000E780E07D83C7E40113899408D8
:10B6B00099E313890403CE85228597000000E78073
:10B6C000407C214693051902228597000000E780FF
:10B6D000607897B7FF1F938727868C432285971042
:10B6E0000000E780C082214693858402228597006E
:10B6F0000000E78020761773FFFF6700E39F177352
:10B70000FFFFE702439B397197F00000E780E0B448
:10B710009305400661E997800000E78000606302BE
:10B72000051497A7FF1F83C7276013B7170097A6B5
:10B73000FF1F238BE65E014499CFC16417A9FF1F49
:10B740001309897F9309400EFD1497000000E780DC
:10B7500020836342A40A97F0FFFFE78060094169F4
:10B76000B7290900096AFD7A2A8B81447D199389DA
:10B77000F97B130A0A71938A8AC797000000E78051
:10B78000208063D7A4041304400EB387840217A754
:10B79000FF1F1307677A0324070B3E948357C401E6
:10B7A0006382270B18403307EB4063EAE9008347C5
:10B7B00044008507B3874703D6976365F7080146BA
:10B7C0008145094597F0FFFFE780C04AAA8B29E52C
:10B7D00097400000E780808385476317F5068965F9
:10B7E0009385057117A5FF1F13054552971001009A
:10B7F000E780A04F95A0B30734030327090BBA973E
:10B8000003D7C7016308970003C75700A382070047
:10B810002382E700050415BF9305C5002285970024
:10B820000000E78080E65E852286976501009385AB
:10B8300025DF97F0FFFFE780404F5E8597100000FF
:10B84000E780608A850415BF97A7FF1F9387C76E9F
:10B850009C478D83858BC1F721611773FFFF6700BC
:10B86000038901468545094502D002D202D402D699
:10B8700097F0FFFFE7800040AA8479DD97F0000091
:10B88000E780E09C1389C4002A8481454A8597009B
:10B890000000E780005F0C4041464A8597000000A9
:10B8A000E780405B832944006385090C4E8502D8FC
:10B8B00002DA02DC02DE97300100E780E0382ACEAF
:10B8C000141005462C0808184ECC97500000E7804D
:10B8D000E00A1375F50F51ED8355840093E52500BB
:10B8E0004A8597000000E780E05E11460C104A850B
:10B8F00097000000E7800056014697650100938598
:10B90000A5D2268597F0FFFFE78020422685970085
:10B910000000E780407D5C40A1D3014685450D4590
:10B9200097F0FFFFE7800035AA841DD548401389B2
:10B93000C40097300100E78020312AC64A8597006D
:10B940000000E780404C3246636FC5004C404A859A
:10B9500097000000E780005001468145268597F05A
:10B96000FFFFE780803C268597000000E780A077F6
:10B97000E5B583558400ADB71763FFFFE702237673
:10B9800097A7FF1F9387475B9C471DC193E78700DD
:10B9900017A5FF1F1305853717A7FF1F2322F75A87
:10B9A00097100100E78040321763FFFF670063755F
:10B9B000DD9B17A7FF1F2325F75897300000E7806E
:10B9C000E0647DF117A5FF1F1305453497100100B2
:10B9D000E780E033D1BF1763FFFFE702C36D416922
:10B9E000AA892E8AB28A368BBA8B814417ACFF1F84
:10B9F000130C8C54930C400E7D1997F0FFFFE780D9
:10BA0000205863C4A40001443DA0338494038327D9
:10BA10000C0B3E948357C401638627055A87D6864C
:10BA20005286CE851305040397000000E780E0BB33
:10BA300001C923800B0022851763FFFF6700236B7A
:10BA40008347F40185C35A87D6865286CE8513056F
:10BA5000940897000000E78040B909C58547238016
:10BA6000FB00D1BF850451BF835745006380071E8B
:10BA70001763FFFFE702036501112A8497000000A6
:10BA8000E780C04D09C985476309F506056117635D
:10BA9000FFFF6700636697E00000E780007C7DF5AC
:10BAA000835744004947ED9BE392E7FEC145228559
:10BAB00097000000E7804033AA84228597000000A9
:10BAC000E780204F0357440002CE91472A89631A2A
:10BAD000F700228597000000E780A0513C082ACC9F
:10BAE0003ECE97E00000E78080765C55C5D37408B1
:10BAF0004A86A6850545829751BF03574400D14722
:10BB0000E3F6E7F8032A0400C169014997AAFF1F79
:10BB1000938A8A42130B400EFD1997F0FFFFE780CE
:10BB20002046634FA90E2285032A040097000000D7
:10BB3000E780C042A1452A89228597000000E7805E
:10BB4000A02AAA84228597000000E780804A14403A
:10BB50002A86AA8978082685CA8597000000E7808A
:10BB6000C0E7AA8405D503C7F40189476315F70028
:10BB70008347C10181DF5546D28513856400973024
:10BB80000100E780E0E7014597800000E780C019E9
:10BB900001C583D7C401A5E797A7FF1F9387C739BE
:10BBA0009C4793551900858913D73700058B01CF22
:10BBB0008983858B6399B70001452EC697000000E5
:10BBC000E780C0DBB2454E8597800000E780601FAC
:10BBD0000346C1012A8493751900268597900000B9
:10BBE000E780E03935C1268597800000E780E018BE
:10BBF000268511C0014597800000E780004C9730F2
:10BC00000000E780A0408547E312F5E883C75400B1
:10BC10001307F00FE38CE7E68507A382F400BDB5B8
:10BC2000B304690383A70A0BBE9483D7C401638B53
:10BC300037015546D2851385640097300100E780AF
:10BC4000C0D955DD0509D1BD5DD86DB782801763B8
:10BC5000FFFFE702234797800000E780000C05C143
:10BC6000C164014417A9FF1F1309092D9309400E50
:10BC7000FD1497F0FFFFE780A030634EA40017A5E6
:10BC8000FF1F1305A50897100100E780E003176365
:10BC9000FFFF67006346330534038327090B3E9596
:10BCA0008357C50163889700231205009780000021
:10BCB000E780A00C050475BF97A7FF1F9387C727D0
:10BCC0009C478D83858B8DE31763FFFFE70223413C
:10BCD00017A5FF1F1305850397100100E7802003B8
:10BCE0001763FFFF6700E34182801763FFFFE702EE
:10BCF000033F970500009385C5A017A5FF1F1305F7
:10BD0000E50097100100E78020EE1763FFFF670052
:10BD1000433F1763FFFFE702833C8841B7E7040016
:10BD2000BC5B050542054181829709C58547230013
:10BD3000F50005051763FFFF6700A33C83C7F5FF08
:10BD40002E858507A38FF5FE828083C7F5FFFD173B
:10BD500093F7F70FA38FF5FE99EF1763FFFFE70245
:10BD60000338B7E70400BC571385F5FF82971763C4
:10BD7000FFFF6700033982801C41035745008D8F08
:10BD8000BA951CC12312B5003E85828093D78500E9
:10BD9000A2051441DD8D835745001387E6FF18C1C6
:10BDA00089072312F50013D685004111238FB6FEB3
:10BDB000A38FC6FE4101828018419307F7FF1CC183
:10BDC0008357450085072312F500A30FB7FE828035
:10BDD000835745008D8F2312F5001C41BE950CC181
:10BDE0002E858280AA8703D7470008410D8FAA9528
:10BDF0002392E7008CC38280184108453305A74091
:10BE0000828083574500035765001D8F1C410845FC
:10BE10003385A7403305A74082801763FFFFE70201
:10BE2000032C41112EC62A8497000000E780A0FD54
:10BE3000B2456373B50001A0835744000840BE9526
:10BE40002312B4003E9541011763FFFF6700632B87
:10BE50001763FFFFE702A32841112E84B28532C683
:10BE600097000000E780A0FB3246A28597300100D2
:10BE7000E78000B941011763FFFF6700832817635C
:10BE8000FFFFE702C3252E84854597000000E78069
:10BE900000F9230085001763FFFF670083261763FF
:10BEA000FFFFE702C32341112317B1008945970023
:10BEB0000000E780C0F68347E1002300F5008347D8
:10BEC000F100A300F50041011763FFFF6700632342
:10BED0001763FFFFE702A32093D78500A205411156
:10BEE000DD8D2317B100894597000000E78020F31E
:10BEF0008347E1002300F5008347F100A300F5002C
:10BF000041011763FFFF6700C31F1763FFFFE702CD
:10BF1000031D1397850193D78501C166938606F0AB
:10BF2000D98F13D78500758FD98FA2053707FF00EA
:10BF3000F98D4111DD8D2EC6914597000000E780F7
:10BF400000EE6C00114697300100E78060AB4101C4
:10BF50001763FFFF6700E31A1763FFFFE702231869
:10BF60001C41854503C4070097000000E78080E678
:10BF700022851763FFFF6700C3181763FFFFE702FF
:10BF800003161C414111894503C7070083C71700E9
:10BF90002307E100A307F10097000000E78080E39A
:10BFA0000355E10041011763FFFF67008315176325
:10BFB000FFFFE702C3121C414111894503C7070077
:10BFC00083C717002307E100A307F10097000000D3
:10BFD000E78040E08357E100410113D58700A207C5
:10BFE0005D8D420541811763FFFF67008311176371
:10BFF000FFFFE702C30E0C4141112A84114668007D
:10C0000097300100E780C09F91452285970000008E
:10C01000E78040DCB247C166938606F0139787013C
:10C0200013D58701598D13D78700758F598DA207B6
:10C030003707FF00F98F5D8D41011763FFFF670030
:10C04000430C1C45BE950CC18280AE87944391E69B
:10C05000584101EF0CC15CC1828003C757001367D0
:10C060001700A382E700B687D5B70CC3EDB7AA8740
:10C07000084119CD1841D44398C36313D500D8C3E0
:10C080002A87034657009376160081E6232007008F
:10C090008280944381CA8C4203A847008CC3639377
:10C0A0000601CCC3799A14C3A302C7003687D1BF57
:10C0B0001C45DC471D8DB777DBB6938777DB098599
:10C0C0003305F502420541818280F147B385F502CF
:10C0D00048452E9582808347450085072302F50059
:10C0E00082801763FFFFE70283FF2A8409E4176356
:10C0F000FFFF6700030183474400F5DBFD1793F75B
:10C10000F70F2302F400E5F71C4403D727000507C7
:10C110002391E700DC4399C3228582974C4889CD5F
:10C1200083475400898B99E71C4422859C479C4394
:10C130009C478297232A04000040232004007DB7F7
:10C140001763FFFFE702A3F98357250041112EC6AD
:10C1500081EB0144228541011763FFFF670063FA09
:10C16000035705008147F146E305F7FEB385D70283
:10C17000404585072E948345440008C4F5F5B24731
:10C18000AA8481E7232A040009A81C456C002285A3
:10C190009C439C43829748C84DDD85472312F40099
:10C1A000B24723200400231804002319F4005C483C
:10C1B0005CC483D72400FD172391F40061BF17638B
:10C1C000FFFFE702C3F197A7FF1F938727B68843B6
:10C1D0002326050023240500410597100100E78070
:10C1E00000B31763FFFF6700C3F11763FFFFE702A8
:10C1F00003EF17A4FF1F130464B31C40411199CF30
:10C200009C472300B5002AC65CC197000000E78068
:10C2100040FB1C40DC4399C33245829741011763C0
:10C22000FFFF670003EE0347450029E3584DAA8747
:10C230007D551DCF1763FFFFE70263EA1CC3DC4790
:10C2400097A6FF1F23A4E6AEF1561305070123901E
:10C25000D700970500009385050297100100E7803D
:10C26000A09801451763FFFF6700A3E97D55828011
:10C2700082801763FFFFE70283E601116146814573
:10C2800028009760FFFFE78080E897A7FF1F93874C
:10C29000E7A99C4328009305F00FDC473EC69700B2
:10C2A0000000E780C0F405611763FFFF670063E5E6
:10C2B00097A7FF1F938787A79C43D847A1679387BA
:10C2C000C702631EF70A397106DE22DC26DA800017
:10C2D0004AD84ED652D456D23285B2849700000046
:10C2E000E780C0C7AA89268597000000E78020C99B
:10C2F0002318A4FC268597000000E78040C8231976
:10C30000A4FC268597000000E78060C783D744001F
:10C310000A8A231AA4FC858393F7F70F230EF4FCF3
:10C320008607BD0793F7073F3301F1408A8A014929
:10C330008347C4FD6367F902CE85130584FC232C73
:10C3400054FD97000000E78080EA5281130104FC4D
:10C35000F2506254D2544259B259225A925A21612F
:10C360008280268597000000E78060C1931719003E
:10C37000D69705092390A7001379F90F55BF82803E
:10C3800097A7FF1F9387879A9C43D847A1679387F6
:10C39000A702631AF70A397106DE22DC26DA80006A
:10C3A0004AD84ED652D456D23285B2849700000075
:10C3B000E780C0BAAA89268597000000E78020BCE4
:10C3C000FD572318A4FC26852319F4FC97000000D0
:10C3D000E780E0BA83D744000A8A231AA4FC858345
:10C3E00093F7F70F230EF4FC8607BD0793F7073F7B
:10C3F0003301F1408A8A01498347C4FD6367F9022A
:10C40000CE85130584FC232C54FD97000000E780A3
:10C4100000DE5281130104FCF2506254D25442599E
:10C42000B259225A925A21618280268597000000D3
:10C43000E780E0B493171900D69705092390A70069
:10C440001379F90F55BF828097A7FF1F9387078E37
:10C450009C43D847A16789076310F70A397106DE44
:10C4600022DC26DA80004AD84ED652D456D2328503
:10C47000328997000000E78060AEAA894A8597005C
:10C480000000E780C0AF835749000A8A2318A4FC44
:10C49000858393F7F70F230CF4FC8607BD0793F70A
:10C4A000073F3301F1408A8A8144834784FD63E773
:10C4B000F402CE85130584FC232A54FD9700000066
:10C4C000E780E0D25281130104FCF2506254D2544E
:10C4D0004259B259225A925A216182804A85970064
:10C4E0000000E780C0A993971400D6978504239095
:10C4F000A70093F4F40F55BF828097A7FF1F93877F
:10C50000E7829C43D847A1679387E704631EF70A35
:10C51000397106DE22DC26DA80004AD84ED652D4A3
:10C5200056D23285B28497000000E78020A3AA8902
:10C53000268597000000E78080A42318A4FC2685A8
:10C5400097000000E780A0A3231AA4FC268597008B
:10C550000000E780C0A283D744000A8A2319A4FC04
:10C56000858393F7F70F230EF4FC8607BD0793F737
:10C57000073F3301F1408A8A01498347C4FD63675D
:10C58000F902CE85130584FC232C54FD970000008E
:10C59000E780E0C55281130104FCF2506254D2548A
:10C5A0004259B259225A925A2161828026859700B7
:10C5B0000000E780C09C93171900D69705092390C7
:10C5C000A7001379F90F55BF82809797FF1F9387B4
:10C5D000E7759C43D847A1679387C704631AF70A96
:10C5E000397106DE22DC26DA80004AD84ED652D4D3
:10C5F00056D23285B28497000000E7802096AA893F
:10C60000268597000000E7808097FD572318A4FC3B
:10C610002685231AF4FC97000000E780409683D714
:10C6200044000A8A2319A4FC858393F7F70F230E8D
:10C63000F4FC8607BD0793F7073F3301F1408A8A70
:10C6400001498347C4FD6367F902CE85130584FC65
:10C65000232C54FD97000000E78060B9528113013C
:10C6600004FCF2506254D2544259B259225A925A9E
:10C6700021618280268597000000E7804090931713
:10C680001900D69705092390A7001379F90F55BF14
:10C6900082809797FF1F938767699C43D847A1675C
:10C6A000DD076317F7041763FFFFE70243A3797100
:10C6B0003285328497000000E780408A2AC62285AE
:10C6C00097000000E780A08B2311A102228597002C
:10C6D0000000E780A088B2452300A1022808970047
:10C6E0000000E780C0B045611763FFFF670063A1EA
:10C6F00082809797FF1F938767639C43D847A16702
:10C70000938787046317F7041763FFFFE702239DEE
:10C7100079713285328497000000E78020842AC630
:10C72000228597000000E78080852311A1022285E1
:10C7300097000000E7808082B2452300A10228080C
:10C7400097000000E780A0AA45611763FFFF67001C
:10C75000439B82809797FF1F9387475D9C43D847F1
:10C76000A1679387A7046312F7021763FFFFE7022D
:10C77000039701112800814597000000E78020A75A
:10C7800005611763FFFF6700C39782809797FF1FBC
:10C790009387C7599C43D847A1679387570263196A
:10C7A000F7021763FFFFE70283930111328597F0C9
:10C7B000FFFFE780A07A2308A100814528009700A9
:10C7C0000000E780C0A205611763FFFF6700639365
:10C7D00082809797FF1F938767559C43D847A1672F
:10C7E0009387E702631BF7041763FFFFE702238FBA
:10C7F00001113285328497F0FFFFE7804078AA84E8
:10C80000228597F0FFFFE7808077854709E9228539
:10C8100097F0FFFFE78080744205B337A00028003F
:10C820008145231891003ECA97000000E780209CB4
:10C8300005611763FFFF6700C38C82809797FF1F16
:10C840009387C74E9C43D84799476313F7081763EC
:10C85000FFFFE702C38879713285328497F0FFFFCA
:10C86000E780C06F2AC6228597F0FFFFE78020711E
:10C870002310A102228597F0FFFFE780206E23019D
:10C88000A102228597F0FFFFE780406DA301A1027E
:10C89000228597F0FFFFE780606C2302A1022285CA
:10C8A00097F0FFFFE780806B2313A102228597F0AA
:10C8B000FFFFE780A06AB2452314A1022808970071
:10C8C0000000E780C09245611763FFFF6700638344
:10C8D00082809797FF1F938767459C43D847A1673E
:10C8E0009387C7036313F7081753FFFFE702237FFC
:10C8F00079713285328497F0FFFFE78020662AC67F
:10C90000228597F0FFFFE78080672310A102228530
:10C9100097F0FFFFE780A0662311A102228597F020
:10C92000FFFFE780A0632302A102228597F0FFFFAB
:10C93000E780C062A302A102228597F0FFFFE78093
:10C94000E0612303A102228597F0FFFFE7800061E9
:10C95000B245A303A102280897000000E7802089C0
:10C9600045611753FFFF6700C37982801753FFFFAC
:10C97000E702E37601112A8497F0FFFFE780005E6B
:10C98000AA84228597F0FFFFE780605F228597F0F9
:10C99000FFFFE780C05E035744008D4763F7E70061
:10C9A000228597F0FFFFE780805D228597F0FFFFEB
:10C9B000E780E05C2800A68597000000E7802083E0
:10C9C00005611753FFFF6700C3739797FF1F938796
:10C9D000E7359C43D847A167FD07631FF70017534E
:10C9E000FFFFE702C36F328597000000E78040F841
:10C9F0001753FFFF6700E37082809797FF1F9387AD
:10CA0000E7329C43D847A167E5076315F70817533A
:10CA1000FFFFE702C36C79713285328497F0FFFF24
:10CA2000E780C0532AC6228597F0FFFFE780205594
:10CA3000228597F0FFFFE78080542310A102228512
:10CA400097F0FFFFE780A053520551812311A10207
:10CA500022852302010297F0FFFFE7802050A30206
:10CA6000A102228597F0FFFFE780404F2303A10238
:10CA7000228597F0FFFFE780604EB245A303A10235
:10CA8000280897F0FFFFE780807645611753FFFF86
:10CA90006700236782809797FF1F938727299C430E
:10CAA000D847A1679387E703631FF7001753FFFF7A
:10CAB000E702E362328597000000E78060EB1753DE
:10CAC000FFFF6700036482809797FF1F9387072605
:10CAD0009C43D847A16793874704631EF702175307
:10CAE000FFFFE702C35F79713285328497F0FFFF61
:10CAF000E780C0462AC6228597F0FFFFE7802048DE
:10CB0000B245280897F0FFFFE780606E4561175334
:10CB1000FFFF6700035F82809797FF1F93870721BE
:10CB20009C43D847A167938787026310F704175384
:10CB3000FFFFE702C35A79713285328497F0FFFF15
:10CB4000E780C0412AC6228597F0FFFFE7800041B9
:10CB5000B2452300A102280897F0FFFFE780206973
:10CB600045611753FFFF6700C35982801753FFFFCA
:10CB7000E702E356011197F0FFFFE780203EAA8508
:10CB8000280097F0FFFFE780806605611753FFFFDD
:10CB9000670023579797FF1F938747199C43D847F0
:10CBA000A167D107631FF7001753FFFFE702235365
:10CBB000328597000000E780A0FB1753FFFF670056
:10CBC000435482809797FF1F938747169C43D8470B
:10CBD000A167C507631FF7001753FFFFE702235044
:10CBE000328597000000E780A0F81753FFFF670029
:10CBF000435182809797FF1F938747139C43D847E1
:10CC0000A167B907631FF7001753FFFFE702234D22
:10CC1000328597000000E780A0F51753FFFF6700FB
:10CC2000434E82809797FF1F938747109C43D847B6
:10CC3000A167AD07631FF7001753FFFFE702234A01
:10CC4000328597000000E780A0F21753FFFF6700CE
:10CC5000434B82809797FF1F9387470D9C43D8478C
:10CC600089476318F7021753FFFFE7024347011193
:10CC7000328532C897F0FFFFE780402EAA85280052
:10CC800097F0FFFFE780A05605611753FFFF67008D
:10CC9000434782809797FF1F938747099C43D84754
:10CCA000A1678D076311F7041753FFFFE7022343C2
:10CCB00001113285328497F0FFFFE780202A1306A6
:10CCC0006100AA844C00228597300000E780C023D1
:10CCD0002800A68597F0FFFFE78060510561175394
:10CCE000FFFF6700034282809797FF1F93874704E7
:10CCF0009C4381CFDC4391CB1753FFFFE702233ED8
:10CD000082971753FFFF6700C33F82801753FFFFCF
:10CD1000E702E33C79713C08AE843ED2A165B707D7
:10CD20000A002A843ED448103C08DD053ED636C4AD
:10CD300032C63AC297D0FFFFE780402C1247481016
:10CD4000BA8597F0FFFFE780C01332464810B285DE
:10CD500097F0FFFFE780E014A2464810B68597F0F1
:10CD6000FFFFE7800012501001478146A68522850B
:10CD700097D0FFFFE780E04D45611753FFFF670045
:10CD800043381753FFFFE702833501117C00032965
:10CD9000C501AE843ECAA165B70707002A843ECC10
:10CDA00048087C00C5053ECE97D0FFFFE7800025F0
:10CDB0008345D900480897F0FFFFE780800C5008B2
:10CDC00001478146A685228597D0FFFFE78060480E
:10CDD00005611753FFFF6700C3321753FFFFE702D8
:10CDE000033083C7950093F7F707A384F5009700F6
:10CDF0000000E78040F91753FFFF670083301753A7
:10CE0000FFFFE702C32D79713C08AE843ED2A165D5
:10CE1000B70709002A843ED448103C08938545048E
:10CE20003ED632C636C497D0FFFFE780201DA2460B
:10CE30004810B68597F0FFFFE780A00432464810FF
:10CE4000B28597F0FFFFE780C0055010014781468B
:10CE5000A685228597D0FFFFE780A03F4561175345
:10CE6000FFFF6700032A1753FFFFE702432783C72B
:10CE7000950041112A8493F7F707A384F5003285C2
:10CE80002EC697F0FFFFE780800F85672AC4637086
:10CE9000F50297700000E78020E92246B24509EDCF
:10CEA00011478146228597000000E78060E6410136
:10CEB0001753FFFF6700E32401478346F501DDB701
:10CEC0001753FFFFE702032001113C003ECAB707DA
:10CED0000A003ECC3C003ECE83C79500AA8932852D
:10CEE00093F7F707A384F5002E8497F0FFFFE78000
:10CEF00000098567637DF504A165AA84938585048F
:10CF0000480897D0FFFFE780600F268597700000E4
:10CF1000E78080E12A8929E19145480897F0FFFFE1
:10CF2000E78020F6A685480897F0FFFFE78060F7C6
:10CF3000CA85480897F0FFFFE780A0F401478146C3
:10CF40005008A2854E8597D0FFFFE78080300561AD
:10CF50001753FFFF6700431A8145480897F0FFFF0A
:10CF6000E78020F20349090275BF1753FFFFE7026C
:10CF7000631579711C103ECAB7070F003ECC404DB7
:10CF80001C10AA84AE894808994532C636893ECE1F
:10CF900097D0FFFFE780800632464808B28597F0B9
:10CFA000FFFFE78000EE630C0902A545480897F0F3
:10CFB000FFFFE780C0E62546CA8597200100E7808D
:10CFC00020A4500801478146CE85268597D0FFFFD3
:10CFD000E780202845611753FFFF6700E311835561
:10CFE000C402480897F0FFFFE780A0EB0355E40276
:10CFF000814505C5854785456301F502C167FD1774
:10D000009305F00F630BF5007D1597700000E78026
:10D01000208E9305150093F5F50F480897F0FFFF54
:10D02000E78020E683450403480897F0FFFFE78088
:10D0300040E583451403480897F0FFFFE78060E46C
:10D0400083552403480897F0FFFFE78080E5835568
:10D050004403480897F0FFFFE780A0E49DB717530B
:10D06000FFFFE702C30783C795008146014693F798
:10D07000F707A384F50097000000E78040EF1753FF
:10D08000FFFF670003081753FFFFE70243057971AD
:10D090003E841C103ECA2E89B7070F00A1653ECC06
:10D0A000FD051C10AA84480842C03AC23ECE36C4D0
:10D0B00032C697D0FFFFE78060F432464808B28559
:10D0C00097F0FFFFE780E0DBA2464808B68597F0BF
:10D0D000FFFFE78000DD12474808BA8597F0FFFFA1
:10D0E000E78020DC0248630C08029145480897F06D
:10D0F000FFFFE780C0D21146A28597200100E7809C
:10D100002090500801478146CA85268597D0FFFFA9
:10D11000E780201445611753FFFF670083FE8945B0
:10D12000480897F0FFFFE78080CF83470400230083
:10D13000F50083471400A300F500E1B71753FFFF84
:10D14000E70243F883C7950001112A8A93F7F7078E
:10D15000A384F5003285AE8432C697F0FFFFE780E6
:10D1600000E232462A89328597F0FFFFE78000DF30
:10D1700085676373F902AA894A8597700000E78082
:10D18000A0BA2A8419ED114781464A86A6855285A0
:10D1900097000000E780C0B705611753FFFF6700E5
:10D1A000A3F59387E9FF93F7F70F0547E366F7FECB
:10D1B0008347F50195EB8947E380F9FE8346F40147
:10D1C000528501474A86A68597000000E78040B453
:10D1D000A167D90748083ECC230A010002CE970078
:10D1E0000000E780A0B04DBF639EE7008947639EC3
:10D1F000F90093071020231FF50097700000E780C7
:10D20000C0B76DBF0947E39BE7FA8D47E398F9FA8A
:10D21000228597700000E78080DF9797FF1F938734
:10D2200027D09C4399E79797FF1F938727B99C4383
:10D2300099C703D5040097800000E780A0CE231F84
:10D24000040022855DBF1753FFFFE70243E9011188
:10D250003C003ECAB7070B003ECC3C003ECE83C725
:10D2600095002A89328593F7F707A384F500AE84E9
:10D2700097F0FFFFE780A0D093170501C187635A9D
:10D28000F006A1652A849385E502480897D0FFFF40
:10D29000E780C0D6A285480897F0FFFFE78060C00E
:10D2A0009797FF1F938787B19C43A9EB0144937520
:10D2B000F40F480897F0FFFFE780A0BC9355844027
:10D2C00093F5F50F480897F0FFFFE78080BB935573
:10D2D000044193F5F50F480897F0FFFFE78060BA27
:10D2E000014781465008A6854A8597D0FFFFE78011
:10D2F00040F605611753FFFF6700A3E041658546CF
:10D300000546A2857D1597500000E78060BD59DD78
:10D31000510597000100E780808F130440063344D5
:10D32000850271B71753FFFFE70263DB0111B707EF
:10D3300006003EC683C7950021642A8993F7F70744
:10D34000A384F500AE8428009305A4040AC40AC887
:10D3500097D0FFFFE78080CA300001478146A6854D
:10D360004A8597D0FFFFE780C0EE97E0FFFFE78098
:10D37000E01113049404480822CC230A010002CED1
:10D3800097000000E780809605611753FFFF670054
:10D3900043D71753FFFFE702E3D2C1642A89014450
:10D3A0009799FF1F938949B9130A8002FD1497E0EA
:10D3B000FFFFE780E0BD6347A40001451753FFFF6F
:10D3C000670083D3B307440303A7C90ABA9703D7F7
:10D3D00007006306970083D72700638427010504AD
:10D3E000F9B70545E1BF1753FFFFE702A3CD2A8A2E
:10D3F0002E8999C123A0050081498144979AFF1F76
:10D40000938A4A93614B97E0FFFFE780A0BE63C712
:10D41000A4004E851753FFFF670003CE33846403D7
:10D4200083A70A003E948357040099E76304090028
:10D43000232089008504C1BF4146D28513054400DD
:10D4400097100100E780605975F5A289E5B7175379
:10D45000FFFFE70223C739717C083ED4B7070A00F3
:10D460003ED67C083ED883C795002A8A328593F73A
:10D47000F707A384F5002E8932C697F0FFFFE780F7
:10D4800000B085676373F5083246AA84328597F049
:10D49000FFFFE780A0AC8547AA8963E8A706A165DE
:10D4A00093858504281097D0FFFFE78020B5268557
:10D4B00097700000E78040872A8429ED9145281065
:10D4C00097F0FFFFE780E09BA685281097F0FFFF0D
:10D4D000E780209DCE85281097F0FFFFE780609AB7
:10D4E000014781463010CA85528597D0FFFFE780FB
:10D4F00040D6A1679387770448183EDC230A0102CF
:10D5000002DE97F0FFFFE780607E21611753FFFF87
:10D51000670083BE8145281097F0FFFFE780609683
:10D52000A685281097F0FFFFE780A0979797FF1F29
:10D53000938707D79C4381CB22856389090097D0C5
:10D540000000E78040248345040271B797D00000B3
:10D55000E780C022CDBF1753FFFFE702A3B683C702
:10D5600095004111AA8993F7F707A384F500328546
:10D57000AE84328A97F0FFFFE78060A08567637F03
:10D58000F5022A8997600000E780007A2A84914694
:10D5900031C58347F50105476387E70291C70D470A
:10D5A0006366F704AD461DA89305050303250A002D
:10D5B000414697100100E78040420DE941011753B1
:10D5C000FFFF670063B39305950803250A004146F2
:10D5D00097100100E7806040814669F54A86A6857C
:10D5E0004E8597000000E780C081C9BF83250A00EF
:10D5F0001305940897700000E780A02919C1C1465F
:10D60000F1BF9797FF1F9387A7919C4399E797874F
:10D61000FF1F9387A77A9C4399C7228597800000B4
:10D62000E780208A69FD8547A30FF400228597B023
:10D630000000E7806084228597600000E780E07347
:10D640004E8581464A86A68597F0FFFFE780607B7E
:10D65000A1679387570448003EC42302010002C615
:10D6600097F0FFFFE780806891BF1753FFFFE70245
:10D6700083A483C795004111AA8993F7F707A38470
:10D68000F50032852E89B28A97F0FFFFE780208F60
:10D6900085676374F50EAA8497600000E780C06810
:10D6A0002A840DED416B014A979BFF1F938BCB881A
:10D6B000130C400E7D1B19A833048A0383A70B0BA0
:10D6C0003E948357C40163836705050A97E0FFFF13
:10D6D000E780008BE342AAFE95460DA08357C50163
:10D6E000639697029305050303A50A004146971028
:10D6F0000100E780802E994611E181462686CA8581
:10D700004E8597F0FFFFE780C06F85A883A50A00CC
:10D710001305040397700000E780A017C14679FD48
:10D720002285231E940097A00000E780E0742285E4
:10D7300097600000E78060649797FF1F938747B664
:10D740009C43A9C323000402228597D00000E780F0
:10D7500040F04E8581462686CA8597F0FFFFE78018
:10D76000406AA1679387070448003EC42302010072
:10D7700002C697F0FFFFE780605741011753FFFF94
:10D780006700E39689472300F402E1B7397106DEAA
:10D7900022DC4AD8800052D456D25AD026DA4ED64D
:10D7A0005ECE2E8A32892A8B97D0FFFFE780407A9F
:10D7B0000605710541998A8A3301A140232224FC80
:10D7C000231404FC97D0FFFFE780807883479A00FA
:10D7D0000605350593F7F7072315A4FCA304FA0003
:10D7E0004A85232624FC97E0FFFFE78040799317C2
:10D7F0000501C1876340F0025681130104FCF25019
:10D800006254D2544259B259225A925A025BF24B94
:10D8100021618280AA844A8597E0FFFFE780207615
:10D82000AA894A8597E0FFFFE7806075A165938527
:10D83000C5022A89130544FC97C0FFFFE780007CDE
:10D84000268597C0FFFFE7804070854511C94A864D
:10D85000CE8597C0FFFFE780C069AA8B21E9894583
:10D86000130544FC97E0FFFFE780A061A685130540
:10D8700044FC97E0FFFFE780C062CE85130544FCBF
:10D8800097E0FFFFE780E061CA85130544FC97E05D
:10D89000FFFFE780006101478146130644FCD28503
:10D8A0005A8597D0FFFFE780C09AB9B78145130525
:10D8B00044FC97E0FFFFE780C05CA685130544FCAD
:10D8C00097E0FFFFE780E05DCE85130544FC97E01D
:10D8D000FFFFE780005DCA85130544FC97E0FFFF6A
:10D8E000E780205C814497D0FFFFE7806066E3D447
:10D8F000A4FA83A70B0113971400BA9783D50700E6
:10D9000099C5130544FC97E0FFFFE7808059850423
:10D91000D9BF797106D622D44AD000184ECE52CC47
:10D9200056CA26D25AC8AE893289AA8A97D0FFFF32
:10D93000E78000620605690541990A8A3301A14022
:10D94000232A24FC231C04FC97D0FFFFE7804060BF
:10D9500083C7990006052D0593F7F707231DA4FC3F
:10D96000A384F9004A85232E24FC97E0FFFFE7807B
:10D97000006193170501C187634FF00052811301C5
:10D9800004FDB250225492540259F249624AD24ADA
:10D99000424B45618280AA844A8597E0FFFFE78079
:10D9A000005EA1659385A5022A89130544FD97C0F1
:10D9B000FFFFE780A064268597C0FFFFE780E0585F
:10D9C000854509C9CA8597C0FFFFE78080552A8B26
:10D9D00029E18945130544FD97E0FFFFE780604A90
:10D9E000A685130544FD97E0FFFFE780804BCA85BD
:10D9F000130544FD97E0FFFFE780A04A01478146F9
:10DA0000130644FDCE85568597D0FFFFE7806084DE
:10DA1000B5B78145130544FD97E0FFFFE7806046F9
:10DA2000A685130544FD97E0FFFFE7808047CA8580
:10DA3000130544FD97E0FFFFE780A046814497D09F
:10DA4000FFFFE780E050E3DBA4FA83270B01139785
:10DA50001400BA9783D5070099C5130544FD97E0D4
:10DA6000FFFFE78000448504D9BF1743FFFFE702AB
:10DA7000036783474500404DD5EFFD575DC483469E
:10DA8000940009476363D70A0346B400854663EEF2
:10DA9000C6088306E40063CA06085C45F95623906D
:10DAA000D7009787FF1F83C7272999E3A304E400C2
:10DAB0009787FF1F938787309C4381E78947A30699
:10DAC000F4009787FF1F9387A77D9C4381E78947D1
:10DAD0002306F4009705000093854506AA841305E4
:10DAE000040197F00000E7802010FD57231AF4028C
:10DAF00081471CDC01489787FF1F23AB872297874C
:10DB0000FF1F93872723232E040304C0804397D04D
:10DB1000FFFFE780204E61463306C502814522851E
:10DB20009740FFFFE780A05E81473E851743FFFFD8
:10DB30006700235DFD57D5BF1743FFFFE702235A58
:10DB40002A840355450297600000E780E01D19E52F
:10DB5000231E04001743FFFF6700A35A8357E40105
:10DB6000F5DB930504FF174501001305A5E597E0D4
:10DB70000000E780E014F9BF1743FFFFE7022356D8
:10DB80002E89A16541119385E5032A8436C432C6E6
:10DB9000BE843AC297C0FFFFE78040461247228505
:10DBA000BA8597E0FFFFE780C02D32462285B28517
:10DBB00097E0FFFFE780E02EA2462285B68597E03A
:10DBC000FFFFE780002E630309029145228597E05D
:10DBD000FFFFE780C0241146A68597100100E7806B
:10DBE00020E241011743FFFF6700A35189452285C9
:10DBF00097E0FFFFE780A02283C704002300F50021
:10DC000083C71400A300F500E9BF1743FFFFE70235
:10DC1000034D83C79500444D054793F7F707A38449
:10DC2000F5001C42411183C707006367F7062E8485
:10DC30002A89B1C003C7D400630FF7021787FF1FFB
:10DC40001307C717184305C3A386F40097A0000065
:10DC5000E780404A83C7D40099E741657D15974026
:10DC60000000E780403083D72403918B89C797E079
:10DC70000000E780C0134A85A28597F0FFFFE78088
:10DC80008010A167C10748003EC42302010002C6FC
:10DC900097F0FFFFE780800541011743FFFF670012
:10DCA00043461743FFFFE702834303D745008D47F1
:10DCB000AA8441112E8432892E8563E3E70297E01E
:10DCC000FFFFE780C02BAA8523000900268597C0A7
:10DCD000FFFFE780002541011743FFFF6700634214
:10DCE00097E0FFFFE780A0292AC6228597E0FFFF83
:10DCF000E780E028B24585472A862300F90026857B
:10DD000097C0FFFFE780E01EF9B7397106DE22DC1D
:10DD100026DA80004ED652D456D24AD85AD05ECE99
:10DD2000AE89B284AA8A97D0FFFFE78060210605FA
:10DD30001305250241990A8A3301A140232224FCBC
:10DD4000231404FC97D0FFFFE780801F83C799004E
:10DD500006054D0593F7F7072315A4FCA384F900E6
:10DD60002685232624FC97E0FFFFE78040219317B8
:10DD70000501C1876340F0025281130104FCF25097
:10DD80006254D2544259B259225A925A025BF24B0F
:10DD900021618280AA8B03AB040097C0FFFFE7805C
:10DDA000C01A51E583D7440001498544F11793B760
:10DDB0001700A301F4FC834734FCA165C9C7938510
:10DDC000E504130544FC97C0FFFFE7802023A685E8
:10DDD000130544FC97E0FFFFE780A00ADE851305EA
:10DDE00044FC97E0FFFFE780C00B834734FC1146FB
:10DDF00091E30946DA85130544FC97E0FFFFE780CD
:10DE000060058144630A0900416B7D1B97D0FFFFC9
:10DE1000E780001363CCA40201478146130644FC4B
:10DE2000CE85568597C0FFFFE780A042B1B7A68593
:10DE3000130634FC97000000E780E0E693341500F9
:10DE40002A8986048DBF9385C504A5BF8327C90091
:10DE500013971400BA9783D50700638865011305EB
:10DE600044FC97E0FFFFE780C003850445B71743F4
:10DE7000FFFFE702432479711C103EC4B7070F006F
:10DE80003EC61C103EC883C79500AA8A328593F708
:10DE9000F707A384F500AE89328497E0FFFFE7809F
:10DEA000000E93170501C187635AF0062A8A22855E
:10DEB00097E0FFFFE780A00C2A895285032B04001E
:10DEC00097C0FFFFE780600839ED83574400814425
:10DED0000544F11793B71700A303F10083457100C0
:10DEE000DA872287CA865286280097000000E780DA
:10DEF000E0C8014781463000CE85568597C0FFFFB8
:10DF0000E7802035A1679387D70348083ECC230AD2
:10DF1000810026CE97F0FFFFE78040DD4561174383
:10DF2000FFFF6700C31CA285130671009700000065
:10DF3000E78060D7AA84094455D13544E30055FBF6
:10DF40004A8597F0FFFFE78000450D4441D9014421
:10DF500097D0FFFFE780C0FE634DA400C16B014472
:10DF6000FD1B97D0FFFFE780A0FD634EA400154482
:10DF7000B5B7DC4413171400BA9783D7070063833F
:10DF800027030504F1B7D84493171400BA9703D7B1
:10DF90000700631B770123902701268597A00000C7
:10DFA000E78080DB01441DBF050465BF1743FFFF09
:10DFB000E702431183C7950041112A8A93F7F707B7
:10DFC000A384F50032852E89328497E0FFFFE78035
:10DFD00000FB93170501C1876353F006AA892285C8
:10DFE00097E0FFFFE780A0F92311A1004E85832A67
:10DFF000040097C0FFFFE78040F539E583574400F0
:10E0000085440144F11793B71700A300F1000348BA
:10E01000110003572100D6875285CE862686CA85F1
:10E0200097F0FFFFE7806006A167F10748003EC454
:10E030002302910022C697F0FFFFE78020CB410129
:10E040001743FFFF6700430BA285130611009700DB
:10E050000000E78040C52A84894455D983572100B0
:10E0600011678544BA97C2071167C1831307F7EF99
:10E07000E36FF7F89787FF1F938787EA9C4381CB6D
:10E0800085451305210097500000E78020758355D2
:10E0900021002285814497C0FFFFE780A0E125D9B8
:10E0A00023100500228597A00000E78040CD85B7AA
:10E0B0001743FFFFE702230083C7950041112A8B16
:10E0C00093F7F707A384F50032852E8A328497E010
:10E0D000FFFFE780C0EA93170501C1876351F0068F
:10E0E000AA8A228597E0FFFFE78060E92A895685A2
:10E0F000832B040097C0FFFFE78020E531E58357BD
:10E10000440081440544F11793B71700A301F100BF
:10E1100003483100DE875A854A87D6862286D28513
:10E1200097F0FFFFE78060F6A167ED0748003EC467
:10E130002302810026C697F0FFFFE78020BB410144
:10E140001743FFFF6700A3FAA2851306310097006B
:10E150000000E78040B5AA8409445DD99167CA9759
:10E16000C2071167C1831307F7EF0544E362F7FAAB
:10E17000CA8597C0FFFFE780E0D3014451F9814988
:10E1800097D0FFFFE780C0DC63DBA9009848939736
:10E190001900BA9703D7070005EF2390270197D0FE
:10E1A000FFFFE780E0DA1544E384A9F6268597A00F
:10E1B0000000E780C0BC9787FF1F938767D69C430A
:10E1C0000144B9D74A8597500000E780C05889B705
:10E1D00085097DB71743FFFFE702C3EE79713E84DF
:10E1E0007C083EC82E8AB7071400A1653ECAE50523
:10E1F0007C08AA89080836C4428932C6BA8AC6840D
:10E200003ECC97C0FFFFE78060DFCA85080897E033
:10E21000FFFFE78000C732460808B28597E0FFFF9E
:10E22000E78020C8A246630A09049D45080897E0D4
:10E23000FFFFE780C0BE1D4681459740FFFFE78096
:10E2400000ED63890A089145080897E0FFFFE78021
:10E2500000BD1146A68597000100E780607A10088E
:10E2600001478146D2854E8597C0FFFFE78060FE5B
:10E2700045611743FFFF670023E8B685080897E06C
:10E28000FFFFE78000C21C400808D8439355C70130
:10E29000858912075183B205D98D97E0FFFFE7808A
:10E2A00040C01C40080883C5870097E0FFFFE78057
:10E2B00040BD1C40080883C5A70097E0FFFFE7802A
:10E2C00040BC1C40080883C5970097E0FFFFE7802B
:10E2D00040BB85BF8945080897E0FFFFE78020B471
:10E2E00083C704002300F50083C71400A300F500D2
:10E2F000BDB71743FFFFE702E3DC83C79500411179
:10E30000AA8993F7F707A384F5003285AE84328497
:10E3100097E0FFFFE780A0C693170501C187635D03
:10E32000F0042A89032A040097C0FFFFE780E0C1B8
:10E3300019E9835744000548F11793B71700A3075D
:10E34000F100814631A81306F100A2859700000074
:10E35000E78060951DC51C459DC783D647000148D1
:10E360000347F10093078500D2884A86A6854E852B
:10E3700097000000E78040E641011743FFFF670078
:10E38000A3D709487DBF1D486DBF1743FFFFE702B4
:10E3900063D365715C083EC4B7077B013EC65C0869
:10E3A0003EC883C795002A8A328593F7F707A3846E
:10E3B000F500AE8997E0FFFFE78040BA8357E100A0
:10E3C000E1C78945280097C0FFFFE78020C381454A
:10E3D000280097E0FFFFE780C0AA97C0FFFFE78013
:10E3E00000C99787FF1F9387A7EB9C431784FF1FE4
:10E3F00003448494AA843334800099C313642400B2
:10E400009787FF1F9387879B9C4399C3136444009E
:10E410009787FF1F9387C7B09C4399C313648400F9
:10E4200083D504002800014997E0FFFFE78060A73B
:10E4300083D52400280097E0FFFFE78080A683D5DE
:10E440004400280097E0FFFFE780A0A597D0FFFFDA
:10E45000E78000AB93150501C181280097E0FFFF1D
:10E46000E78020A4A285280097E0FFFFE78060A353
:10E470009C446360F902014781463000CE85528595
:10E4800097C0FFFFE780E0DC59611743FFFF67009B
:10E49000A3C6DC441314490028003E9497E0FFFF14
:10E4A000E7806096834744000347540089070607C6
:10E4B000BA978607E36AF5FC835524002800814A51
:10E4C00097E0FFFFE780E09D83454400280097E048
:10E4D000FFFFE780009B83455400280097E0FFFF83
:10E4E000E780209A8347440063C9FA00814A834742
:10E4F000540063C1FA020509A5BF1C4413975A00D2
:10E500002800BA9783D50700850A97E0FFFFE780C8
:10E510004099C9BF032BC40093975A0028003E9B23
:10E5200083552B00850A97E0FFFFE780809783558E
:10E530000B00280097E0FFFFE780A0964DBF174330
:10E54000FFFFE702C3B95C4993E717005CC997A0D6
:10E550000000E78020B61743FFFF670083BA174328
:10E56000FFFFE702C3B72E84814597F0FFFFE780E6
:10E57000C0E705C583570500FD172310F50009C442
:10E58000835725002310F40097000000E78060FB0C
:10E5900001451743FFFF6700C3B631457DD82310FF
:10E5A0000400C5BF1743FFFFE702C3B183C795004F
:10E5B00041112A8A93F7F707A384F50032852E8943
:10E5C000328497E0FFFFE780809B93170501C187A6
:10E5D0006356F006AA89C145228597E0FFFFE780D0
:10E5E000A0802A8B4E85832A040097C0FFFFE78016
:10E5F000C09531E983574400231101000544F11708
:10E6000093B71700A300F10081440348110003579A
:10E610002100D6875285CE862286CA8597F0FFFFD5
:10E62000E780A0A6A1679387170248003EC4230293
:10E63000810026C697E0FFFFE780406B410117434A
:10E64000FFFF670063AB13061100A28597F0FFFF81
:10E65000E7806065AA8409E523110100094475B7C4
:10E66000930521005A8597000000E78080EF8357CB
:10E6700021002A84D9DB9787FF1F9387678A9C43F1
:10E6800081CB85451305210097500000E7800015D8
:10E69000835521002685314497C0FFFFE7808081A4
:10E6A0002DD523100500268597900000E780206D6A
:10E6B0000144A1BF1743FFFFE70263A241112E8966
:10E6C0006C00AA8402C697F0FFFFE78000D20DC15C
:10E6D0000357050005072310E50097000000E780B9
:10E6E00040E681473E8541011743FFFF670063A174
:10E6F0003247954765DBCA85268597300000E7805D
:10E70000400DC147E34005FE324485474146231092
:10E71000F40083570900A685130544002311F40073
:10E7200097000100E780C02D228545BF1743FFFFFA
:10E73000E702439983C795004111AA8A93F7F70727
:10E74000A384F5003285AE89328497E0FFFFE7802D
:10E75000008393170501C1876356F0062A8AC145D5
:10E76000228597D0FFFFE7802068AA845285032B7B
:10E77000040097B0FFFFE780407D31E983574400F4
:10E78000231101008544F11793B71700A300F1008E
:10E7900001440348110003572100DA875685D286C9
:10E7A0002686CE8597F0FFFFE780208EA1679387AE
:10E7B000070248003EC42302910022C697E0FFFFF3
:10E7C000E780C05241011743FFFF6700E392A28533
:10E7D0001306110097F0FFFFE780E04C2A8409E55B
:10E7E00023110100894475B7268593052100970000
:10E7F0000000E78060ECAA8449FD83552100228552
:10E8000097B0FFFFE780006B49F5014997C0FFFF14
:10E81000E7800074635DA900184893171900BA9740
:10E8200003D707000DEF035721002390E70097C09F
:10E83000FFFFE780E071630625039777FF1F93874B
:10E84000276E9C4399C70355210097500000E7802D
:10E8500080F0228597900000E78060521DBF050977
:10E8600075B795443DB705C19307F00F630FF500E9
:10E87000C547630CF5009307F5FF05453315F50013
:10E880004205418182800145828041657D158280FB
:10E89000B9E91743FFFFE702838403450603328487
:10E8A00097000000E78060FC9305803EB305B50249
:10E8B000C205C18181CD0357E402854763F8E700B3
:10E8C0001305040197E00000E78020428357E4022B
:10E8D00041677D176385E700FD172317F40217438F
:10E8E000FFFF6700038282801733FFFFE702A37CEC
:10E8F000004283C79500444D0349140093F7F7077E
:10E90000A384F50083470400220911673369F900E5
:10E91000A167B347F90041112A8BAE8A63ECE70E79
:10E92000834724001307C00EB91793F7F70F6373DB
:10E93000F71003473400C14763EEE70E83474400F6
:10E940001307E00793C707086371F70C8349840036
:10E9500083477400A209B3E9F900856763F7F90AF0
:10E96000034A6400834754004E85220A336AFA0042
:10E9700097500000E780403B61C123962403834BFE
:10E980003400137AFA00239A3403238874032399FA
:10E99000440393890401631C090023A604022398FD
:10E9A00004024E8597E00000E78060363DA00349F1
:10E9B00024004A8597000000E78020EB2397A402FB
:10E9C000834744004E85A388F402E38D0BFCE30BE0
:10E9D00009FC97E00000E780202F97900000E78077
:10E9E000007381460146D6855A8597E0FFFFE78090
:10E9F0000058A167938797033EC423020100480093
:10EA000002C697E0FFFFE780602E41011733FFFF4A
:10EA10006700E36D8544A2862686D6855A8597E0F1
:10EA2000FFFFE780C054A167938797033EC423028A
:10EA30009100F1B7BD44C5B79144F1BF1733FFFF53
:10EA4000E702436801111C08404D3EC2B7070F00A2
:10EA50003EC41C083EC62A89AE8997C0FFFFE780E6
:10EA600000D7585C1C5C6346B70E6394E50063E214
:10EA7000A70E3385A740B3B7A700B305B740130669
:10EA8000803E81469D8D97000100E78080B79314FA
:10EA90000501C180A1659385C503480097B0FFFFBC
:10EAA000E780C0558145480097D0FFFFE780603D73
:10EAB00083550404480097D0FFFFE780803E8355CC
:10EAC0002404480097D0FFFFE780A03D814589CC12
:10EAD000C167FD179305F00F6388F40026859750F2
:10EAE0000000E780E0E0AA85480097D0FFFFE780BC
:10EAF000403903554404814501CDC167FD17930595
:10EB0000F00F6307F50097500000E78060DEAA85EC
:10EB1000480097D0FFFFE780C03683456404480073
:10EB200097D0FFFFE780E03583457404480097D015
:10EB3000FFFFE7800035500001478146CE854A85BA
:10EB400097B0FFFFE780E07005611733FFFF6700B4
:10EB5000A35A814481B71733FFFFE702435883C7A5
:10EB6000950093F7F707A384F50097000000E7806E
:10EB700020ED1733FFFF6700C3581733FFFFE7028D
:10EB8000635483C795004111404D93F7F707A38461
:10EB9000F5002A8A3285B284AE8997D0FFFFE780DC
:10EBA000003E2A8B268597D0FFFFE780403D2A89CB
:10EBB000268597D0FFFFE780603A93170B0163CA61
:10EBC0000702E177CA97C207C183116763E3E702CF
:10EBD00093070910C207C1831307B00F637BF700C7
:10EBE00093170901C187AA8A634AF000C54763FEEB
:10EBF000570141011733FFFF6700035097B0FFFF34
:10EC0000E7802025E31725FFD5B763080B026306CD
:10EC10000902814463890A02B7077F002310640553
:10EC2000231124057CC0568597000000E780E0C3CF
:10EC30009304803EB304950239A0B7077F002320D8
:10EC400004047CC081440355240497E00000E7805D
:10EC5000A0A3A1C497C0FFFFE78060B7269593D714
:10EC6000F44133379500AE97BA9708DC5CDCCE856B
:10EC7000528597000000E780A0DC99E0232204047D
:10EC8000A1679387B70348003EC42302010002C670
:10EC900097E0FFFFE7808005A9BF814701481CDCA2
:10ECA000232E0403E9B71733FFFFE702434397C05E
:10ECB000FFFFE7802034E1473305F5029145975087
:10ECC0000000E78000C5E55711C59777FF1F23A314
:10ECD000A70681473E851733FFFF670083428547BC
:10ECE0001777FF1F230AF70482801733FFFFE7021D
:10ECF000033F9777FF1F9387A70380433DC0835748
:10ED000004046390A70683572404639CB7043689E0
:10ED1000B28497C0FFFFE78080AB5C5C63C3B7043D
:10ED20006395B7001C5C63EEA7028347640463F33A
:10ED3000F400A6872303F4048347740463F3970065
:10ED4000A687A303F4048357440441677D176385B2
:10ED5000E70085072312F4043C4481C7CA85268551
:10ED600082971733FFFF6700C3399777FF1F938799
:10ED700027FC9C43014599C303C587008280173354
:10ED8000FFFFE702C3350111B70707003EC683C77F
:10ED90009500584D0AC493F7F7070AC8A384F500F5
:10EDA0002A89AE8411CB1C4283C707002304F700D5
:10EDB00097900000E78000342164930554022800F6
:10EDC00097B0FFFFE780802397000000E78020FADC
:10EDD000AA85280097D0FFFFE780A00A30000147EE
:10EDE0008146A6854A8597B0FFFFE78080461304D9
:10EDF0004402480822CC230A010002CE97E0FFFF1C
:10EE0000E780C0EE05611733FFFF6700832F1733DC
:10EE1000FFFFE702C32C01117C003ECAB7070700C1
:10EE20003ECC7C003ECE83C795002E84AA8493F707
:10EE3000F707A384F500A16593855502480897B0AC
:10EE4000FFFFE780A01B97000000E78040F2AA8543
:10EE5000480897D0FFFFE780C0025008014781466D
:10EE6000A285268597B0FFFFE780A03E0561173396
:10EE7000FFFF670003299777FF1F938767EB9C438A
:10EE8000094599C303C5970082809777FF1F938731
:10EE900027EA9C43094599C303C5D7008280977729
:10EEA000FF1F9387E7E89C43014599C303C5A7006B
:10EEB00082801733FFFFE702E3200111B707080044
:10EEC0003EC683C79500404D0AC493F7F7070AC8AA
:10EED000A384F5002A89AE8429C41442854703C758
:10EEE000060063E0E70A834794000946814963808E
:10EEF000C702B307F740A304E400B339F00083C7A7
:10EF000016002305F40097900000E780A01E035729
:10EF10002403058B19C76386090097D00000E7809A
:10EF200000E9216493058402280097B0FFFFE78081
:10EF3000E00C97000000E78040F4AA85280097D0F5
:10EF4000FFFFE78000F497000000E78080F5AA85C6
:10EF5000280097D0FFFFE780C0F2014781463000CC
:10EF6000A6854A8597B0FFFFE780A02E13047402A0
:10EF7000480822CC230A010002CE97E0FFFFE78079
:10EF8000E0D605611733FFFF670003171733FFFF54
:10EF9000E702E31401117C003ECAB70708003ECC2B
:10EFA0007C003ECE83C795002E84AA8493F7F70792
:10EFB000A384F500A16593858502480897B0FFFFFB
:10EFC000E780C00397000000E78020EBAA8548088F
:10EFD00097D0FFFFE780E0EA97000000E78060EC51
:10EFE000AA85480897D0FFFFE780A0E950080147AD
:10EFF0008146A285268597B0FFFFE78080250561C1
:10F000001733FFFF6700E30F9777FF1F938747D200
:10F010009C43014599C303C5B70082801733FFFFA6
:10F02000E702E30B0111B70707003EC683C795004F
:10F03000404D0AC493F7F7070AC8A384F5002A894C
:10F04000AE8405C81C42054783C707006368F706FE
:10F050000347B400630FF700A305F4009790000086
:10F06000E78040098347B400B9CF97D0FFFFE7801E
:10F0700040BE21649305B400280097B0FFFFE780ED
:10F08000E0F797000000E78060F8AA85280097D095
:10F09000FFFFE78000DF014781463000A6854A85F3
:10F0A00097B0FFFFE780E01A2904480822CC230A22
:10F0B000010002CE97E0FFFFE78040C305611733F0
:10F0C000FFFF6700030497D0FFFFE78020BF55B71D
:10F0D0001733FFFFE702A30001117C003ECAB70708
:10F0E00007003ECC7C003ECE83C795002E84AA84C8
:10F0F00093F7F707A384F500A165AD05480897B01D
:10F10000FFFFE780A0EF97000000E78020F0AA85CE
:10F11000480897D0FFFFE780C0D6500801478146D6
:10F12000A285268597B0FFFFE780A01205611733FF
:10F13000FFFF670003FD9777FF1F938767BF9C431F
:10F14000094599C303C5C70082801733FFFFE70253
:10F1500003F901117C00AE843ECAA165B707070020
:10F160002A843ECCD1057C0048083ECE97B0FFFFF4
:10F17000E780C0E897000000E78020FCAA854808E7
:10F1800097D0FFFFE780E0CF500801478146A68572
:10F19000228597B0FFFFE780C00B05611733FFFFA3
:10F1A000670023F61733FFFFE70263F383C7950079
:10F1B00093F7F707A384F50097000000E78020F994
:10F1C0001733FFFF6700E3F31733FFFFE70283EF17
:10F1D00083C795000329C501411193F7F707A3845D
:10F1E000F5001C4283C90700854763E63707977718
:10F1F000FF1F9387E70A9C432E84AA8485CF97003C
:10F200000000E78080F389476306F5026304090282
:10F210008347C900638037032306390197900000B4
:10F22000E78040ED83572903898B89C797D0000079
:10F23000E780E0B72685A28597000000E78020F1EF
:10F24000A167CD0748003EC42302010002C697E033
:10F25000FFFFE780A0A941011733FFFF6700C3E963
:10F260009777FF1F9387C7AC9C431D4599C303C580
:10F27000E70082801733FFFFE70263E60111B7075B
:10F2800007003EC683C79500584D0AC493F7F70799
:10F290000AC8A384F5002A89AE8415C71C4283C717
:10F2A000070093968701E18663C40606854663815D
:10F2B000D7068346E7006388F6002307F700979098
:10F2C0000000E78020E321649305E400280097B064
:10F2D000FFFFE780A0D297000000E780A0F8AA8592
:10F2E000280097D0FFFFE780C0B901478146300072
:10F2F000A6854A8597B0FFFFE780A0F5350448084A
:10F3000022CC230A010002CE97E0FFFFE780009E97
:10F3100005611733FFFF6700C3DE1733FFFFE70206
:10F3200003DC01117C003ECAB70707003ECC7C001D
:10F330003ECE83C795002E84AA8493F7F707A38453
:10F34000F500A165B905480897B0FFFFE78000CB3D
:10F3500097000000E78000F1AA85480897D0FFFFDA
:10F36000E78020B2500801478146A285268597B0E4
:10F37000FFFFE78000EE05611733FFFF670063D8EA
:10F380001733FFFFE70203D4AA8401441779FF1F54
:10F390001309499AE14997C0FFFFE780A0C563447C
:10F3A000A400014519A833053403832709003E95BD
:10F3B000835725006397970011051733FFFF6700F8
:10F3C000A3D30504C9BF032E8500630A0E12177369
:10F3D000FF1F1303E3B40323030063150300294352
:10F3E0006390061203234E01631503001D436399C6
:10F3F00007101733FFFFE70203CCC689428A3E8914
:10F40000BA8AB684328BAE8B2A84B5E103554E009E
:10F4100019E501431A851733FFFF670043CDA16744
:10F42000A98F116763FBE70097000000E78080F574
:10F43000814597F0FFFFE780C0120844B70700E05E
:10F440005841F98F18455CC1B707001FF98F1CC5DB
:10F450005C4991C7610597E00000E780408BE38A33
:10F4600009FA228597900000E78060C65DB7328573
:10F4700097C00000E78040430D4349DD1C441167FD
:10F4800003D54700A167A98F63FBE7009700000041
:10F49000E78040EF814597F0FFFFE780800C032372
:10F4A000840093164B01D1828347B3000356630057
:10F4B0008588FD8BA305F300FD777D8E558EFD7647
:10F4C000FD16B204F18E83274301C58E231273010A
:10F4D0002313D3002304530123052301A304430171
:10F4E000BDDF228597B0FFFFE78080C9AA85084469
:10F4F000B5D1610597D00000E780207F8DB71D430F
:10F500001A8582801733FFFFE702C3BB0569AA840F
:10F51000AE89328A0144FD5A7D1997C0FFFFE7800A
:10F5200020A26347A40001451733FFFF6700C3BC57
:10F53000D84493171400BA9703D70700631F370303
:10F540002390570163070A00268597900000E78003
:10F55000A0809C449DC383D76700B3F72701639EB7
:10F560003701D288014881470147814601468145DC
:10F57000268597000000E78040E5050479BF173332
:10F58000FFFFE70223B479711C103EC4B7070F00D8
:10F590003EC61C103EC883C79500AA8A328593F7E1
:10F5A000F707A384F5002E89328497D0FFFFE78008
:10F5B000009D93170501C187635AF006AA89228529
:10F5C00097D0FFFFE780A09B2A8A4E85032B04007B
:10F5D00097B0FFFFE780609739ED8357440081447F
:10F5E0000544F11793B71700A303F1008345710099
:10F5F000DA872287D2864E86280097E0FFFFE780D1
:10F60000E057014781463000CA85568597B0FFFF15
:10F61000E78020C4A1679387F70348083ECC230AFC
:10F62000810026CE97D0FFFFE780406C45611733FD
:10F63000FFFF670063ACA2851306710097E0FFFF30
:10F64000E7806066AA84094455D1528597E0FFFFA0
:10F65000E78060D40D4459D90546D28526859700A8
:10F660000000E78060EA2A8451B71733FFFFE70202
:10F6700003A7835507000346270041112A842E85DE
:10F6800032C62EC497E0FFFFE780E0D001C93246C2
:10F69000A245228597000000E78000E7410117336B
:10F6A000FFFF670003A61733FFFFE702C3A083C76E
:10F6B00095004111AA8A93F7F707A384F5003285D4
:10F6C000AE89328497D0FFFFE780608B93170501E6
:10F6D000C1876357F00AC1452A8A228597C0FFFF78
:10F6E000E78080702A8D228597D0FFFFE7802089F0
:10F6F0002A89228597D0FFFFE7804086930705F887
:10F7000093F7F70F1307E007AA8B637BF7062285B1
:10F7100097D0FFFFE78080842A8C228597D0FFFF57
:10F72000E780C083AA8C5285032B040097B0FFFFAB
:10F73000E780A08139E98357440023110100814407
:10F74000F11793B71700A300F10005440347110018
:10F7500083562100938784005685DA882288528652
:10F76000CE8597F0FFFFE78020A7A167E907480053
:10F770003EC42302810026C697D0FFFFE7800057D2
:10F7800041011733FFFF6700839613061100A2851E
:10F7900097E0FFFFE7802051AA8409E523110100CB
:10F7A00009446DB7930521006A8597F0FFFFE78054
:10F7B000A0F02A8441FD835521009356C9001316F9
:10F7C000490185486688E2875E87858A5182268559
:10F7D00097000000E78060BF2A848DBF1733FFFFCA
:10F7E000E702638D83C7950041112A8B93F7F707D2
:10F7F000A384F5003285AE89328497C0FFFFE7808D
:10F80000007893170501C1876352F00A2A8A22857E
:10F8100097C0FFFFE780A076AA8A228597C0FFFFE6
:10F82000E780E0752A89228597C0FFFFE780007393
:10F83000930705F893F7F70F1307E0072A8C637710
:10F84000F706228597C0FFFFE7804071AA8C2285CA
:10F8500097C0FFFFE78080702A8D5285832B0400BC
:10F8600097A0FFFFE780606E39E583574400854429
:10F870000144F11793B71700A301F10003473100CA
:10F88000930784005A85DE882688D6865286CE85E0
:10F8900097F0FFFFE78040948D4748003EC4230265
:10F8A000910022C697D0FFFFE78040444101173303
:10F8B000FFFF6700C383A2851306310097E0FFFFB7
:10F8C000E780603E2A84894455D99356C9001316AF
:10F8D000490185486A88E6876287858A5182D6858C
:10F8E00097000000E78060AEAA8449BF1723FFFF9E
:10F8F000E702437D2A8981440144617A916A176B4A
:10F90000FF1F130BEB6197B0FFFFE780606463C7D5
:10F91000A40022851723FFFF6700037E83270900C9
:10F9200093991400CE9703D507003307450142078A
:10F9300041836364570305C103270B0019C785453D
:10F940003E8597400000E78060E9832709000504B1
:10F95000CE972390070085047DB797000000E780CD
:10F9600060A2832709000504CE972390070065D580
:10F97000814597F0FFFFE780C0BEF1BF1723FFFF6F
:10F98000E702437483C7950041112A8A93F7F7076A
:10F99000A384F50032852E89328497C0FFFFE7806B
:10F9A000005E93170501C187635AF004AA89832A70
:10F9B000040097A0FFFFE780405931E583574400DA
:10F9C00085440144F11793B71700A301F1000348E0
:10F9D0003100D68752850147CE862686CA8597D0C4
:10F9E000FFFFE780806AA167F50748003EC4230255
:10F9F000910022C697D0FFFFE780402F41011723D7
:10FA0000FFFF6700636FA2851306310097E0FFFFD9
:10FA1000E78060292A8489445DD99767FF1F93870F
:10FA200027509C4381CF044997B0FFFFE7804052A5
:10FA3000AA85268597400000E78040DA1305040177
:10FA400097000000E780C0EA228597800000E780E9
:10FA500000338144ADBF1723FFFFE702C36583C7AF
:10FA600095004111AA8A93F7F707A384F500328520
:10FA7000AE8932842311010097C0FFFFE780205038
:10FA800093170501C1876354F0062A8AC145228570
:10FA900097C0FFFFE7804035AA8B5285032B0400F7
:10FAA00097A0FFFFE780604A21E98357440085441F
:10FAB0000144F11793B71700A300F10003481100A8
:10FAC00003572100DA875685D2862686CE8597D0C1
:10FAD000FFFFE780805BA1679387270248003EC451
:10FAE0002302910022C697D0FFFFE780202041012A
:10FAF0001723FFFF6700A35FA2851306110097E09D
:10FB0000FFFFE780401A2A8489444DD99767FF1F79
:10FB10009387074198433E8901CF044997B0FFFF7F
:10FB2000E7800043AA85268597400000E78000CB48
:10FB30001305040197000000E78080DB97B0FFFF0A
:10FB4000E780004195443DD9930521005E8597F0FB
:10FB5000FFFFE78060B6AA8435F11C4803572100F7
:10FB600022852390E70097800000E78040218327CB
:10FB70000900A9D70355210097400000E780A0BDE8
:10FB800035BF1723FFFFE702035383C795004111D9
:10FB9000AA8A93F7F707A384F5003285AE893284E9
:10FBA00097C0FFFFE780A03D93170501C187635110
:10FBB000F0062A8A228597C0FFFFE780403C2A8909
:10FBC0005285032B040097A0FFFFE780003831E542
:10FBD0008357440085440144F11793B71700A301EC
:10FBE000F10003483100DA8756854A87D286268697
:10FBF000CE8597D0FFFFE7804049A167F90748000D
:10FC00003EC42302910022C697D0FFFFE780000E7A
:10FC100041011723FFFF6700834DA28513063100C2
:10FC200097E0FFFFE78020082A8489445DD9916727
:10FC3000CA97C2071167C1831307F7EF8544E362D0
:10FC4000F7FA9767FF1F9387A72D9843BE8B01CFC5
:10FC5000044997B0FFFFE780A02FAA85268597402B
:10FC60000000E780A0B71305040197000000E780BB
:10FC700020C897B0FFFFE780A02D95443DD11C48D8
:10FC8000228581442390270197800000E780200F80
:10FC900083A70B00B9D74A8597400000E780A0AB47
:10FCA00089B71723FFFFE70283432A844105B28403
:10FCB00097000000E780C0C311C52285978000002F
:10FCC000E780E00B81460146A685228597800000EB
:10FCD000E780C04E1C4C89C7DC4799C322858297B8
:10FCE0001723FFFF6700E3419767FF1F93874704D0
:10FCF0009C43014599C31385070182809767FF1FC5
:10FD000093870703884382801723FFFFE702233D81
:10FD10009317C600DD8DC2054111C1812A8432C608
:10FD200097C0FFFFE780E017324622851182937566
:10FD3000F60F97C0FFFFE780C01441011723FFFFB4
:10FD40006700233C1723FFFFE702C33779713C08A4
:10FD50003ED2B7070C003ED43C083ED683C7950080
:10FD6000AE842A8993F7F707A384F500A1659385EC
:10FD70003504481097A0FFFFE7804028C165FD15B6
:10FD80000144176AFF1F130A2A1B930A400EAE890B
:10FD90002E8B2EC697B0FFFFE780801E420593177B
:10FDA00004014181C183B24563E9A702C167FD1720
:10FDB0006387F500481097C0FFFFE780800E501062
:10FDC00001478146A6854A8597A0FFFFE7806048E6
:10FDD00045611723FFFF670023323307540383274E
:10FDE0000A0BBA9703D6C701630A3601638A350145
:10FDF000481097000000E78060F1DA85050451BFE4
:10FE0000B285EDBF1723FFFFE702E32A79717C0873
:10FE10003EC8B70711003ECA7C083ECC83C7950098
:10FE2000AA89328593F7F707A384F5002E8997C036
:10FE3000FFFFE780C01485676378F504A165AA8495
:10FE40008905080897A0FFFFE780401B268597409B
:10FE50000000E78060ED133415000A04A28508084D
:10FE600097C0FFFFE780E001A685080897C0FFFF65
:10FE7000E780200325CC014781461008CA854E85BE
:10FE800097A0FFFFE780E03C45611723FFFF670075
:10FE90000326B30754030327CA0ABA9703D70700F8
:10FEA000631C970003D62700638065050808970048
:10FEB0000000E780A0E5DE8505042EC697B0FFFFB1
:10FEC000E780000D4205931704014181C183B245CB
:10FED000E3E1A7FCC167FD17E38FF5F8080897C0B9
:10FEE000FFFFE78000FC41BFB285F9B7C165FD1592
:10FEF0000144176AFF1F130A2A04930A80022E8BFB
:10FF0000AE8B65BF1723FFFFE702631D18418347D0
:10FF1000170083460700A207D58FD207D18323900D
:10FF2000F50083472700034717008D45A207D98FA7
:10FF300091832310F60097C0FFFFE780A0E9172305
:10FF4000FFFF6700031C1723FFFFE702A317C1642D
:10FF500001441769FF1F130929FE93098002FD144C
:10FF600097B0FFFFE780C0026347A4000145172355
:10FF7000FFFF67006318330534038327C90A3E95E2
:10FF800083570500E38597FE0504D9BF1723FFFFBC
:10FF9000E70243132A8AAE89B284B68A97400000EA
:10FFA000E78080D819E591473E851723FFFF67005A
:10FFB000A3142A894E8597C00000E780E08E2A842A
:10FFC000638E0A048D476DD103570500C547E31DB5
:10FFD00047FD0347F9018546AD47E317D7FC834743
:10FFE000450081CF4146A6855D0597F00000E7807A
:10FFF000C09E814755D9AD4745BF1309650123020E
:020000040001F9
:10000000E500CA85268597100000E780606231C14F
:10001000A547E38B0AF82302040079B705C183578B
:100020000500E39247F94146A685190597F00000BF
:10003000E780A09A81472DD99947BDB74E85970093
:100040000000E78080F02A84954739DD13095500C8
:100050004DBF4146A68523104401231134011305E9
:10006000190097F00000E780A09922859780000092
:10007000E780A0EA81470DBF1723FFFFE7022306B1
:1000800079717C003ECCB7070A003ECE7C003ED0A2
:1000900083C79500B2842E8493F7F707A384F500F5
:1000A0001306A1002A892C00268597000000E7800E
:1000B000A0E5A16528088D0597A0FFFFE78000F463
:1000C00090408355A10003558100854697000000AC
:1000D000E78000ECAA84AA85280897C0FFFFE78084
:1000E00040DA0356A10083558100280897000000DC
:1000F000E780C0C1300801478146A2854A8597A0A4
:10010000FFFFE7800015854748103ED42302910287
:1001100002D697D0FFFFE78060BD45611723FFFF40
:10012000670023FE1723FFFFE70263FB79717C0062
:100130003ECCB7070A003ECE7C003ED083C7950078
:10014000B2842E8493F7F707A384F5001306A10069
:100150002A892C00268597000000E780E0DAA16557
:1001600028088D0597A0FFFFE78040E99040835560
:10017000A10003558100814697000000E78040E11F
:10018000AA84AA85280897C0FFFFE78080CF03567E
:10019000A10083558100280897000000E78000B780
:1001A000300801478146A2854A8597A0FFFFE78076
:1001B000400A48102302910202D402D697D0FFFFD2
:1001C000E780C0B245611723FFFF670083F3172361
:1001D000FFFFE702C3F097000000E78060DB172312
:1001E000FFFF670003F29767FF1F9387A7B4884359
:1001F00082801723FFFFE70283EE8357250041111A
:10020000AE842A842307B10017F5FFFF13052546A6
:100210006C002316F10097A0FFFFE780804591C492
:10022000228597800000E780E0D6FD572310F40078
:10023000130620028145130554009720FFFFE78035
:1002400000ED41011723FFFF6700A3EB1723FFFF1A
:10025000E70243E779717C003ECCB7070A003ECE47
:100260007C003ED083C79500AA89AE8493F7F70738
:100270003285A384F5001306A1002C00970000002E
:10028000E78080C803558100114497400000E78053
:10029000A0A915C50355A100014497B00000E7804F
:1002A000A06011CD035705008357810045446318B2
:1002B000F700854597000000E780E0F301442169DD
:1002C00093053900280897A0FFFFE78020D3A28577
:1002D000280897C0FFFFE780C0BA0356A1008355E6
:1002E0008100280897000000E78040A230080147FD
:1002F0008146A6854E8597A0FFFFE78080F54810D0
:100300004AD42302810202D697D0FFFFE780009EE5
:1003100045611723FFFF670023DE1723FFFFE70276
:1003200063DA9767FF1F9387A7A02A8488432E89E3
:1003300015C5035745038357C4016311F7022326EC
:10034000050223180502410597D00000E780209C94
:100350006306090097800000E78060DB81449769AD
:10036000FF1F938969BD130A800297B0FFFFE780E2
:1003700020C263C4A4049767FF1F938727A49C43EC
:1003800099C70355C40197200000E780C0BD6307EB
:100390000900228597800000E780C0A01306400E68
:1003A000814522859720FFFFE78060D6FD57231EF9
:1003B000F4001723FFFF670023D43385440383A78A
:1003C000C90A3E95035705008357C4016317F70018
:1003D000CA8597000000E78000E2850479B71723FB
:1003E000FFFFE70223CE83C795004111AA8993F747
:1003F000F707A384F5003285AE8497C0FFFFE7803E
:1004000000B885676378F5042A8997400000E78083
:10041000A091014401CD83D70400314463882701B2
:10042000854597000000E78080EF01444E85A28655
:100430004A86A68597D0FFFFE780A09CA167938797
:10044000170448003EC42302810002C697D0FFFF74
:10045000E780C08941011723FFFF6700E3C9172325
:10046000FFFFE70223C69767FF1F9387678C8043D0
:1004700029C4014597C00000E78000218147014859
:10048000C1641CDC232E0403232004041769FF1F0E
:10049000130989AA01449309400EFD1497B0FFFF88
:1004A000E78000AE634FA400814517F5FFFF1305F9
:1004B000857F97A0FFFFE780C01B1723FFFF670022
:1004C000A3C3330534038327090B3E958357C50126
:1004D00063879700854597000000E78040E40504A6
:1004E00075BF9357050113D78700A380F5009317B5
:1004F0000501C183A1832380E5002381F500A38149
:10050000A50082801723FFFFE70263BD23000500DB
:1005100083C71500A300F50083C725002301F5005C
:1005200083C73500A301F50083C745002302F5000A
:1005300083C75500A302F50083C7650093059500A6
:10054000A30305002303F50023040500328597006B
:100550000000E78040F91723FFFF670083BA1723E5
:10056000FFFFE70223B64111E9540DCD85CD93F984
:10057000C5FF2E842A89AA84338AA900B7EA040019
:1005800063189A020D88854411CCB7E704009C5F7C
:1005900082972AC622866C003305390197E0000055
:1005A000E7800046268541011723FFFF6700C3B49B
:1005B00083A78A039104829793170501C183A183BE
:1005C000A38EF4FE93570501238FF4FEA183238E9F
:1005D000A4FEA38FF4FE6DB763E6D5021723FFFFD9
:1005E000E702E3AFB28741113686BE8536C697E093
:1005F0000000E780E040B246410136851723FFFF47
:10060000670023B081463685828083870500138783
:10061000F5003D05FD8793F77708834607007D15B4
:100620008606B58FA300F5006307B7007D178347E3
:1006300017009D83DDB782801723FFFFE70223AAFF
:10064000B7E7040083A7070932872A863A8582978D
:10065000133515001723FFFF6700A3AA15C18147B3
:100660008DC11723FFFFE70283A7414697E00000F3
:10067000E780003985473E851723FFFF670063A8A1
:1006800081473E8582801DCD1723FFFFE70223A50A
:10069000414681452A849720FFFFE78040A74146D5
:1006A0008145130504039720FFFFE78040A601471B
:1006B000C1672322040438C87CC805451723FFFFFF
:1006C000670023A40145828081473DCDB5CD172326
:1006D000FFFFE702C3A0B2842E891306800581457F
:1006E0002A849720FFFFE78080A2CA8524C426853C
:1006F00097000000E780C0F641468145228597209B
:10070000FFFFE780C0A03044A2852285970000004B
:10071000E780C0F293040401A285268597000000BB
:10072000E780E0EEA6851305040297000000E7804D
:1007300000EE228597000000E78020F585473E8582
:100740001723FFFF6700E39B3E8582801723FFFF8F
:10075000E70243974111E9540DCD85CD93F9C5FFCB
:100760002E842A89AA84338AA900B7EA04006398F0
:1007700044030D88814411CCB7E704009C5F829745
:100780002AC622866C003305390197E00000E78015
:100790002027268541011723FFFF6700E39583A7E4
:1007A0008A039104829793170501C183A183A38EC5
:1007B000F4FE93570501238FF4FEA183238EA4FE3C
:1007C000A38FF4FE6DB765CD1723FFFFE702838F7C
:1007D000B28411E605451723FFFF6700E3912A84E1
:1007E0002E890145EDD93C487848B3E6E700E5D6C7
:1007F0009386F7FFB3B7F6007D17032A4404BA9730
:1008000034C87CC863050A06C14913050A03B389C5
:1008100049412295637D3601B2862E86A6859700D2
:100820000000E780A0DB7C40BE9464C065B7CE8644
:100830002E86CE8597000000E78040DAC114D2945E
:100840004E9923220404A2879306040103C70700DC
:1008500003C607038507318FA38FE7FEE398F6FEF3
:100860003044A285228597000000E78020DD26998C
:10087000C1493306994063EC9900A9DCA686A68598
:100880001305040397000000E78040D579BF814736
:10089000B306F4003307F6000347070083C50600DC
:1008A00085072D8F2380E600E39437FF3044A2852F
:1008B000228597000000E78060D8C1145DBF014524
:1008C00082800DC11723FFFFE702638113068005B5
:1008D00081459720FFFFE780808305451723FFFFB1
:1008E0006700238201458280814749C5C1C517132E
:1008F000FFFFE702C37EFC4141462E84AA84639930
:10090000C70413860501A2878146C14503C70700B6
:1009100003C507038507298F3305D6000345050066
:100920008506298FA38FE7FEE392B6FE3044A285A9
:10093000268597000000E78060D0228597000000A0
:10094000E78060F885473E851713FFFF6700637BEC
:10095000138507031D8E814522959710FFFFE780C1
:10096000007B7C40130700F813060402A29723883B
:10097000E70251BF3E8582801713FFFFE70223760F
:100980006D712E84B284AA85901028003689970054
:100990000000E780A0D309EDD55725A050400C40BA
:1009A000280097000000E78040E27DD5FD14210477
:1009B000F5F42C004A8597000000E78020F381477A
:1009C00061DD3E8551611713FFFF670083731713C5
:1009D000FFFFE702C37041112EC432C62C0005464A
:1009E00097000000E78080F941011713FFFF6700BF
:1009F00043711713FFFFE702836E01112A842EC68D
:100A000002C802CA02CC02CE97E00000E780C023F1
:100A1000B2462A86A285080897000000E78060FB9E
:100A20001375F50F05611713FFFF6700836D17132B
:100A3000FFFFE702C36A7971B2872A84214623083F
:100A4000B10013051101BE853AC436C697E0000017
:100A5000E78000FBB24693059101368597000000C0
:100A6000E78060A82285141035460C089700000026
:100A7000E78020F62A84224701E921460C103A85B6
:100A800097E00000E780C0F7228545611713FFFF5C
:100A9000670023671713FFFFE70263647171AE8479
:100AA000AA850A85328497000000E78060BB11C9DF
:100AB0000A86A685228597000000E78020B8814736
:100AC00011E1C5473E854D611713FFFF6700636362
:100AD0001713FFFFE702A35D1D712A8AB289BE8446
:100AE00035468547130511012E8CB68A3A8BC28C88
:100AF000468D2308F10097E00000E78060F01010B9
:100B00000C085285231F010097000000E780C0F801
:100B10002A843DEDA1476313FD089307900591E0FA
:100B2000E5473546E2851305110113990A012308AB
:100B3000F1001359090197E00000E78060EC1357BA
:100B4000890093978A00D98F90080C085285231F3B
:100B5000F10097000000E78020F42A8415E9A1E461
:100B60009387FA0091831379F9003EC66313090055
:100B70004149668B8144C14B854DB247639F970CB9
:100B80006A868C0033855C0197E00000E78040E7CF
:100B9000228525611713FFFF6700235593079004F3
:100BA000C9F0A547BDBF834701050947C14B2308CD
:100BB000F10083471105A58FA308F1009387240056
:100BC000814463E1FB04014714083386E6008C0886
:100BD000B386E400BA95DA9683C6060083C505009D
:100BE0000507AD8E2300D600E390E7FE4147639CE6
:100BF000E70490080C08528597000000E780C0E9E0
:100C000025D181A0B3069B00BA871008B305F60072
:100C100090083E9603C50600034606008507850634
:100C2000298E2380C500E39277FF998F90080C08E6
:100C30005285BE9497000000E78000E6894701478F
:100C400049D12A84B1B790083E960346060014089D
:100C5000BE962380C600850759BFB24785046387C7
:100C6000971481471808B306F70098083E97338613
:100C7000F90003470700034606008507318F2380EC
:100C8000E600E39177FF90080C085285970000007A
:100C9000E78080E05DF53546E28513051101230804
:100CA000B10197E00000E780A0D5139704014183CC
:100CB000939784002183D98F10180C085285231F25
:100CC000F10097000000E78020DD25FD8147101826
:100CD0003387F9003E960347070003460600B30634
:100CE000FB008507318F2380E600E39277FF65A83C
:100CF0001808B306F70098083E973386F9000347B3
:100D00000700034606008507318F2380E600E3E1F4
:100D100027FFCA87639E770990080C0852859700C1
:100D20000000E78060D711FD81479800B306F70007
:100D3000900818103E973E960347070003460600AA
:100D40008507318F2380E600E39177FF3546E28502
:100D5000130511012308B10197E00000E78040CAA4
:100D6000139704014183939784002183D98F10182E
:100D70000C085285231FF10097000000E780C0D1C6
:100D8000E31105EC814710183387F9003E960347BD
:100D9000070003460600B306FB008507318F23805A
:100DA000E600E3E227FFC109410BC1BB814785B7DC
:100DB0009408BE9683C6060018083E972300D70005
:100DC000850789BF638006321713FFFFE702232ED2
:100DD00059712A84BE89B28B8547354613051102A5
:100DE0002E8B468C4289BA8A368A2300F10297E01C
:100DF0000000E780E0C010180C10228523170102C4
:100E000097000000E78040C963180512A147631FDF
:100E1000FC069307900563930900E5473546DA859C
:100E20001305110293140A012300F102C18097E017
:100E30000000E780E0BC93178A0013D78400D98FA5
:100E400090080C1022852317F10297000000E7801C
:100E5000A0C47DE1639209049307FA00BD889183E1
:100E600091E0C144C207C183DE8C814A3EC6414D38
:100E7000B24763E2FA0E6286B3854B01881097E0B1
:100E80000000E78080B54DC93D557DA093079004D3
:100E9000E39609F8A54759B7834701050947C14CAF
:100EA0002300F10283471105B3C7F900A300F10243
:100EB00093872900814963E1FC04814618103306B9
:100EC000D7008C083387D900B6955697034707009B
:100ED00083C5050085062D8F2300E600E390D7FE2D
:100EE00041476390E70690080C10228597000000A8
:100EF000E78080BA35D189A0B3863A01BA8710104D
:100F0000B305F60090083E9603C5060003460600AA
:100F100085078506298E2380C500E39297FF3387D6
:100F2000EC4090080C102285BA9997000000E780E9
:100F3000A0B68947014741D165611713FFFF6700DC
:100F4000C31A90083E96034606001410BE962380EE
:100F5000C600850779B7B247850A93990A01939D20
:100F60008A0093D909016391570F85473546DA8581
:100F7000130511022300F10293D9890097E00000C4
:100F8000E78000A8B3ED3D0190000C1022852317E7
:100F9000B10397000000E78020B059FD8147A68982
:100FA00063EA970626860C084A8597E00000E780EA
:100FB00020A581471810B306F700100898083E973F
:100FC0003E9603470700034606008507318F2380BE
:100FD000E600E3E197FE639FA90590080C102285C7
:100FE00097000000E78040AB21F981479810B306D5
:100FF000F700900818183E973E96034707000346EF
:1010000006008507318F2380E600E391A7FF4109A1
:10101000C10CB9BD18089000B306F7003E9633879F
:10102000FC0003470700034606008507318F238035
:10103000E600B5B798084E97034707001C10CE97F7
:101040002380E700850941BF85473546DA851305CA
:1010500011022300F10293D9890097E00000E78094
:10106000209AB3ED3D0190000C1022852317B103A7
:1010700097000000E78040A2E31005EC81471808C4
:101080009000B306F7003E963387FC000347070045
:10109000034606008507318F2380E600E391A7FF12
:1010A00041460C084A8597E00000E780609581473B
:1010B0001810B306F700100898083E973E960347AD
:1010C0000700034606008507318F2380E600E39181
:1010D000A7FF90080C10228597000000E780C09BB6
:1010E0001DD599BD7D5582801713FFFFE70223FFB1
:1010F00001112A842E8593055100328902C002C253
:1011000002C402C69304740097F0FFFFE780A03D7D
:101110001D46A6851305910097E00000E780408EEC
:1011200010088A854A8597000000E780E09619ED4F
:1011300093071400180883C60700034607008507B5
:101140000507B18EA38FD7FEE397F4FE0561171351
:10115000FFFF670003FB1713FFFFE702A3F62E84D0
:101160008C414111AA89838715003289914463D348
:101170000700A1449757FF1F938787129C43A1C77D
:10118000C1CA8D472310F10083C725004A8523017A
:10119000F10083C73500A301F10083C74500230296
:1011A000F10083C75500A302F10083C765009305D2
:1011B0009100A30301002303F1002304010097F031
:1011C000FFFFE78040320C404A860A8597F0FFFF18
:1011D000E78080330328040083564400A6881D0856
:1011E00081470147E51642868A854E8597000000B3
:1011F000E780408E2A8919E5A685228597B0FFFFF2
:10120000E780E0C14A8541011713FFFF6700C3EE85
:101210004A860A8597F0FFFFE780002F6DB7171306
:10122000FFFFE70223EA2E848C414111AA898387BC
:1012300015003289914463D30700A1449757FF1FDB
:10124000938707069C43A1C7C1C68D472310F100B1
:1012500083C725004A852301F10083C73500A30118
:10126000F10083C745002302F10083C75500A302A4
:10127000F10083C7650093059100A30301002303D8
:10128000F1002304010097F0FFFFE780C0250C4028
:101290004A860A8597F0FFFFE780002783564400BF
:1012A000032804008A85858EC2061D08C182231288
:1012B000D400A68881470147E51642864E859700EF
:1012C0000000E78060B041011713FFFF6700C3E231
:1012D0004A860A8597F0FFFFE78000234DBF17136A
:1012E000FFFFE702C3DFB335B000011185052A898E
:1012F0001315F601336515012308B100930511019B
:1013000036843AC632C03EC442C297F0FFFFE7803F
:10131000801DA2471248425593D68700230BF10047
:101320009305910193578800A30AD100A30BF10004
:10133000230C010197F0FFFFE780E01A32470246D5
:1013400003280400B337E000835644009207914419
:1013500011C2A1444A85A68842860C0897F0FFFF77
:10136000E78040772A8919E5A685228597B0FFFF97
:10137000E780E0AA4A8505611713FFFF670063D87D
:101380001713FFFFE70203D401113EC68647B335AA
:10139000B0008505AA891315F6015D8D2308B100FB
:1013A0009305110136843A89B28442C446C297F04B
:1013B000FFFFE78040132248924816459357880064
:1013C000A30AF1009305910193D78800230B010133
:1013D000A30BF100230C110197F0FFFFE780A01091
:1013E0003247104083564400B337E0009207032889
:1013F0000900914891C0A1480C084E859700000053
:10140000E780809CAA8401E9835544004A8597B00F
:10141000FFFFE780C0A0268505611713FFFF670067
:10142000A3CDAA959307F00F170701001307075DD7
:101430006317B50013C5F7FF1375F50F8280050517
:101440008346F5FFB58FBA9783C70700D5B7035713
:10145000450014419307F00F170601001306065AC2
:10146000369742074183139506014181631BE500CE
:10147000AD8FB29703C50700130515F3133515009B
:101480008280850603C5F6FFA98FB29783C7070040
:10149000D9BF1713FFFFE70283C4B28736842E86B5
:1014A000BA86AA853E85BA8497F0FFFFE78060522E
:1014B000634F0500228597D00000E780E0782A86F8
:1014C000A686A285268597F0FFFFE7808050171338
:1014D000FFFF670003C31713FFFFE702A3BE5D71A1
:1014E0002A8BAE8A170501001305C54E2C00B28465
:1014F000368ABA893E8997F0FFFFE780C04F2A8479
:101500005DE134104146DA85280097F0FFFFE7805F
:10151000404C2A8449E98547A303F100A6C29307FA
:1015200071002408BEC4A68685470D462C182810D5
:1015300002DC02DED6C0BEC697F0FFFFE7800044A3
:101540002A8435E183477102A6860D4693F7F70793
:101550002300FA00C1473EDE2C188947281026DCFC
:10156000A303F10097F0FFFFE78040412A8405EDD7
:101570004146A6854E8597D00000E78060488D479C
:10158000A6860D462C182810A303F10097F0FFFF44
:10159000E780C03E2A8401E94146A6854A8597D066
:1015A0000000E780E045228561611713FFFF6700B7
:1015B000A3B41713FFFFE70283B297F700009387E6
:1015C000E7A0984383C7470079712A89AE8417053D
:1015D00001001305A5400C083AC42306F10097F05A
:1015E000FFFFE78040412A8405ED14104146CA857B
:1015F000080897F0FFFFE780C03D2A8415E1140832
:1016000015462C00081097F0FFFFE780803C2A84E5
:1016100001E921462C08268597D00000E780403E4E
:10162000228545611713FFFF6700A3AD1713FFFF66
:10163000E702E3AA97F70000938747999C477971DF
:10164000AA842E84170501001305C5390C083EC66F
:1016500097F0FFFFE780203A0DE914104146A68578
:10166000080897F0FFFFE780C03605E1140811462F
:101670006C00081097F0FFFFE780A03519E583475D
:10168000F10193F7F7032300F40045611713FFFFFF
:10169000670023A71713FFFFE70263A43688A1485A
:1016A00081470147E54697F0FFFFE780A042171307
:1016B000FFFF670003A51713FFFFE70243A2368869
:1016C000A14881470147E54697F0FFFFE780C06FDB
:1016D0001713FFFF6700E3A21713FFFFE70223A022
:1016E00001112A842E850C0832C697F0FFFFE7808F
:1016F000803009ED3247970601009386262D1008A9
:10170000C145228597000000E780E0D805611713E6
:10171000FFFF6700039F1713FFFFE702439C411180
:10172000C1472EC032C48A8509463EC23EC697F0E4
:10173000FFFFE780A02441011713FFFF6700639CB0
:101740001713FFFFE702A3994111AE861306100994
:10175000AA850A8502C002C202C402C697F0FFFF32
:10176000E780202741011713FFFF670083991713B4
:10177000FFFFE702C396328797060100938606278C
:101780002E869305000297000000E780C0D0171353
:10179000FFFF670003971713FFFFE7024394797178
:1017A000C1472ACC2ED032D42C080D4628003ECE7C
:1017B0003ED23ED602C402C602C802CA97F0FFFF5C
:1017C000E780C01B45611713FFFF67008393171362
:1017D000FFFFE702C3900111AA842E8417050100C0
:1017E000130545218A8597F0FFFFE780C02015E5A6
:1017F00014084146A6850A8597F0FFFFE780601D23
:1018000009ED8347E1010347F101A207D98FCA0718
:10181000C9836177D98F2310F40005611713FFFF87
:101820006700238E15CD1713FFFFE702438B974701
:10183000FF1F9387A75490439745FF1F93854554F7
:101840001745FF1F1305854F97D00000E78000C59F
:101850001745FF1F1305854E1713FFFF6700638AA7
:101860001745FF1F1305854D82808DCD1713FFFF90
:10187000E702E3869747FF1F938747509443011180
:101880002E840A869745FF1F9385854F97D00000C9
:10189000E78040C60A850294014505611713FFFFE2
:1018A000670023867D5582801713FFFFE70223839D
:1018B00097D00000E78080D19747FF1F23A0A74C57
:1018C00017F5FFFF1305E5C997B00000E780C07466
:1018D0001713FFFF6700E3821747FF1F1307474CEB
:1018E0009317150008433E95FD572310F50082809D
:1018F0001703FFFFE702A37E2A84084009E51713B8
:10190000FFFF670003801C4158401CC06313E500C3
:101910005CC08347550023200500F99BA302F50016
:1019200097A0FFFFE780207CC9BF1703FFFFE702F6
:1019300063799747FF1F9387A74898432A8411CB61
:101940008347350093F7070289C70355050089458A
:1019500002971305440197B00000E780403B835590
:1019600004000355E40097300000E780A00C4858BD
:1019700019C597A0FFFFE7800077232A040213050B
:10198000840397000000E780E0F68144B149979016
:10199000FFFFE780206A63CBA40283473400232043
:1019A000040493F727FCA301F40000489790FFFF7D
:1019B000E780406913161500814522859700FFFFD7
:1019C000E780E0741703FFFF67000373B3873403F6
:1019D0000329040385043E994A8597000000E780A7
:1019E00060F12304090065B78347350093F70702C8
:1019F00099E3014582808357E500E39CB7FEC16708
:101A0000FD176316F60005458280054599A8170362
:101A1000FFFFE702C36C93170601C187B2842A84D3
:101A200001496359F002835705009DCB0145636767
:101A3000F600034584003E953325A6001375F50F87
:101A40000DA01C4813171900BA9783D70700E38E1F
:101A500097FA05099790FFFFE780C05EE343A9FE70
:101A600001451703FFFF6700C3691703FFFFE70284
:101A70006365AE89AA849790FFFFE78060522A844D
:101A800097D0FFFFE780A02EAA86014713068401A6
:101A900097050000938585E41745FF1F13058530E2
:101AA0009790FFFFE780E0182A8925C98C4413042A
:101AB000C50022859E0593F5050897A0FFFFE780E6
:101AC000403CCC4083877400E18163DD070493E5EB
:101AD0000508228597A0FFFFE780A03A0D46938571
:101AE0004400228597A0FFFFE780C03683D504001D
:101AF000228597A0FFFFE780E03D83D52400228563
:101B000097A0FFFFE780003D03D6490083A50900A9
:101B1000228597A0FFFFE780E0334A851703FFFF88
:101B20006700835D93F5F5076DB71703FFFFE702C5
:101B3000035B01112A84328532C697A0FFFFE7803C
:101B4000E0279780FFFFE780C030835704001747E6
:101B5000FF1F1307673E3246231BF100930700F86F
:101B6000A30DF1001C471843231AA1008983858B1C
:101B7000B307F740B28548083ECE231C0100230D71
:101B8000010097000000E78080EE05611703FFFF6A
:101B9000670023571703FFFFE702C35200410145C7
:101BA0003DC49304C40026853289AE8997A0FFFF07
:101BB000E780C02495452A8A2685035B040197A007
:101BC000FFFFE7802021268597A0FFFFE780603E8A
:101BD0008D45AA8A268597A0FFFFE780A01F26854E
:101BE00097A0FFFFE780E03C5C48420A135A0A01D5
:101BF000D2975CC423186401814763983A01460573
:101C00004D81330625419337160013F5F70F17035F
:101C1000FFFF6700634E1703FFFFE702C3498969AF
:101C20002A8BAE8B328AB68A81440144314CFD192D
:101C30009790FFFFE780004063CDA4009790FFFFDF
:101C4000E7804042018D33B5AA001703FFFF67000C
:101C5000034A3389840383270B003E9963170A00E4
:101C60008347890085043E94E1B703560A00DE8568
:101C70004A8533F6C90097000000E780E0F16DD196
:101C80000545E1B71703FFFFE702634501112A8409
:101C90007C000355E5003ECAB70707003ECC7C0038
:101CA0003ECE97200000E78020082A898545480815
:101CB00097A0FFFFE78020399945480897A0FFFFCC
:101CC000E780E015AA844A8597200000E780A008F5
:101CD0002380A4009747FF1F938707269C434166F4
:101CE000130606F09396870113D78701558F93D675
:101CF0008700F18E558FA207B706FF00F58FD98FA9
:101D000011462C00138514003EC497D00000E780D4
:101D100020CF5008A3820400894522859700000047
:101D2000E780E0E019C9AA851305840397A0FFFFA7
:101D3000E780E0313C4085073CC005611703FFFFA9
:101D40006700233C1703FFFFE70263399790FFFF0B
:101D5000E78040312A8405049790FFFFE780802FB9
:101D60003305A402F14791453305F50297200000A1
:101D7000E78020BA11E565551703FFFF6700633858
:101D80009747FF1F23A6A7029790FFFFE780802DAC
:101D90002A8405049790FFFFE780C02B3305A40237
:101DA0008945060597200000E780A0B669D59747CA
:101DB000FF1F23A7A7FE9790FFFFE780A02A2A8492
:101DC00005049790FFFFE780E0283304A4029747BB
:101DD000FF1F239987FC9790FFFFE780A0282A84A4
:101DE0009790FFFFE7800027930714003385A70231
:101DF0009747FF1F2399A7FA970701009387478307
:101E00001747FF1F2324F7FA0145BDB71703FFFF4C
:101E1000E702432BAA842E8901449749FF1F938927
:101E2000A911130A80069790FFFFE780A02263475D
:101E3000A40001451703FFFF6700032C330544038B
:101E400083A709024A86A6853E9597000000E78091
:101E5000E0B919E10504C1BF0545E9BF1703FFFF5C
:101E6000E7026325AA8A2E8BB28B368C3A8A81448C
:101E700001448149974CFF1F938C0C0C130D800675
:101E80009790FFFFE780001D63C9A40011E085491A
:101E90004E851703FFFF670083253389A40383A7BB
:101EA0000C025E86D6853E994A8597000000E78041
:101EB000E0B31DC19790FFFFE780C01A0544636D32
:101EC0004501D2866286DA85130509039700000072
:101ED000E780A0D411C1854985045DB71703FFFFD2
:101EE000E702431EC16441112A8901449749FF1F3B
:101EF00093898904130A8006FD1436C632C42EC2A3
:101F00009790FFFFE780001592452246B24663484E
:101F1000A400014541011703FFFF6700E31D3305DE
:101F2000440383A709023E9509C683473500C18B48
:101F30009DC791C68347350093F707028DC363069B
:101F400099008357E500639C27010357050001CBE7
:101F500063E7E50083478500BA97E3CDF5FA05040A
:101F600069BF1703FFFFE702E315C1642A89014433
:101F70009749FF1F938949FC130A8006FD14979027
:101F8000FFFFE780200D6346A4001703FFFF6700F3
:101F9000A3163305440383A709023E958357E50042
:101FA000638A9700630499006396270197000000F5
:101FB000E780E0970504E1B71703FFFFE702230F6F
:101FC00089692A8AAE8A328BB68B8144174CFF1FEF
:101FD000130C8CF6930C8006314DFD199790FFFF82
:101FE000E780400763C6A4001703FFFF6700E30F05
:101FF0003389940383270C028355CA015A863E997C
:102000004A8597000000E780609E31C1814D15A090
:102010003384AD038327090303D60B00D68533F63B
:10202000C9003E94228597000000E780E0B609E9E8
:10203000850D9790FFFFE780E0FFE3CBADFC01A8A3
:10204000228597000000E780E08A230404008504CD
:1020500071B71703FFFFE70203064169AA8A014A25
:10206000174BFF1F130B4BED7D19C14B054C979080
:10207000FFFFE78020FE6346AA001703FFFF67000B
:10208000030793098006B3073A0383290B02BE991D
:1020900083D7E900638E270163842A01639A57017D
:1020A00003A4890301E84E8597000000E780C0BDC6
:1020B000050A75BF83570401639977099304C40027
:1020C000268597A0FFFFE78060D385452A8D26856A
:1020D000835C040197A0FFFFE780C0CF268597A00F
:1020E000FFFFE780A0E762056185635905048D4520
:1020F000268597A0FFFFE780E0CD8945268597A03C
:10210000FFFFE78020CD8945268597A0FFFFE78068
:1021100060CC8545268597A0FFFFE780E0CC83470C
:102120000500094793F7F707639AE7009945268565
:1021300097A0FFFFE78040CBA30285014848337D8D
:102140002D01231894016A9548C40040A1BF1703CC
:10215000FFFFE702C3F837E404008327041D8297DA
:102160009747FF1F83C747CA1715FF1F1305053C75
:10217000A300F5008327441C82978327841C814693
:102180001306F00F8145014582971703FFFF670093
:1021900043F71747FF1F130727B718439745FF1F3C
:1021A00083C585C69747FF1F938787C483468703E8
:1021B000034697036397D5009747FF1F2386C7C43D
:1021C000828083C587010347A7036317B60097473B
:1021D000FF1F238BE7C2828003C687016317C700F6
:1021E0009747FF1F2382D7C2828083C687011307C8
:1021F00050026319D700930760021747FF1F23059A
:10220000F7C0828083C68701130660026315D6007B
:1022100093077002DDB783C7870155BF9747FF1F3C
:10222000938707BDD44B0947638DE6081703FFFF6B
:10223000E702E3EA1749FF1F1309C9B83E84834741
:102240000900918B9DCFB7E4040083A7041D8297FA
:1022500083A7441C1745FF1F130545B7829783A723
:10226000841C81461746FF1F034646B88145014539
:10227000829721C583470900ED9B1747FF1F230362
:10228000F7B48347040093F7F70F85CB91471747BF
:10229000FF1F2329F7B697000000E78080EB970027
:1022A0000000E78040EFB7E70400BC4F414691458E
:1022B0001745FF1F034545B482971703FFFF6700CB
:1022C00043E482801703FFFFE70263E18D4741117A
:1022D0006306F504C5476308F50285476310F502F8
:1022E0009747FF1F2384A7B2B7E70400BC4B9305B1
:1022F00000101745FF1F034525B0829741011703C2
:10230000FFFF670003E085471747FF1F2300F7B073
:10231000B7E70400BC4B93050020E1BF9747FF1FC0
:10232000938707ADD44B1147638DE600B7E70400F0
:1023300083A7071D8297B7E70400BC4B93050004F1
:102340004DBF05491747FF1F232E27AB83C7070043
:1023500032C62E8493F7F70FD5D3B7E4040083A7D2
:10236000041D7D141374F40F8297E37689FCB24543
:10237000994703C61500E3F0C7FCFC44090617455E
:10238000FF1F1305E5A88297BC4893050008174571
:10239000FF1F034565A6829779BF1703FFFFE7027A
:1023A00003D41747FF1F1307A7A44047184B1C402F
:1023B0009746FF1F23A4F6A46316E4001747FF1FE8
:1023C0002320F7A4130584FE9790FFFFE78060A603
:1023D000035564FF9780FFFFE780E06E97A0FFFF43
:1023E000E78060D01703FFFF6700A3D11703FFFF4B
:1023F000E702E3CE9747FF1F9387879FD84BDC47C1
:1024000089C797000000E78080F985471747FF1FBD
:10241000232AF79E9747FF1F9387078F9C439305B7
:1024200000021745FF1F0345259D83C787031747F4
:10243000FF1F230BF79CB7E70400BC4B82971703E1
:10244000FFFF670003CC9747FF1F23A5A79A828051
:102450001703FFFFE70203C737E404007C4CA145E4
:102460001745FF1F0345459982977C48A1451745AD
:10247000FF1F034565989744FF1F938464978297D5
:10248000DC4489EB97000000E78080D91703FFFF49
:10249000670083C603D567FF9780FFFFE780A062D0
:1024A000AA896DD1D84891476310F7027C4C9145B9
:1024B0001745FF1F0345459482977C489145174572
:1024C000FF1F03456593829703A9490103D40901BE
:1024D0008947B7E904001747FF1F2325F79283A711
:1024E000091D21044204829783C784011715FF1F29
:1024F0001305C50361191717FF1FA309F70283A767
:10250000491C418082979747FF1F2381079083A72B
:10251000C91C814609469375F40F4A85829711E9D3
:102520009747FF1F83C7C79E89C79700FF1FE78094
:10253000606CB7E70400BC4F2146A1451745FF1F5B
:102540000345858B829799B71703FFFFE70223B9ED
:1025500093F7052001112E8481CF97000000E780BA
:1025600020E91345042005611703FFFF670063B9E5
:1025700093F70510A9CF9744FF1F93846487DC4825
:1025800097000000E78020C11737FF1F1307C777A8
:10259000184383C78401034787036318F700DC44AB
:1025A00089C797000000E78080DF85471747FF1F36
:1025B000232AF784B7E70400BC4B930500021745B4
:1025C000FF1F0345658382971345041069BF93F786
:1025D0000508BDC79747FF1F83C79783E9171946AB
:1025E0009745FF1F9385E5821305D10093F4F70FFC
:1025F0001749FF1F0349C98197C00000E780404089
:1026000093970401C1831747FF1F1307E780231D1A
:10261000F100231CF1009737FF1F9387677D3ACEA7
:102620003ACAD8432306010009CBDC43931589013C
:1026300054080D46E185680082971345040825B7C4
:1026400093F72500A5C39737FF1F9387677AD84B69
:1026500089476306F7029737FF1F83C7A77613F7EB
:10266000270011EF918B99CFB7E70400BC4F1306F9
:10267000000A89451735FF1F0345057882971345E2
:102680002400D5B59737FF1F938707689C4383C7FE
:1026900087031737FF1F2309F77697000000E780AD
:1026A00060DBF1BF93F7050281CB97000000E78064
:1026B00060DA1345040245BD93F7850081CB97008E
:1026C0000000E780E0D21345840071BD93F7150048
:1026D00081CB97000000E780A0B41345140061B5DA
:1026E00093F7450081CB97000000E78060B3134566
:1026F000440095BD93F7050495C39737FF1F83C723
:10270000276F91CB97000000E780A0A4914717376F
:10271000FF1F2329F76E13450404B1B593F7050194
:102720000145E38207E49737FF1F9387676CD84B17
:1027300091476310F7049737FF1F9387A7689C435F
:1027400013D727008583D98F858B91E7B7E70400DE
:1027500083A7071D8297B7E70400FC4F9145173503
:10276000FF1F03456569829785471737FF1F232B96
:10277000F76813450401C5BB9737FF1F238AA77865
:1027800082801703FFFFE70283959737FF1F23A778
:1027900007669737FF1F23A5076685471734FF1F76
:1027A000130484561737FF1F232EF7641C4083C77A
:1027B00087031737FF1F2309F7649790FFFFE78010
:1027C000A08F29C59717FF1F23A6A7D61C40170562
:1027D00000001305A5D783C787031737FF1F2305FD
:1027E000F7621717FF1FA303F7D49737FF1FA381C3
:1027F0000760B7E7040083A7070882979737FF1F92
:10280000238CA75E1703FFFF6700A38FB7C7898ECE
:10281000938767ED1717FF1F232EF7D045BF173794
:10282000FF1F0347E75C795555E79737FF1F9387ED
:10283000275C03C7170005079736FF1FA38AE65AD0
:1028400003C717008D463377D7029736FF1FA38142
:10285000E65A83C617001737FF1F1307E74A1843C6
:1028600093F6F60FA9EE834787031737FF1F230D53
:10287000F75885471737FF1F230CF7569737FF1F69
:10288000938747549C430145998BA9E71703FFFFA2
:10289000E702E38437E404007C48C1451735FF1F95
:1028A0000345855582973C4885451735FF1F0345ED
:1028B000A554829701451703FFFF6700838483C7F0
:1028C000170085466395F6008347970379BF8347D2
:1028D000A70361BF82809737FF1F83C76751A1CFCE
:1028E00017F3FEFFE702A37F37E404009737FF1FCB
:1028F000238007507C4885451735FF1F0345C54F8A
:1029000082977C4C91451735FF1F0345E54E829712
:102910007C4891451735FF1F0345054E82973C487B
:10292000C1451735FF1F0345254D8297014517F314
:10293000FEFF6700037D7955828017F3FEFFE702F3
:10294000037A2A84035565FF9780FFFFE780A0176D
:102950009737FF1F9387C749D847BE841DEF9790CD
:10296000FFFFE78080779C48232004009DEB97378A
:10297000FF1F23A787489737FF1F23A18748B7E783
:102980000400BC4B89451735FF1F0345E546829778
:10299000014517F3FEFF6700C376630A87001843FB
:1029A00075BF80C39737FF1F23AC8744C9BF7955D4
:1029B000CDB717F3FEFFE70283729737FF1F9387A8
:1029C000675588432326050023240500510597A059
:1029D0000000E780C03317F3FEFF6700837217F330
:1029E000FEFFE702C36F1734FF1F1304A4521C40FD
:1029F000411199CF9C472302B5002AC61CC19700FC
:102A00000000E78040FB1C409C4B99C332458297F5
:102A1000410117F3FEFF6700C36E17F3FEFFE702E5
:102A2000036C4111444D328532842EC69790FFFFCE
:102A3000E780C0522AC422859790FFFFE780205488
:102A400003A84400630C0800B245835744001840B3
:102A5000224683D54500AA8626850298410117F3B0
:102A6000FEFF6700036A17F3FEFFE7024367404D6E
:102A70001DC808C097050000938565031305440130
:102A800097A00000E78040169737FF1F938787487D
:102A90009C43014589E79737FF1F23AD874617F30E
:102AA000FEFF670003667D55DDBF17F3FEFFE702FB
:102AB0000363011168009305F00F02C602C802CA41
:102AC00002CC02CE97000000E780A0F1056117F369
:102AD000FEFF670003639737FF1F9387A7439C435D
:102AE000D847A1679D076319F70217F3FEFFE702B6
:102AF000035F011132859790FFFFE7802046230A8C
:102B0000A1008145680097000000E78080ED056125
:102B100017F3FEFF6700E35E82809737FF1F9387FE
:102B2000673F9C43D847A167938777036319F702F0
:102B300017F3FEFFE702A35A011132859790FFFFBA
:102B4000E780C041230AA10081456800970000008A
:102B5000E78020E9056117F3FEFF6700835A828052
:102B60009737FF1F9387073B9C43D84795476316CA
:102B7000F70417F3FEFFE702835601113285328412
:102B80009790FFFFE780803D230AA1002285979060
:102B9000FFFFE780C03E83574400231BA10081450F
:102BA0003ECC1C4068003ECE97000000E78060E30A
:102BB000056117F3FEFF6700C3548280930785FF0A
:102BC0008DC38327C5FF91CFDC4B81CF17F3FEFF69
:102BD000E702E350032585FF829717F3FEFF6700A6
:102BE0004352828017F3FEFFE702634F2A84328547
:102BF0009790FFFFE7808036BD4763EBA70018443E
